:020000040800F2
:1000000000070020F1010008012A00089D290008CE
:10001000DD2900089D290008BD290008F30100081A
:10002000F3010008F3010008F30100081D3E000879
:10003000F3010008F3010008F3010008F3010008D0
:10004000F3010008F3010008F3010008F3010008C0
:10005000F3010008F3010008C54C0008ED4C00084E
:10006000154D00083D4D0008654D0008F3010008DE
:10007000F3010008F3010008F3010008F301000890
:10008000F3010008F3010008F30100081929000832
:100090004529000871290008F30100088D4D00086A
:1000A000F3010008F3010008F3010008F301000860
:1000B000894E0008F3010008F3010008F30100086D
:1000C000F3010008F3010008F3010008F301000840
:1000D000F3010008F3010008F3010008F301000830
:1000E000014E0008F3010008F3010008F3010008C5
:1000F000F3010008F3010008F3010008F301000810
:10010000F3010008F3010008F3010008F3010008FF
:10011000F3010008F3010008F3010008F3010008EF
:10012000F3010008F3010008F3010008F3010008DF
:10013000F3010008F3010008F3010008F3010008CF
:10014000F3010008F3010008F3010008F3010008BF
:10015000F3010008F3010008F3010008F3010008AF
:10016000F3010008F3010008F3010008F30100089F
:10017000F3010008F3010008F3010008F30100088F
:10018000F3010008F3010008F3010008F30100087F
:10019000F3010008F3010008F3010008F30100086F
:1001A000F3010008F3010008F3010008F30100085F
:1001B000F3010008F3010008F3010008F30100084F
:1001C000F3010008F3010008F3010008F30100083F
:1001D000F3010008F3010008F3010008F30100082F
:1001E00009120008000000000000000000000000EC
:1001F00002E000F000F8FEE772B6374880F30888A6
:10020000364880F3098836483649086040F20000D5
:10021000CCF200004EF63471CEF200010860BFF35C
:100220004F8FBFF36F8F40F20000C0F2F0004EF628
:100230008851CEF200010860BFF34F8FBFF36F8F7C
:100240004FF00000E1EE100A4EF63C71CEF20001D4
:100250000860062080F31488BFF36F8F04F022FB40
:1002600004F00CFC4FF055301F491B4A91423CBF33
:1002700041F8040BFAE71D49184A91423CBF41F886
:10028000040BFAE71A491B4A1B4B9A423EBF51F82E
:10029000040B42F8040BF8E700201849184A914271
:1002A0003CBF41F8040BFAE704F000FB04F0ECFB60
:1002B000144C154DAC4203DA54F8041B8847F9E797
:1002C00000F042F8114C124DAC4203DA54F8041B12
:1002D0008847F9E704F0E8BA00070020002300206F
:1002E0000000000808ED00E00001002000070020E9
:1002F00010520008002300208023002080230020CB
:10030000684D0020E0010008E4010008E401000855
:10031000E40100082DE9F04F2DED108AC1F80CD052
:10032000C3689D46BDEC108ABDE8F08F002383F3BF
:1003300011882846A047002003F0DAFEFEE703F00C
:100340005FFE00DFFEE70000F8B500F065FF04F097
:100350003DFA064604F092FA0746A8B92C4B9E4295
:100360002BD001339E422BD026F0FF02294B9A421C
:1003700003D0054641F2883408E0F0B200F046FEB2
:100380003D4642F2107401E00546002400F044FEB0
:1003900008B10024254601F03FFBA0B941F28833A3
:1003A0009C4216D017B11C4B9E4216D1002004F07F
:1003B00019FABDB900F0ACFE26E005460024E5E7D9
:1003C00000240125E2E7032000F030F80024254650
:1003D000E8E74FF47A740125E4E704F047FA0024D3
:1003E0002546E3E700F040F8E4E700F0E3FE4FF4D1
:1003F0007A7003F085FE002CF7D002F009FB401B59
:10040000A042F2D900F030F802F002FB0546F2E714
:10041000010007B0000008B0263A09B0302383F38A
:100420001188854680F308880847704708B50C4B4B
:100430001870032806D8DFE800F00A06020E022032
:1004400000F056FF08BD022000F048FFFAE7054B18
:1004500000225A60F6E7034B00225A60F2E700BF21
:10046000802300208423002008B501F0D5FA03463C
:1004700068B9072B0FD89A0002F1006202F58032AA
:100480001268B2F1FF3F05D00133DBB2F1E7032080
:10049000FFF7CCFF08BD174B5A68013B9A42F9D9C8
:1004A000154B9B6803F1006303F580339A42F1D248
:1004B00004F0AEF904F0C0F9002000F0C9FE0220FB
:1004C000FFF7B4FF0D4B1A6C00221A64196E1A66FE
:1004D000196E596C5A64596E5A665B6E72B6054B4A
:1004E0004FF0E022C2F8083D59681868FFF796FF00
:1004F000D0E700BF000001080023002000380240C0
:10050000094A136899B21B0C49F2690000FB0133D8
:100510001360064B186882B2000C44F2506101FB74
:100520000200186080B270471823002014230020B6
:1005300010B50446FFF7E4FFB0FBF4F304FB13002F
:1005400080B210BD10B40346002202604260826097
:10055000C260044C07CC186059609A605DF8044B87
:10056000704700BF107AFF1F70B50E4614461D4637
:1005700002F05AFF60B9022D33D1012C01D00020C6
:1005800030E019A3D3E90023C6E90023012029E0C4
:10059000282C1FD00CD8012C15D0052C06D114A363
:1005A000D3E90023C6E9002301201BE0002019E065
:1005B000302C06D110A3D3E90023C6E90023012083
:1005C00010E000200EE00EA3D3E90023C6E90023CB
:1005D000012007E00CA3D3E90023C6E90023012092
:1005E00000E0002070BD00BF401DA12026812A0B25
:1005F000F017304A39059E5678F6339F93CACD8D51
:100600009E6AC421818A46EE26417272DF25D7B7E1
:1006100070B58AB006460D4602F0FAF904464FF46A
:10062000C870FFF785FF044404F51674184B1C606E
:10063000EB7E23B9174B00221A700AB070BD05A9D2
:10064000284600F0A3FF0028F7D101A8FFF77AFFA2
:100650009DF81640224601A90DF1170004F07AFC1E
:1006600048B90F2C0BD80B4B1C70094A1368A3F523
:1006700016731360E1E7074B00221A70DDE79DF85F
:1006800014100029D9D0304602F0C6FED5E700BFCD
:10069000A03300209D3300202DE9F041ADF5507DC1
:1006A00007460E460EAC4FF4C4720021204600F0FF
:1006B0003DFE02F0ADF9304BA3FB00239B092F4A0E
:1006C000136007CA84E80700022323744FF0000870
:1006D00084F811800DF15A00FFF734FF042384F8E9
:1006E00020306E2384F821300DF1180C244D0FCDED
:1006F000ACE80F0095E80F00ACE80700ACF800305C
:100700001D2384F832310DF1180CBCE80F00CDF830
:100710006B01CDF86F11CDF87321CDF87731BCE8BE
:100720000700CDF87B01CDF87F11CDF883219CF82F
:1007300000308DF8873171AD01222946204600F046
:1007400049FE80B205900495CDF80C80B37E0293EB
:1007500006F1190301930123009305A3D3E90023B4
:10076000F17E384602F016FF0DF5507DBDE8F081B0
:100770009E6AC421818A46EED34D62108C230020EC
:10078000B84F0008F0B5FDB006460D462B4B1C7A5D
:100790006CBB07A9284600F04BFF002845D19DF807
:1007A0001D70C82F41D84FF4A6620021234800F0E5
:1007B000BDFD032C0AD82202204B4FF48A7101FBA5
:1007C0000433C3F8E4200134E4B2F2E71B4C3A46A8
:1007D0000DF11E0104F1090000F094FDE21900235F
:1007E00053729DF81C3023720BB9EA7E227281226B
:1007F00000213AA800F09AFD5BAC012221463AA8FC
:1008000000F066FF80B20590049400230393AB7E52
:10081000029305F1190301932823009305A3D3E95B
:100820000023E97E304602F0B5FE7DB0F0BD00BF8A
:10083000AFF3008026417272DF25D7B7D433002092
:10084000134BB3F82C35834200D9704710B50446DA
:10085000002100F027FD01340D4BA3F82C450C4B73
:10086000B3F82C0500F002FD88B1094BB3F82C0554
:1008700000F00EFD58B9064C0021B4F82C0500F02C
:1008800011FDB4F82C350133A4F82C35E7E710BD81
:10089000D43300202DE9F041F0B00646274C94F8FF
:1008A000D8304FF48A7505FB004585F8DC30002709
:1008B00085F8E870D82239463AA800F037FD04F1EF
:1008C0000908404600F028FDC2B28DF8F020D5F8A6
:1008D000E4303A933B9741460DF1F10000F012FDF0
:1008E00006AD012229463AA800F02AFF80B2059001
:1008F0000495012303930823029304F1D803019381
:10090000302300930BA3D3E90023217A0C4802F093
:1009100041FEB84203DC002070B0BDE8F08102F077
:1009200077F84FF48A7202FB0646C6F8E000012011
:10093000F2E700BF78F6339F93CACD8DD433002001
:10094000A433002038B502F063F80546002408E01F
:100950000532B3EB420F02D3FFF79CFFF8B101342D
:10096000E4B2032C1BD80E4B93F8D900204400F0BE
:1009700003004FF48A7202FB003393F8E830002B37
:10098000EDD1074B02FB0033D3F8E030002BE3D06E
:10099000EB1A034A1268F92ADAD8FA22D8E738BDE6
:1009A000D4330020F0B58FB000230A938DF8343093
:1009B0008DF835300B930C9300242746002C46D13C
:1009C00001238DF80C3000238DF80D3041F2E80240
:1009D00004FB02F220495518525896680020002165
:1009E000CDE900010DF10D0203A92846B0479DF89D
:1009F0000C604EB3194A536983F48053536100234A
:100A0000069307930893099341F2E80304FB03F369
:100A1000114AD3585F690DF10E0304AA0AA92846AA
:100A2000B84707AB0BAA92E8030083E803009DF8E0
:100A300034308DF824300A9B0693DDE9042306A99F
:100A4000074802F0AFFF37460134E4B2B6E7002FA3
:100A5000B2D10FB0F0BD00BF103900200008024035
:100A6000A433002010B586B0BDF828400494099C3A
:100A700003949DF8204002940193009202460B4695
:100A8000024802F027FD06B010BD00BFA4330020CD
:100A900010B58AB0244802F0C7FC08B10AB010BDF6
:100AA00001F0B6FF214B1B689842F7D301F0B0FF6D
:100AB00004464FF4C870FFF73BFD044404F5167478
:100AC0001A4B1C6000238DF82030194B1B7813B98A
:100AD00001238DF8203004A8FFF734FD144B19785A
:100AE000C1F11004E4B2062C00D90624224604AB5E
:100AF00019440DF1210000F005FC0134029408AB0B
:100B00000193182300930B4B012205A1D1E90001A9
:100B1000FFF7A8FF064B00221A70BFE7AFF3008073
:100B2000401DA12026812A0BA4330020A0330020E1
:100B30009D3300209C33002010B586B001F068FF83
:100B40000F4BA3FB00239B090E48036004AC01225A
:100B5000214600F0F3FC80B2029001941823009328
:100B6000094B40F2551204A1D1E90001FFF77AFFC9
:100B700006B010BDAFF30080F1C6A7C1D068080F62
:100B8000D34D62108C2300200839002010B5024696
:100B90000B46094C204602F035FD204602F044FC8D
:100BA00038B1064B1B7A2BB10322054B5A71FFF764
:100BB000C3FF10BD0222F8E7A4330020D433002085
:100BC0008C230020012800D0704738B54FF6FF7302
:100BD000994200D038BD0025084C002D07DB204687
:100BE00001F034FA04F587540834013DF5E7044A6E
:100BF0000449002004F08AF9ECE700BF1039002016
:100C0000304A0020090C000838B50F4C0F4B9C42AD
:100C100019D0A4F58753A3F108040D4A43F8082C12
:100C200041F26C03E21812793AB9E5582DB1284621
:100C300000F000FF284601F059F804F58250183002
:100C400000F0F8FEE2E738BDF84900201039002036
:100C500018500008F0B587B0254802F0C7FC0028FE
:100C600039D00446002302938DF814308DF81530E6
:100C700003930493027B8DF8142003AA4068A168B3
:100C800003C2226842F0004202921D461C46D5B9BA
:100C900041F2E80305FB03F3164A9E189B581F69AF
:100CA00001F0BAFE144A82184FF00003009341F19C
:100CB000000302A93046B8470028C8BF44F0010429
:100CC0000135EDB2E3E744B90C4B1B78072B0BD889
:100CD00001330A4A137007B0F0BD054802F08AFCE0
:100CE000064B00221A70B7E7014802F083FCF2E7D6
:100CF000A43300201039002040420F0009390020A1
:100D0000CA7EA04B1B7A9A4240F03B812DE9F04706
:100D100000AF08460024032C0CD89A4B4FF48A727B
:100D200002FB043393F8DC20437E9A4211D0013455
:100D3000E4B2F0E7002373B9924B1B68FA3340F634
:100D4000B832934200D913468E4A1360BD46BDE8BF
:100D5000F0870123EFE74FF48A7104FB01F1E031E2
:100D6000884B19440A3100F021FD0028EED1854B53
:100D70004FF48A7202FB0434012384F8E83001F056
:100D800047FED4F8E030C31A192B05D940F6B83223
:100D9000934202D9134600E019237A4AD2ED007A31
:100DA000F8EE677A9FED787A27EE877A07EE903A29
:100DB000F8EE677ADFED756A67EEA67A77EE277A46
:100DC000FCEEE77AC2ED007A3CE013464FF48A72FB
:100DD00002FB0535002385F8E830C5F8E030C5464C
:100DE000684B5B689B0A0133694A1381AEE70020B8
:100DF00042F8040B013B002BF9DA2246304600F0A2
:100E000081FA604B5B68002B4BD05E4B93F8D200AD
:100E100000F02CFA8246002847D05A4BD3F8D43041
:100E2000002B4ED0574BD3F8D430234453454ED8E3
:100E30005FFA89F23146534B586800F081FA002876
:100E40004CD1C5464F4B93F8D9504FF48A7202FBF0
:100E5000053393F8E830002BC2D0E846494A4FF4F6
:100E60008A7303FB0523D3F8E41053689942ACD18D
:100E700044494FF48A7305FB03F3CA18B2F8EC40F7
:100E8000E21C4FEA9209E03319440E314A4609F157
:100E9000FF3392000732D208A8EBC20295466E4695
:100EA000A9E7012000F0D4F9AFE70024354B1C720C
:100EB00000F002FA204600F0CBF9354B0B221A81E4
:100EC0008DE7304B93F8D200FFF7BAFCAAE72D4B21
:100ED00093F8D2000130FFF7B3FCA9E7294B5A6819
:100EE00022445A60D3F8D4602644C3F8D46093F8FF
:100EF000D20000F0BBF986420BD3224B93F8D220EC
:100F0000013283F8D220D3F8D420A2EB0A02C3F82E
:100F1000D420FF2C23D91B4C4FF48A7303FB0545C7
:100F2000002385F8E830C5F8E030D5F8E43003F563
:100F30008063C5F8E43094F8D900FFF7ABFCFFF705
:100F400089FE94F8D93001335A4203F0030302F0CA
:100F5000030258BF534284F8D930C54672E70024D3
:100F6000084B1C7200F0A8F9204600F071F900F05F
:100F700053FD074A108108B1C546E7E6FFF774FA4A
:100F8000FAE77047D43300206666663FCDCCCC3D8F
:100F90008C23002038B505460C4602F045FA50B1C6
:100FA000E38A282B1CD014D8012B0FD121462846C8
:100FB000FFF772FB0CE0237E022B09D1E38A012BA1
:100FC00006D121462846FFF723FB01E0052B0CD074
:100FD00038BD302BFCD121462846FFF791FEF7E7BC
:100FE00021462846FFF7CEFBF2E7BFF34F8F0549B6
:100FF000CA6802F4E062044B1343CB60BFF34F8F27
:1010000000BFFDE700ED00E00400FA05014B187099
:10101000704700BF9823002030B585B04FF00053D3
:101020001A68334B9A4203D14FF00053587D88B968
:1010300003F02EFC044650B12E4A136C43F00073AB
:1010400013642D4B9A6D2D4B9A4227D000242046D5
:1010500005B030BDFFF7DAFF4FF000531A7D284B83
:101060001A720023032B0AD81902254A4FF48A70FA
:1010700000FB0322C2F8E4100133DBB2F2E74FF0C9
:101080000054C92204F116011E4800F03BF9E02289
:101090000021204600F04AF90124D8E7164B1B6EC8
:1010A00023B37F2B01D90024D1E7174A01AB106885
:1010B0005168926807C3032101A800F0DDFB0E4BC5
:1010C0005B6D984201D00024C1E70B4B1B6D994228
:1010D00001D00024BBE7084D0023AB6595F8600004
:1010E000FFF794FFEA6D094B1A60B0E70024AEE702
:1010F0009AAD44C500380240006600405041A0B09F
:10110000D4330020DD330020586600401023002037
:1011100030B583B000F080FC1D4B188102225A715B
:10112000002474B941F2E80304FB03F319481A5888
:1011300055680122184909681844A8470134E4B2E7
:10114000EFE700230193154B0093154B4FF48052AA
:101150001449154802F044F9144B197899B901F073
:1011600057FC04464FF4C870FFF7E2F9044404F555
:1011700016740F4B1C6003F081FB10B1044B0F225F
:101180001A8103B030BD084802F046F9E7E700BF16
:101190008C2300201039002010230020690500084E
:1011A000950F00089C230020A433002098230020E2
:1011B000A033002008B50CE0114B186001F02CFCA6
:1011C000FFF7E4FC13E0C82002F09AFF0D4B1B7AF6
:1011D000A3B1FFF73FFDFFF7E5FBFFF759FC01F077
:1011E00017FC074B1B68C31AB3F57A7FE4D2054B93
:1011F0001B7A002BE7D0FFF7A5FBE4E708BD00BF93
:1012000004390020D433002008B54FF6FF710120C7
:10121000FFF7D8FC08BD00BF10B503F0A3F90A4BD7
:101220001880002406E003F073F90444074A1368A9
:1012300001331360B4F5803F05D2034B1B88034A8A
:1012400010688342EFD810BD244A0020F8490020DE
:1012500008B503F0E1F908BD08B5920000F100609F
:1012600000F5803003F0D4F908BD00BF08B5064B87
:101270001B88064A12689B1A834201D8002008BDC9
:10128000104403F045F9FAE7244A0020F849002009
:1012900008B5034B1B68184403F066F908BD00BF8E
:1012A000F849002008B5034B1B68184403F074F993
:1012B00008BD00BFF849002008B5074B93F824305B
:1012C0000BB9012008BD0449002381F8243008220D
:1012D000086AFFF7C1FFF5E7FC490020022800D0AB
:1012E0007047024B4FF080529A61F9E700080240C4
:1012F000022800D07047024B4FF480529A61F9E700
:1013000000080240002304E011F803C000F803C005
:1013100001339342F8D370470346002000E00130C8
:1013200013F9012B002AFAD1704700BF034602E0EF
:1013300003F8011B624602F1FF3C002AF8D1704716
:101340002DE9F843814688461546214B93F8243011
:1013500033B31F4A126A02EB8303834220D0FFF7A4
:10136000ABFF0346E0B930E0194E96F82400C0F117
:101370000804AC4228BF2C46E4B2A7003A464146D6
:1013800006EB8000FFF7BEFFB944B8442D1BEDB259
:1013900096F824301C44E4B286F82440082C0DD082
:1013A00095B10B4B93F82430002BDDD10848C0F8E1
:1013B00020902022FF21FFF7B9FFD5E7FFF77CFF40
:1013C00003460028ECD100E001231846BDE8F8836D
:1013D000FC4900202DE9F04383B007460E469146B4
:1013E00040F2791200213046FFF7A0FF3B46202251
:1013F0000021304602F052FA3B1D022220213046E5
:1014000002F04CFA7B1D03222221304602F046FAFC
:10141000BB1D03222521304602F040FA07F10803E4
:1014200010222821304602F039FA07F11003082271
:101430003821304602F032FA07F111030822402128
:10144000304602F02BFA07F11203082248213046F9
:1014500002F024FA07F1140320225021304602F052
:101460001DFA07F1180340227021304602F016FAE7
:1014700007F1200843460822B021304602F00EFA58
:1014800007F121030822B821304602F007FAC025EF
:10149000002409E008EB0403023308222946304601
:1014A00002F0FCF9083501340F2CF3D998F812300A
:1014B0008DF807300DF1070308222946304602F067
:1014C000EDF905F1080400259DF807309D420BD287
:1014D00005F110034344033308222146304602F04D
:1014E000DDF908340135EFE797F83231502B28BF8A
:1014F00050238DF80730B9F1000F10D000259DF86A
:1015000007309D4214D205F598733B4403330822FB
:101510002146304602F0C2F908340135EFE70DF1FB
:10152000070307222146304602F0B8F90734E5E701
:10153000E01DC00803B0BDE8F08300BF38B5054624
:101540000C4600212160C4F80310034620222046E7
:1015500002F0A4F92B1D02222021204602F09EF960
:101560006B1D03222221204602F098F9AB1D0322B5
:101570002521204602F092F905F1080310222821C6
:10158000204602F08BF9072038BD00BFF0B583B0CC
:1015900007460D46047F14B1838A122B3CD8009570
:1015A000002307221946384602F076F86B1C009398
:1015B000002301220721384602F06EF854B1BB8A9D
:1015C000DB00083BDB08AB700826AB78102B26D875
:1015D000002414E0AB1C00930023052208213846A8
:1015E00002F05AF80D26F0E72B190333009300237D
:1015F00008223146384602F04FF808360134AB78FD
:101600009C42F1D300243CB90736F6083B7F43B136
:10161000BC8AA41B18BF0124204603B0F0BD0124DE
:10162000F1E7BC8AB4422CBF00240124F4E700BFD8
:101630002DE9F04182B006468846047F14B1838AC2
:10164000CA2B38D8CDF8008000230822194630462E
:1016500002F022F808F1010764B1B38ADB00083B0D
:10166000DB0888F80130082598F80130C82B26D807
:10167000002413E00097002308221146304602F0B0
:101680000BF81025F0E73B190133009300230822E3
:101690002946304602F000F8083501343B789C4278
:1016A000F1D300243CB90735ED08337F4BB1B48A40
:1016B000641B18BF0124204602B0BDE8F08101245C
:1016C000F0E7B48AAC422CBF00240124F3E700BF4A
:1016D000F0B583B006460F461446812200213846F5
:1016E000FFF724FE334608220021384602F0D6F8E0
:1016F000737896F90120002A05DB8DF8073024B1B4
:101700000825002413E07F23F7E70DF107030722E4
:101710000821384602F0C2F80F25F2E733190233E8
:1017200008222946384602F0B9F8083501349DF8F8
:1017300007209442F2D3E81DC00803B0F0BD00BFFB
:10174000F0B583B004460E461546CE220021304641
:10175000FFF7ECFD234628220021304602F09EF8D8
:1017600004F10807237AC82B28BFC8238DF8073057
:1017700015B12825002411E00DF1070308222821C6
:10178000304602F08BF83025F4E73B19013308228C
:101790002946304602F082F8083501349DF80730BA
:1017A0009C42F2D3E81DC00803B0F0BDF0B583B091
:1017B00007460E46047F1CB1838AB3F5827F35D875
:1017C0000096012310220021384601F065FF5CB12C
:1017D000BB8ADB00103BDB08738010257388B3F5F0
:1017E000807F26D8002414E0B31C00930023092234
:1017F0001021384601F050FF1925EFE73319043363
:101800000093002308222946384601F045FF083599
:10181000013473889C42F1D300243CB90735ED08AC
:101820003B7F43B1BC8A641B18BF0124204603B030
:10183000F0BD0124F1E7BC8AAC422CBF0024012496
:10184000F4E700BF00B58E460AE040F3000C0949FA
:101850000CEA010181EA50000133DBB2072BF4D915
:101860001346013A23B11EF8013B58400023F5E727
:101870005DF804FB2083B8ED30B583B004460B4619
:101880004FF0FF30014620E0001849410133DBB240
:10189000072B0BD80029F7DA10EB000C41EB010203
:1018A00010488CEA000010495140EFE70EF1010E9C
:1018B0005FFA8EFEBEF1030F06D801AB13F80E30AF
:1018C00081EA03610023E3E72B465D1EADB22BB135
:1018D00054F8043B01934FF0000EEBE7C043C943BB
:1018E00003B030BD9336EAA9EBE1F042F0B583B026
:1018F0001F4B6A4693E8030082E8030008231D4952
:101900001D4803F037FB30B304460369B3F5702F6D
:1019100023D8418B40F26E42914220D100F118074A
:10192000164A024402F110018B421BD39B1AA3F109
:10193000100511490020FFF785FF06462A46394663
:101940000020FFF77FFFA368B3420DD1E368834215
:101950000CD1002004E00A2002E00B2000E00C2063
:1019600003B0F0BD1020FBE70D20F9E70D20F7E7ED
:10197000D84F0008DCFF0E00000001080800FFF748
:10198000F0B583B0204B6A4693E8030082E8030079
:1019900008231E491E4803F0EDFA38B304460369D4
:1019A000B3F5702F24D8B0F8661040F26E42914221
:1019B00020D100F16407174A024402F15C018B4216
:1019C0001BD39B1AA3F15C0511490020FFF73AFFD6
:1019D00006462A4639460020FFF734FFA368B34283
:1019E0000DD1E36883420CD1002004E00A2002E01C
:1019F0000B2000E00C2003B0F0BD1020FBE70D2011
:101A0000F9E70D20F7E700BFE44F000890FF0E0054
:101A1000000001080800FFF710B5FFF767FF044654
:101A200008B9204610BDFFF7ABFF0028F9D10446E6
:101A3000F7E700BF10B50446037C0BB1204610BD8C
:101A4000006803F07FFAF9E7BFF35B8FC368BFF369
:101A50005B8FBFF35B8F8268BFF35B8F9A4208D9BD
:101A60004268BFF35B8F8068BFF35B8F101A184426
:101A70007047BFF35B8F8068BFF35B8F181A7047A6
:101A8000BFF35B8F0023C360BFF35B8FBFF35B8F3C
:101A90008360BFF35B8F70470346406800B97047AF
:101AA000BFF35B8F9A68BFF35B8FBFF35B8FD9681F
:101AB000BFF35B8F914209D35868BFF35B8FDB683C
:101AC000BFF35B8FD21A013A1044E8E70020F4E735
:101AD00038B505460C46FFF7B7FFA04201D20020FB
:101AE00038BDBFF35B8FA968BFF35B8F0C44696897
:101AF000B4FBF1F301FB1344BFF35B8FAC60BFF3A6
:101B00005B8F0120ECE700BF70B504460E4615461A
:101B1000FFF7C2FFA84200D3284608B9002070BDD5
:101B20002368BFF35B8FE268BFF35B8F13443360BE
:101B30006268BFF35B8FE368BFF35B8FD11A8842A3
:101B400007D971602168B1609B1A1844F0600220C7
:101B5000E5E770600120E2E738B505460C46FFF77F
:101B60009BFFA04201D2002038BDBFF35B8FE96824
:101B7000BFF35B8F0C446968B4FBF1F301FB1344C2
:101B8000BFF35B8FEC60BFF35B8F0120ECE700BF1E
:101B90002DE9F04385B0814688466946FFF7B4FFDA
:101BA0000746002425460EE004AB03EBC40656F8B6
:101BB0000C2C08EB050156F8100CFFF7A3FB56F8A8
:101BC0000C3C1D440134A742EEDC29464846FFF791
:101BD000C3FF284605B0BDE8F08300BFBFF35B8FAD
:101BE000C368BFF35B8FBFF35B8F8268BFF35B8F0C
:101BF0009A4210D94368BFF35B8F8268BFF35B8F53
:101C00009B1A0B6073B10368BFF35B8F8068BFF3EF
:101C10005B8F18447047BFF35B8F8268BFF35B8FA5
:101C20009B1AEEE700207047F0B583B007460E46DA
:101C30001546FFF709FF04460190A84200D32C4641
:101C400014B9002003B0F0BD01A93846FFF7C6FF64
:101C5000019B6BB1A34200D9019430600198706080
:101C6000A0420DD23B68B360241AF4600220E9E779
:101C70003B68336074600023B360F3600120E1E7E8
:101C80000120DFE72DE9F04184B088466946FFF77F
:101C9000CBFF0746002425460EE004AB03EBC40649
:101CA00056F80C2C56F8101C08EB0500FFF72AFB21
:101CB00056F80C3C1D440134A742EEDC284604B023
:101CC000BDE8F08138B50546FFF7DCFF0446014664
:101CD0002846FFF7FDFE204638BD00BF08B500B915
:101CE0000120012103F018F908BD00BF18B108B5A3
:101CF00003F028F908BD704710B5026854681A4609
:101D0000A04710BD0020704700207047704700BFFB
:101D1000002070470E20704700F5805090F8D800E2
:101D2000C0F34000704700BF00F5805090F9E0001C
:101D3000704700BF00F58050C0F8DC1001207047EC
:101D4000F0B583B0BDF820500C6814F0005F40F08F
:101D500089800C7B082C00F28880302484F3118861
:101D6000446AA66816F0806F0ED1A66816F0006F60
:101D70006BD1A66816F0805F02D04FF0020E05E02E
:101D8000002080F311885EE04FF0000EF4460E68EC
:101D9000002E5DDB76050EF1180E4FEA0E1E44F89C
:101DA0000E600E6816F0804F06D00CF11806360152
:101DB000A75947F00207A7510F7B0CF118064FEA0D
:101DC000061E04EB061677608E6804EB0C17C7F846
:101DD0008C614E68C7F8886154F80E6046F00106C1
:101DE00044F80E6041F2780E0EEB4C14044400EB04
:101DF0004C1CE644CEF80020CEF80430D1F800E0C8
:101E00004F688E68C4F808E0E76026618E89A68274
:101E10000CF5845C9CF8144065F300048CF81440C5
:101E2000C5F34006E4B266F341048CF81440E4B212
:101E30006FF3C3048CF81440002484F311880095D8
:101E400000F05AFE012003B0F0BD4FF0010E9DE7F7
:101E5000F60046F004060EF1180E4FEA0E1E44F886
:101E60000E609EE74FF0FF30EDE74FF0FF30EAE7FE
:101E700008B5302383F3118800F58050C06EFFF75A
:101E8000FFFD002383F3118808BD00BF70B5044631
:101E90000D4641F26C068059FFF7FEFD1F2801D860
:101EA000002070BD20222946A059FFF771FE20288E
:101EB00014BF00200120F4E72DE9F04188B0064668
:101EC0000D4617469846302383F3118800220023DD
:101ED000CDE900230024ADF8084003948DF81840A4
:101EE0008DF819400494059441F26C040059FFF7F1
:101EF000ABFD1F2806D8002070B980F3118808B008
:101F0000BDE8F081202269463059FFF7DBFE20282A
:101F100014BF00200120EFE703AB07CB2860696006
:101F2000AA601B88AB81DDE90023C7E90023BDF867
:101F30000830A8F80030002383F3118843463A465E
:101F40002946304600F076FDD9E700BF10B50246BD
:101F50003A4B42F8043B0023436053609360D360E4
:101F6000136153610246364C42F8284B8362137367
:101F70005373C36203639FED2F7B80ED0E7BA0F84C
:101F80004030436480F8503080F851308364C3643B
:101F900000F1580423464FF07F0C0DE09FED257BA8
:101FA00083ED007B00221A81DA601A765A761A6174
:101FB0005A6120330CF1FF3CBCF1000FEEDA00F562
:101FC0008252183200F580539C654FF48054DC65D2
:101FD00000241C665C664FF0010C83F868C0DA666A
:101FE00083F870C000F5835318334FF0020EBEF132
:101FF000000F11DB9C469FED0F7BACEC027B0022B7
:102000009A608CF80C208CF80D20DA601A619A61C5
:1020100020330EF1FF3EEAE700F5805383F8E0102D
:1020200011B9084B436210BD074800F0EBFC00BF3C
:10203000AFF30080000000000000000064500008C2
:102040001850000800640040F04F000810B5044626
:10205000034B19784A1C1A70FFF778FF204610BD11
:102060002C4A0020002977D070B582B00C46424B34
:10207000994211D90A234149B1FBF4FC013BDBB27F
:102080009E46581CBCFBF0F100FB11C131B1022B84
:1020900064D9013BDBB2F3E71123ECE7BCFBF0F0C2
:1020A000411EB1F5806F5CD2C3EBC30E1EF103017C
:1020B0004DD4C1F3C70C8DF800C0A3EB0C05EDB2F5
:1020C0008DF801500CF101064FF47A710CFB0111EF
:1020D000354491FBF5F189B2ADF80210B1F5617F9D
:1020E00018D9BEF1010E34D4CEF3C70E8DF804E03A
:1020F000A3EB0E03DBB28DF805300EF101054FF4B2
:102100007A710EFB01112B4491FBF3F3ADF806300D
:10211000019B00939DF800104B1C9DF80160334417
:1021200000FB03F3154DB5FBF3F3A3421BD10139BB
:10213000C9B20F2919D8D6B1082E1AD80138108083
:1021400000239370D170013E1671012007E0073122
:10215000AFE70EF1070EC7E700207047002002B07E
:1021600070BD0020FBE70020F9E70020F7E7002022
:10217000F5E70020F3E700BF3F420F0080DE80025A
:1021800070B506460D460024B4F57A7F0BD2736A0B
:102190005B6803F00103AB4207D04FF47A7001F0A3
:1021A000AFFF0134F0E7002000E0012070BD00BF68
:1021B000032968D870B588B004460D46164600F568
:1021C000805393F8D830C3F3800113F0040F00D18B
:1021D000114604F5805393F8D82061F3820283F806
:1021E000D82041F2780303EB451304EB030C04EB16
:1021F000451303F5845310331B7913F0010F09D0F5
:1022000046B104EB451303F5845310331B7913F0E7
:10221000080F12D07EB104EB451303F5845310333D
:102220001B7913F0080F06D104EB451404F5845410
:1022300043F00803237508B070BD00220023CDE9E8
:1022400000230023ADF8083003938DF818308DF883
:1022500019300493059303ABDCF80800DCF80C108C
:10226000DCF8102007C3BCF814201A80DDE90C2329
:10227000CDE900230123ADF8083023681B6C6946C3
:1022800020469847C6E77047426A936913F0700F7B
:1022900025D00023936100E00133022B1FDC00EB0B
:1022A000431202F584521032127912F0040FF3D067
:1022B00000EB431202F584521032127912F0020F31
:1022C000EAD0426A064951F82310916000EB4312AC
:1022D00002F58452117D41F004011175DCE770476D
:1022E0000450000870B582B0044616461D46436A85
:1022F0009A6812F0010F16D1636A9A6812F4807F0F
:102300001CD1636A9A6812F4803F24D104F580538B
:10231000D3F8DC0010B103681B6998472046FFF72B
:10232000B3FF02B070BD9A680121996000960195D3
:10233000C2F340020021FFF73BFFDDE79A684FF44C
:102340008071996000960195C2F3402201212046D8
:10235000FFF72EFFD5E79A684FF480319960009619
:102360000195C2F3404202212046FFF721FFCDE74D
:1023700038B50446084600297CD1616A01F10C0C8D
:10238000DCF8001011F0030F73D0DCF80010616A64
:1023900000F11B052D014D5915F0040F6ED100F110
:1023A0001B052D014D596D0DA56200F11B052D0179
:1023B0004D5915F0020F03D0A56A45F08045A5627E
:1023C00000F11B0501EB05156D6805F00F0E84F893
:1023D00034E001EB0011D1F8B80184F82C00D1F8F9
:1023E000B801000A84F82D00D1F8B801000C84F877
:1023F0002E00D1F8B801000E84F82F00D1F8BC01EE
:1024000084F83000D1F8BC01000A84F83100D1F81A
:10241000BC01000C84F83200D1F8BC11090E84F81C
:1024200033103821CCF80010A56AE06A216B65648E
:10243000A064E164A18EA4F85010A263E3630023BA
:10244000A4F8403023681B6C04F1380120469847FB
:1024500004F5805393F8D82042F0040283F8D82082
:10246000D3F8DC0010B103681B6998472046FFF7DA
:102470000BFF38BD616A01F1100C81E700F11B050B
:102480002D014D59ED08A56245F00045A5628CE788
:10249000302181F311880021022938DC30B502E0B7
:1024A000013102292FDC00EB411C0CF5845C0CF19E
:1024B000100C9CF804C01CF0040FF1D100EB411C7F
:1024C0000CF5845C0CF1100C9CF804C01CF0100F8F
:1024D000E6D000EB411E41F2780C0EEB0C045EF8E6
:1024E0000C50646895429C41DAD2446A0A4D55F812
:1024F0002150A5600EF5845C9CF814E04EF0040EAB
:102500008CF814E0CCE7002383F3118830BD00235E
:1025100083F31188704700BF0450000808B53023CA
:1025200083F31188FFF7B0FE002383F3118808BD01
:10253000436A9B6803F0E053B3F1E05F2CD070B5C1
:1025400005460E4653B3302383F31188002400E080
:102550000134022C1BDC05EB441303F584531033C8
:102560001B7913F0080FF3D105EB441303F58453E3
:1025700010331B7913F0040FEAD104F1840105EB49
:102580004111304600F00AFB0028E1D100E00120B3
:10259000002383F3118870BD012070470020FAE703
:1025A00008B5302383F3118800F58050C06EFFF723
:1025B0004BFA002383F311881F288CBF00200120D1
:1025C00008BD00BFF8B507460E4614461D46002359
:1025D0001370FFF7E5FF80F00103337025B1294642
:1025E0003846FFF7A5FF2070F8BD00BFF8B50446D8
:1025F0000D4616461F4600F00FFA02460B46297894
:1026000009B9307860B12046FFF742FF2046FFF756
:1026100085FF3B46324629462046FFF7D3FF01207F
:10262000F8BD00BF302383F311881B4B1A6C42F0B6
:1026300000721A641A6A42F000721A621A6A22F070
:1026400000721A62002383F3118800F5805393F817
:10265000D83013F0010F1ED110B5044601B910BDDA
:10266000302383F311880321132001F037FC032169
:10267000142001F033FC0321152001F02FFC04F598
:10268000805494F8D83043F0010384F8D830002304
:1026900083F31188E3E770470038024000F5805368
:1026A00093F8E030012B00F232812DE9F0418AB03D
:1026B00004460E461746974A52F82320002A37D080
:1026C000E66184F82070934B1B68002B34D004F52E
:1026D000805393F8E030012B06D18E4B18680368C5
:1026E0001B6B9847002836D001212046FFF79AFF40
:1026F000302383F31188626A136823F002031360A6
:10270000626A136843F001031360626A0023536135
:1027100083F3118801212046FFF732FD034648BBB1
:10272000626A4FF40041116018460AB0BDE8F081BA
:10273000784A42F82300C3E741F2E800FFF7CEFAF7
:10274000054610B10021FFF701FC724B1D60002D02
:10275000BDD10023E8E76F4D00212868FFF762FF35
:10276000286803685B683A46314698470346002864
:10277000BAD1D9E704F58053D86EFFF781F94FF04D
:1027800000082BE0202200216846FEF7CFFD002341
:1027900002938DF814308DF815300393049306934B
:1027A00041F2780505EB481504EB050EEC46BCE854
:1027B0000F006051CEF80410CEF80820CEF80C308F
:1027C000BCE80700CEF81000CEF81410CEF81820A0
:1027D0009CF800308EF81C3008F10108B8F1020FA7
:1027E000D0D904F5805393F8D8206FF3820283F890
:1027F000D8200023ADF820308DF822308DF823301A
:102800008DF8243008AA31462046FFF72BFC0346FA
:1028100000286FD0636A61221A609DF822301B067F
:1028200003F040739DF82320120402F47022134336
:102830009DF82420120502F4E0021343BDF8202085
:10284000C2F309021343022F59D00021626A0B43DD
:10285000D361636A13225A61626A136823F0010329
:10286000136000212046FFF78BFC0346002849D067
:1028700004F5805292F8E0209ABB616AD1F80022F8
:1028800042F00102C1F80022616AD1F8002222F46C
:102890007C5222F00E02C1F80022616AD1F80022B7
:1028A00042F46062C1F80022616A0022C1F8142279
:1028B000616AC1F80422616A41F6FF70C1F80C0236
:1028C000616AC1F84022616AC1F84422626A01214A
:1028D000C2F81C12616AD1F8002222F00102C1F88C
:1028E000002204F5805494F8D82042F0020284F8C3
:1028F000D82019E7626A4FF40041116014E74FF0E5
:102900000041A3E7626A4FF4004111600CE7002325
:1029100018467047284A002008B500F07DF80246A6
:102920000B4652EA030102D0013A43F1FF33044956
:10293000086808B1FFF7D6FC01F0A4FA08BD00BF93
:10294000284A002008B500F067F802460B4652EA14
:10295000030102D0013A43F1FF330449086810B182
:102960000021FFF705FD01F08DFA08BD284A00207F
:1029700008B500F051F802460B4652EA030102D0B6
:10298000013A43F1FF330449086810B10121FFF710
:10299000EFFC01F077FA08BD284A002000B59BB093
:1029A000EFF3098168226846FEF7ACFCEFF305837C
:1029B000014B9B6BFEE700BF00ED00E000B59BB054
:1029C000EFF3098168226846FEF79CFCEFF305836C
:1029D000014B9B6BFEE700BF00ED00E000B59BB034
:1029E000EFF3098168226846FEF78CFCEFF305835C
:1029F000014B5B6BFEE700BF00ED00E0FEE700BFB0
:102A0000FEE700BF0FB408B5029801F02BFBFEE70C
:102A100008B501F073FE08BD08B501F049FE08BD18
:102A20000020704701207047002070470020704749
:102A3000704700BF1B8813F0040F20D1F0B583B09E
:102A400005460E46041D00F11C0709E02B68DB6BF0
:102A50002846984763683246C1B2206898470834D0
:102A6000BC4209D00023009301932368002BEDD1D1
:102A70006368002BEAD1F2E7012003B0F0BD01202A
:102A8000704700BF84B0EC468CE80600002201E0ED
:102A90000132D2B2022A18D800210291039100EB30
:102AA000C20149680029F3D100EBC20189680029FD
:102AB000EED100EBC20000F1040C694603C98CE8BA
:102AC000030001321A70012000E0002004B07047BA
:102AD0000139C9B202290DD882B0002300930193B5
:102AE00000EBC100031D02AA12E9030083E8030002
:102AF00002B07047704700BF2DE9F0438BB0054628
:102B00000E46BDF84880041D00F11C074FF0000977
:102B100006E0636863B902E0B9F1000F15D008342C
:102B2000BC4236D00023089309932368002BF0D0D1
:102B300018F0040FF0D12B68DB6B284698476368C8
:102B40003246C1B220689847E9E700220023CDE968
:102B500000230023ADF8083003938DF818308DF86A
:102B600019300493059303AB30687168B26807C3EA
:102B7000B2891A80FFF750FFCDE900010423ADF8B8
:102B800008302B681B6C6946284698474FF00109AE
:102B9000C5E701200BB0BDE8F08300BF036823F058
:102BA000604C0A6822F06041D00FB0EBD37F0FD0A9
:102BB000002B08DB002A09DB8C4513D08C452CBF89
:102BC0000020012070474FEA9C4CF3E7890CF3E7A3
:102BD000C3F38073C2F380708C4504D08C452CBF46
:102BE0000020012070478342FCD1F7E70846704778
:102BF000084670470846704708467047401A83B237
:102C0000002800DB704703F1200000B2FAE700BFA4
:102C100003780133DBB203701F2B01D9002303704B
:102C2000704700BF082818D909280BD00A280BD0F4
:102C30000B280BD00C280BD00D280BD00E280BD056
:102C4000402070470C2070471020704714207047B8
:102C5000182070472020704730207047082818D966
:102C60000C280BD910280BD914280BD918280BD9EC
:102C700020280BD930280BD90F2070470920704726
:102C80000A2070470B2070470C2070470D207047BA
:102C90000E207047034621F0604C20F06042C00FC8
:102CA000B0EBD17F0FD0002908DB002B09DB944566
:102CB00013D094452CBF0020012070474FEA9C4C54
:102CC000F3E7920CF3E7C1F38071C3F3807094458E
:102CD00004D094452CBF0020012070478142FCD1D4
:102CE000F7E700BF2DE9F04107460D46D0F82480F4
:102CF000B8F1000F0CD046464446A4B1696860683C
:102D0000FFF7C8FF30B9236826465BB11C46F4E7DD
:102D1000796208E0A04502D035602C6003E02C60A9
:102D20007D6200E02560BDE8F08100BFC37DC3F394
:102D30008402013262F38603C375C38A6FF3090309
:102D4000C382C37D6FF3C713C375704738B504469C
:102D50000D46006A04E0016804F10C00FFF74AFF29
:102D600010B10369AB42F6D138BD00BF2DE9F04385
:102D7000079CCE0803EBD40501F0070304F0070419
:102D80001A442AE003F0070804F00707C646B845CE
:102D900038BFBE46CEF1080ED11A8E4528BF8E46EA
:102DA0004FF47F4C2CFA0EFC5FFA8CFC4CFA07FCBB
:102DB000D90800EB060919F8011001FA08F1F940E9
:102DC000C9B24FEAD40815F8087079400CEA01013D
:102DD0004F4005F80870734474449342D2D1BDE863
:102DE000F08300BF2DE9F04F87B004900E460592A6
:102DF0000393838AB1EBC30F80F084801146DA001D
:102E000031448A4204D2D2B2F3B2D21AD3B2059379
:102E1000049BDB683BB3272E36D8C6F12803059AFE
:102E20009A422ED35FFA86FBCBF1280B5FFA8BFB1D
:102E300000230093039B5A46314604988068FFF7AD
:102E400095FF5E44059BA3EB0B04E4B2049B9F8AB1
:102E500007F10057053FFF00D3F80C9028214B469F
:102E6000B9461F4627E0049B1B69002BD3D10023E2
:102E70000093039B059A314604988068FFF776FF1C
:102E800033E0DDF814B0D3E7059C4FF0000BDDE72D
:102E90002546CDF800B0039B2A46711A381DFFF76E
:102EA00065FF2E44AB445FFA8BFB641BE4B2A9EBD5
:102EB0000A093F684146A7B19CB1CA46B9F1E00F83
:102EC00028BF4FF0E00A0AEB01084645EFD2A8EB15
:102ED00006039C42DCD35FFA88F5F3B2ED1AEDB23B
:102EE000D7E7049B186900B124B9BDF9140007B0F5
:102EF000BDE8F08FCDF800B0039B2246711AFFF7B2
:102F000035FFF2E70020F2E7002070470139002387
:102F100007E0C25C10F801C000F803C0425401335E
:102F200001398B42F5D3704780EA0120002303E08A
:102F3000400080B20133DBB2072B09D810F4004FF8
:102F4000F6D0400080B280F4815080F00100F1E7BB
:102F5000704700BF70B516461D46002411E0C4F14D
:102F60002003A4F1200C26FA04F105FA03F3194317
:102F700025FA0CFC41EA0C01C9B2FFF7D5FF083471
:102F8000A4B23F2CEBD970BD38B50C4604E014F860
:102F9000011BFFF7C9FF2A46551E002AF7D138BD8D
:102FA00038B5058C072D0BD90446D0E902234FF61E
:102FB000FF70FFF7CFFF2A46E169FFF7E5FF38BD55
:102FC0004FF6FF70FBE700BF10B4016100F1040C85
:102FD000002305E001EB4314CCF80040A446013384
:102FE0009A42F7D80023CCF80030028143818381D4
:102FF00003605DF8044B70470346406848B10268BF
:103000005A605A89013292B25A8199898A4200D90A
:103010009A81704708B5FFF7EFFF08B100230360FE
:1030200008BD00BF2DE9F84F8246894616461F4667
:10303000CB8AC3F30903052B34D018460024042B94
:103040000BD8BAB2A24208D9315D09EB0302D1769E
:1030500001339BB20134A4B2F1E7BBB2A34218D949
:10306000B9F816B0CBF3090BABF1050293083E4952
:10307000A1FB0313C3EBC303A2EB83031FFA83F883
:10308000D9F8041081B15046FFF7B0FD0546012381
:103090001CE00344B9F8162063F30902A9F81620CE
:1030A000012055E00024DBE75046FFF7B3FF05465B
:1030B00001465046FFF79CFDC9F80400002D49D099
:1030C0004FF000082CE001339BB215462A68002A15
:1030D000F9D107EB0B02053A92082349A1FB021232
:1030E00092B2013292B293421AD2B8F1000F17D1C4
:1030F0005046FFF78FFF286078B3054610E0325D39
:1031000005EB0C031A710CF1010C1FFA8CFC013455
:10311000A4B2BCF11B0F01D8A142F0D8A14204D83F
:10312000B9B2A1420AD9C446F3E75046FFF772FF8D
:103130002860A8B105464FF00008F1E7B9F816304D
:10314000C3F30902114461F30903A9F81630012001
:10315000BDE8F88F6FF00200FAE76FF00200F7E7C2
:103160006FF00200F4E700BF2549922443680B602A
:1031700041604389013B4381704700BFF8B5064673
:103180000D460EE006F10C042046FFF72FFD014628
:1031900007682046FFF7EAFF39462046FFF728FD7B
:1031A000686069680029EDD1EB8A6FF30903EB824F
:1031B00000200021F8BD00BF08B5FFF71DFF034642
:1031C00028B10022026042608260C260026118463B
:1031D00008BD00BF2DE9F04F83B001921D465B6929
:1031E000002B00F09C8081468B462B8C1BB1EA693A
:1031F000002A00F09780072B18D902339BB20633C0
:103200004E4A82FB03121344C3F38F03B9F8142010
:10321000B9F81610521A92B2934200F289804FF018
:10322000800A4FF000084446474656E009F10C007A
:10323000FFF7C2FF0446002877D02A8CE9690830DE
:10324000FEF760F8288C013080B2FFF707FDFFF72A
:10325000E9FC431E9BB22B84013323746B691B78FA
:1032600003F01F032A8C43F0C003224413724BF077
:103270000043636021464846FFF734FD0127384686
:1032800003B0BDE8F08F002037E02B8CA34243D081
:10329000013080B2FFF7E2FCFFF7C4FC013880B2D6
:1032A0004FEA4813DBB243EA0A0A6B691B7803F062
:1032B0001F034AEA030A331883F808A04BF00043BF
:1032C00073600130307431464846FFF70BFD01371B
:1032D0003FB288F001084FF0000A2B8CA342CED0F9
:1032E00009F10C00FFF768FF064620B3002CCAD195
:1032F000019B03721B0A4372022003460628C4D8AE
:103300002A8CA242C1D9EA69125D33441A72013093
:1033100080B20134A4B2F0E74FF0400AB8E76FF092
:103320000107ACE76FF00107A9E76FF00207A6E716
:103330006FF00207A3E76FF00207A0E7932449921A
:1033400030B589B004460D46202200216846FDF7BD
:10335000EDFF04952046FFF74FFE8646A0B1EC46F0
:10336000BCE80F00CEF80000CEF80410CEF808201C
:10337000CEF80C30BCE80F00CEF81000CEF81410D8
:10338000CEF81820CEF81C30704609B030BD00BF12
:1033900070B5044600F10C063046FFF7D1FF054634
:1033A00028B1216A3046FFF727FC286025622846AD
:1033B00070BD00BF38B504460D46036A1BB1FFF768
:1033C000C5FC38B138BD0C30FFF7BAFF0028F9D082
:1033D0002062F7E729462046FFF7DAFFF2E700BF51
:1033E000F8B504460E4615461F4630220021FDF76B
:1033F0009DFFA760069B6360079BA3626A09B5F502
:10340000001F01D34FF6FF7292B2314604F10C0057
:10341000FFF7DAFDF8BD00BF037823B919B111F049
:10342000800F00D101707047007870472DE9F84394
:1034300005460C46D1F81C90B9F1000F23D094F842
:103440001880B8F11F0F3BD82846FFF7EDFF06465E
:10345000F8B9228C072A36D8278A37F0030335D1EA
:1034600049464FF6FF70FFF78FFD47F6FE730340A6
:103470005B0243EA08633F0207F440773B431E4385
:103480004FF6FF720EE00B8C002BD8D06FF00105C9
:103490000FE0238A1B0243EA08631E432046FFF71E
:1034A0007FFD0246234631462846FFF793FE051E60
:1034B00002DC2846BDE8F8836069FFF7A9FBF8E75E
:1034C0006FF00105F5E76FF00305F2E76FF0010516
:1034D000EFE700BF70B58AB0044616461D462822A5
:1034E00000216846FDF722FF02960395BDF83830AB
:1034F000ADF810300F9B05939DF840308DF81830D3
:10350000119B0793BDF84830ADF82030694620463E
:10351000FFF78CFF0AB070BD2DE9F04106460F465B
:103520001546D3692BB395F81880B8F11F0F2AD828
:103530003046FFF779FF48B32C8A240444EA086434
:103540002B7844EAC33444EA0724044344F080045B
:103550002846FFF725FD02462B4621463046FFF759
:1035600039FE041E02DD2B78012B08D02046BDE871
:10357000F081138C002BD6D06FF00104F6E7686958
:10358000FFF746FBF2E76FF00104EFE76FF003048B
:10359000ECE700BFF0B58BB004460D4617461E465B
:1035A000282200216846FDF7C1FE9DF84C30012B12
:1035B00014BF002301238DF80030029703969DF875
:1035C0004030ADF81030119B05939DF848308DF8D0
:1035D0001830149B0793BDF85430ADF820306A467C
:1035E00029462046FFF798FF0BB0F0BD406A00B1B6
:1035F0000430704708B5416A0B6843620C30FFF72E
:10360000B5FD08BD2DE9F041054616469846076A06
:103610003C4619E021462846FFF7B0FD05F10C07AE
:103620002B6A19683846FFF7E5FA286221463846C2
:10363000FFF79CFD2C6A274606E0216805F10C0087
:10364000FFF7D8FA274604460CB3A168E368711A5D
:1036500068EB03030F4A8A424FF0000272EB030348
:10366000EBD22B6AA342D5D021462846FFF786FD30
:1036700023683B6005F10C0321461C461846FFF702
:1036800075FD39682046FFF7B5FA0446DCE7BDE86A
:10369000F08100BF80841E002DE9F04182B0089EB9
:1036A000002800F0E28014461D460746002E00F078
:1036B000DF80531EDBB23F2B00F2DD80012A02D1F6
:1036C000002D40F0DB800023009301936B462246DF
:1036D0003846FFF787FB071E3BDD14F0070F0AD0C3
:1036E00002AB03EBD40111F8083C624202F007027E
:1036F000134101F8083C012C0BD0082C2DD9102CBB
:103700002ED9202C2FD9402C00F2BB804FF0080876
:1037100000E0A046FFF7F8FB40BB9DB1B4EBC80F3B
:1037200010D0082C27D89DF80020631E22FA03F33E
:1037300013F0010F06D00123A3405B42DBB2134319
:103740008DF80030002D72D0082C5ED89DF9003025
:103750003370384602B0BDE8F0814FF00108D9E778
:103760004FF00208D6E74FF00408D3E74146684619
:10377000FFF7CCFBD1E7102C0FD8BDF80020631E5B
:1037800022FA03F313F0010FDCD00123A3405B42C4
:103790009BB21343ADF80030D4E7202C0CD8009A2C
:1037A000631E22FA03F313F0010FCBD00123A340D1
:1037B0005B421A430092C5E73F2C65D8DDF800C094
:1037C000019A631EC4F12100A4F121012CFA03F334
:1037D00002FA00F0034322FA01F10B4313F0010F48
:1037E000B0D00123A4F12001C4F1200003FA01F1BB
:1037F00023FA00F00143A3405B4261EB41014CEA34
:1038000003030A43009301929CE7102C03D8BDF9EF
:10381000003033809DE7202C02D8009B336098E76E
:10382000402C34D8DDE90023C6E9002391E7012CC0
:1038300005D0082C07D89DF80030337089E79DF833
:103840000030337085E7102C03D8BDF8003033808A
:103850007FE7202C02D8009B33607AE7402C19D8F0
:10386000DDE90023C6E9002373E76FF0010770E785
:103870006FF001076DE76FF001076AE76FF001076E
:1038800067E76FF0080764E76FF0080761E76FF01C
:1038900008075EE76FF008075BE700BFF0B585B08B
:1038A00005460E46402A03D8144612B9012400E00A
:1038B0004024002202920392012C06D0082C22D828
:1038C0001B788DF80830012703E01B788DF808304D
:1038D0002746FFF719FB68BB14F0070F0AD004ABAB
:1038E00003EBD40111F8083C624202F00702934056
:1038F00001F8083C00962B462246002102A8FFF75B
:1039000035FA05B0F0BD102C04D81B88ADF808308E
:103910000227DEE7202C03D81B6802930427D8E790
:10392000402C05D8D3E90023CDE902230827D0E7AE
:103930000027CEE7394602A8FFF7E8FACCE700BF38
:1039400070B506460C4605E00D6806F10C00FFF761
:103950000DFCE560E1680029F6D10023E360A36077
:103960002361A38270BD00BF10F0800F04D010F45B
:10397000004F03D00120704702207047002070479D
:1039800010B50446FFF7F0FF022802D0C4F3074049
:1039900010BDC4F30F2014F07F0FF9D100F0030025
:1039A000F6E700BF2DE9F04F99B006460D460392A9
:1039B0000493D1F800904846FFF7D6FF0746022847
:1039C00000F08980C9F30628B9F1000F80F2068261
:1039D00019F0C04F40F005822C7B002C00F00482CF
:1039E000022F05D03046FFF71FFD404540F0FF8114
:1039F000C9F30463099309F07F0A4846FFF7C0FF43
:103A00000A9040EA074949EA8A4949EA4869013C7B
:103A10002C4494F8048000220023CDE916235FEAA9
:103A2000D81302935AD07468CDF800A03B460246E2
:103A300016A93046A047002800F0DC8149463046F0
:103A4000FFF7B8FC0446002800F0D781A368E168BE
:103A5000039A0593D01A0790049B069163EB010328
:103A6000089395F80DC0CDF82CC094F81AC0CDF885
:103A700030C094F81790C9F3840908F01F0B594619
:103A80004846FFF7BBF80D9049465846FFF7B6F891
:103A90006368059A069952EA010C35D09F4A079946
:103AA0008A424FF00002089972EB010CC0F081804D
:103AB0000B9A0C998A421BD0994B079A93424FF06C
:103AC0000003089A934176D2029B002B75D00F28F1
:103AD00075DD002319E04FF0000875E749463046D0
:103AE000FFF734F904460028B0D16FF00C0088E1EC
:103AF000029A002AE0D00D9A012A01DD012304E098
:103B0000002BD9D0012300E00123002B59D16A7B7F
:103B1000A37E9A4240F07481029B13B118F0400FCB
:103B20006AD1C8F34013E27DB3EBD21F40F06C8141
:103B3000C2F384039B4540F06A81029B002B00F096
:103B4000948018F0400F40F090802B7B032B40F2C4
:103B50006181039BA360049BE360E38A6FF3090325
:103B6000E382AF1D2B7B033BDBB23A46214606F1D5
:103B70000C00FFF757FA00286DDB2B796A7943EACE
:103B800002232383DDE916234FF6FF70FFF7E2F9E6
:103B9000A0822A7B033AD2B23946FFF7F5F9A08218
:103BA000E37DDA43C2F3C01262F3C713E37500206A
:103BB00027E10123A9E70023A7E70023A5E70123C5
:103BC000A3E7E37D68F38603E375DBB26FF3C71306
:103BD000E37521463046FFF7D1FA6B7BA376029B53
:103BE000002B94D1E37DC3F38402013262F3860398
:103BF000E3756FF00C0004E1039BA360049AE2609C
:103C0000202200210EA8FDF791FB039B0E93049A3E
:103C10000F922B1D10932B7B013BDBB2ADF84C3088
:103C20000A9BADF84E308DF850708DF851B0099B5D
:103C30008DF852308DF853A096F82C3083F00103A4
:103C40008DF85430B3680EA9304698472046FFF7E8
:103C50006DF80020D5E021463046FFF78FFA204668
:103C6000FFF764F86FF00200CBE0029B13B918F085
:103C7000400F1ED095F80C9009F1FF395FFA89F9D1
:103C8000B4F81680C8F30908B8F1040F30D84346D9
:103C90004FF00008042B53D8C84551D205EB080259
:103CA0001179E218D176013308F101085FFA88F83A
:103CB000F0E72F1D2B7B013BDBB23A46214606F194
:103CC0000C00FFF7AFF9002808DB2A7B013AD2B2DB
:103CD0003946A08AFFF758F9A08261E721463046AD
:103CE000FFF74CFA2046FFF721F86FF0020088E05A
:103CF000616806F10C00FEF779FF024608B1052362
:103D000004E04FF000081BE01C330A46116800294C
:103D1000FAD1A8EB03034FF000080DE080841E00E9
:103D200040420F0005EB08010879D11808710133F2
:103D300008F101085FFA88F81B2B01D8C845F1D3B8
:103D4000039B0E93049B0F9304F11B031093616874
:103D500006F10C00FEF74AFF1190C84535D2A84481
:103D600008F104031293E38AC3F309039944ADF8FD
:103D70004C900A9BADF84E308DF850708DF851B0D4
:103D8000099B8DF852308DF853A096F82C3083F0B3
:103D900001038DF85430002363602A7B013A291D0A
:103DA000A08AFFF7F1F8A082238B98420FD00EA9CA
:103DB0003046FFF7C5FD2046FEF7B8FFA28A238BE9
:103DC0009A4209D06FF010001BE00023CAE7B368E5
:103DD0000EA930469847EAE7002012E06FF009008C
:103DE0000FE06FF009000CE06FF0090009E06FF0E0
:103DF0000A0006E06FF00B0003E06FF0020000E045
:103E0000002019B0BDE8F08F6FF00D00F9E76FF0FA
:103E10000E00F6E76FF00F00F3E700BFEFF3098342
:103E2000683305494A6B22F001024A6383F309882B
:103E3000002383F31188704700EF00E0302080F307
:103E4000118862B60C4BD96821F4E0610904090CB1
:103E50000A4A0A43DA60D3F8FC2042F08072C3F8C1
:103E6000FC2007490A6842F001020A602022DA7742
:103E700083F82200704700BF00ED00E00003FA0560
:103E8000001000E0302383F31188104B5B6813F4BB
:103E9000006F03D1002383F31188704710B5F1EE52
:103EA000103AEFF30984683C4FF08073E361084BEC
:103EB000DB6B236684F3098800F096F810B1054B9C
:103EC000A36110BD044BA361FBE700BF00ED00E060
:103ED00000EF00E03F030008420300080901C9B2F7
:103EE000074A131883F8001300F01F01400901234B
:103EF0008B4000F1600142F8213042F820307047D9
:103F000000E100E00023037503691B68996882687B
:103F10009142FAD203605A6842601060586070475C
:103F200008B50846302383F311880B7D032B0ED090
:103F3000042B10D043B14FF0FF338361FFF7E2FF52
:103F4000002383F3118808BD83F31188FBE78B6995
:103F500000221A60EFE74A680B6813604A685A60EB
:103F6000E9E700BF0023037503691B68996882684D
:103F70009142FAD803605A684260106058607047F6
:103F800008B5FFF7BFFF08BD08B5064BD96808752F
:103F9000186802681A60536001220275D860FCF745
:103FA000B9F908BD384A002030B587B004460C4B3B
:103FB000DD68B1F1FF3F0FD02B460A4A684600F09A
:103FC0001BF92046FFF7E0FF009B13B1684600F0A5
:103FD00021F9A86907B030BDFFF7D6FFF9E700BFA8
:103FE000384A0020213F0008044BDA681B689868B3
:103FF0009368984294BF002001207047384A0020FF
:1040000010B5084BD8681C6822681A6053600122FA
:104010002275DC60FFF7A6FF01462046FCF77AF91F
:1040200010BD00BF384A002008B50B4B01221A70A2
:10403000002353B109490A4800F06EFC064B0222E6
:104040001A70002383F3118808BD034A02EB830230
:10405000002151600133ECE7A04C0020AC50000877
:10406000384A002008B572B6044B186500F0EEFA25
:1040700000F0CCFB024B03221A70FEE7384A002006
:10408000A04C002008B500F0FFF808BD8B600223AB
:104090000B7500234B7508610846704708B58168A9
:1040A000A1F1840341F8143C026941F8442C4269AF
:1040B00041F8402C044A41F8242CC3680268203996
:1040C0000248FFF7E3FF08BD2D030008384A00202F
:1040D00008B5FFF7E3FFFFF753FF08BD08B5034B33
:1040E000DB6898610F20FFF74FFF08BD384A0020BA
:1040F00008B5302383F31188FFF7F0FF08BD00BF38
:1041000008B50146302383F311880820FFF74CFFE0
:10411000002383F3118808BDF8B515461C46C2601C
:104120008B60486003680B6059600160092C00D8FF
:104130000A24C068204400F0DBFB0A2700F0D4FB0F
:104140000646431B9C4202D90A2F07D8F8BD7C1CA7
:10415000281900F0DBFB27463546EFE7012000F089
:104160001BFCF3E770B504460D46092900D80A2563
:104170000A26601900F0CAFB00F0B6FB041BA5423A
:1041800002D90A2E04D870BD013635460446F0E740
:10419000012000F001FCF6E7F8B505460E4617468B
:1041A00000F0A2FB2B689D4209D0EC68041B3C196F
:1041B00000D33C469B68A34208D82B680CE03B46E2
:1041C000024631462846FFF7A7FF14E03946FFF7BD
:1041D000C9FFF2E7A41A1B689A689442FAD8B4603F
:1041E00033605A68726016605E609A68121B9A604B
:1041F0004FF0FF33AB60F8BD08B50361C260002328
:1042000043610A4601460248FFF7C6FF08BD00BFEA
:10421000484A002008B51B4B1B69984210D04268E1
:104220000368136042685A600268816893680B44AF
:10423000936000230360134B4FF0FF329A6108BD77
:104240001968104A134643F8101F4B6000210160A3
:1042500012699A4212D0816893680B44936000F00F
:1042600043FB084AD369A0EB030C126991686145CE
:10427000E5D91B1A1944FFF775FFE0E700F040FB92
:10428000DDE700BF384A0020F8B50BE0002383F3D8
:104290001188E368216920469847302383F3118809
:1042A0006369CBB92C4D2C6900F01EFBEB69C21A77
:1042B000A568954242D81D44274BDD61616822689C
:1042C0000A60616851600022226053F8102F9A4200
:1042D000DCD100F015FBD9E700F006FB0746461BD2
:1042E0006269B2420CD32B1A13441B4A52F8101FB6
:1042F00091420AD09E1900D23346174A12690CE047
:10430000022000F049FB0023EFE73A46214613481C
:10431000FFF702FF1FE05B1A126891688B42FAD820
:10432000A3602260516861600C6054609168CB1A90
:104330009360094B4FF0FF329A61B3E7064A52F897
:10434000101F914207D0044AD0611B1AA16819447A
:10435000A160FFF707FFF8BD384A0020484A002057
:1043600038B500F0C1FA054AD2E90845031B18190F
:1043700045F10001C2E9080138BD00BF384A0020FC
:1043800000207047FEE700BF704700BF4FF0FF30CE
:10439000704700BFBFF34F8F024BDB6813F4803FC1
:1043A000FAD17047003C0240014BF322DA607047BB
:1043B000003C024008B50B4B1B7803B108BDFFF76A
:1043C000E9FF094B1B69002B05DB074A136823F43F
:1043D00080631360F2E7044B044A5A6002F18832AA
:1043E0005A60F2E7A84C0020003C024023016745D8
:1043F00008B50C4B1B7803B108BDFFF7CBFF0A4B88
:104400001A6942F000421A611A6842F480521A6036
:104410001A6822F480521A601A6842F480621A60A4
:10442000EAE700BFA84C0020003C024012F0010F58
:1044300065D1F8B504460E4615461318B3F1016F61
:104440005FD8314B1B6813F0010F01D1002059E0F8
:10445000FFF7B0FFFFF7A8FFFFF79CFF032D29D957
:1044600014F0030F26D1294A136923F44073136112
:10447000136943F4007343F0010313613768276045
:10448000BFF34F8FFFF786FF23689F4203D1043DA0
:1044900004360434E2E71D4A136923F00103136173
:1044A00004E01A4A136923F001031361FFF7A0FF28
:1044B000002027E0012D19D9144A136923F4407311
:1044C0001361136943F4807343F00103136133886C
:1044D0002380BFF34F8FFFF75DFF23889BB23288A5
:1044E0009A42DED1023D02360234E3E7074A1369FD
:1044F00023F001031361FFF77BFF012002E000209E
:1045000070470020F8BD00BF00380240003C024068
:10451000014B53F820007047B85000080B281AD8F8
:1045200070B506460D4B1B788BB900244FF0006523
:1045300008E00B4B43F824502046FFF7E9FF054401
:104540000134E4B20B2CF4D9044B01221A70044B51
:1045500053F8260070BD0020704700BFDC4C0020DF
:10456000AC4C00200C2070470B2801D9002070476C
:1045700038B50546FFF7D2FF04462846FFF7C8FFC7
:1045800030B12368B3F1FF3F04D104380434F7E7B6
:10459000012038BD0020FCE70B2801D9002070471E
:1045A00038B50446FFF7F6FEFFF704FFFFF7FCFE01
:1045B000154BA3FB0423DB081A4603EB4303A4EBD0
:1045C0008303DB00DBB2D201D2B2134343F40073A6
:1045D00043F002030D4A1361136943F480331361FE
:1045E000FFF7D8FE2046FFF799FF05462046FFF764
:1045F0008FFF0146284600F005F9FFF7F9FE204637
:10460000FFF7B2FF38BD00BFABAAAAAA003C024028
:1046100008B5FFF70BFF08BD08B5034610B10A4AFD
:10462000127822B113B9084B1B7833B908BDFFF7D4
:10463000C1FE054B01221A70F8E7034B00221A70E5
:10464000FFF7D6FEF2E700BFA84C002010B500240B
:104650000BE0074804EB44039A00134603445968EF
:10466000805800F0D1F80134E4B2012CF1D910BD2A
:10467000E850000808B50846114600F04DFC08BD9A
:1046800008B5084600F05EFC08BD00BF302383F388
:1046900011887047002383F311887047302383F318
:1046A00011887047002383F311887047FFF758BEC5
:1046B000EFF3118303BB00B583B0EFF30583C3F3BE
:1046C000080363B9FFF7E2FFFFF7F0FFCDE9001041
:1046D000FFF7E0FFDDE9001003B05DF804FBFFF732
:1046E000DDFFFFF7E3FFCDE90010FFF7DBFFDDE9BA
:1046F000001003B05DF804FBFFF7D8BF38B5FFF733
:10470000D7FF114C114AC00840EA4170A0FB025E7D
:10471000C908A0FB040C1CEB050CA1FB04404FF0E6
:1047200000035B41A1FB02121CEB040C43EB0000F5
:1047300011EB0E0142F10002411842F1000009099B
:1047400041EA007038BD00BFCFF753E3A59BC420FA
:1047500009E000F1010C064A52F8202041F8042B30
:104760001A465FFA8CF0531EDBB2002AF1D1704773
:104770005028004010B4124B1B6F13F4004F08D1A7
:104780000F4B1C6F44F400741C671C6F44F400440E
:104790001C670C4C236843F48073236009E000F12C
:1047A000010C51F8044B084A42F820401A465FFABF
:1047B0008CF0531EDBB2002AF1D15DF8044B704738
:1047C00000380240007000405028004000B583B01F
:1047D000012201A90020FFF7BBFF019803B05DF89B
:1047E00004FB00BF10B582B00446FFF7EFFFA04204
:1047F00001D102B010BD0194012201A90020FFF7F0
:10480000B9FFF6E7704700BF704700BF704700BFB1
:10481000074B45F255521A6003225A6040F2FF726C
:104820009A604CF6CC421A60024B01221A70704713
:1048300000300040E44C0020034B1B781BB1034BBD
:104840004AF6AA221A607047E44C0020003000406B
:10485000044B1B6823B9044BD3F87428014B1A602E
:10486000704700BFE04C002000300240024B4FF088
:104870008072C3F8742870470030024008B5FFF713
:10488000E7FF024B1868C0F3407008BDE04C002001
:1048900008B5FFF7DDFF024B1868C0F3007008BDD4
:1048A000E04C0020704700BFFEE700BF084B0949FD
:1048B00003E051F8042B43F8042B074A9342F8D342
:1048C00002E0002243F8042B044A9342F9D37047D4
:1048D000684D002090520008684D0020684D00206F
:1048E00008B500F0DBF808BD4FF08043586A704708
:1048F0004FF08043586300221A610222DA60704749
:104900004FF080430022DA60704700BF4FF08043D1
:1049100058637047FEE700BF70B586B004460E4688
:10492000194B5860002585620163FFF787FA246000
:104930006460A560E56204F11003236163614FF0D8
:10494000FF33A361E561FFF7CFFF02462B46C4E9C1
:104950000823256580230D4A04F134012046FFF722
:1049600095FBE06001230375094A00927268019289
:10497000B26802920393074B049305956846FFF7CC
:10498000A7FB06B070BD00BFA04C0020005100087E
:104990000851000815490008024AD36A0343D3624C
:1049A000704700BF384A00204B6843608B688360C3
:1049B000CB68C3600B6943614B6903628B694362D7
:1049C0000B680360704700BF10B5214B1A6940F2B5
:1049D000FF110A431A611A6922F4FF7222F00102E0
:1049E0001A611A691A6B0A431A631A6D0A431A6527
:1049F0001B6D184C21461848FFF7D6FF04F11C0127
:104A00001648FFF7D1FF04F138011548FFF7CCFF36
:104A100004F154011348FFF7C7FF04F17001124875
:104A2000FFF7C2FF04F18C011048FFF7BDFF04F14E
:104A3000A8010F48FFF7B8FF04F1C4010D48FFF7C4
:104A4000B3FF04F1E0010C48FFF7AEFF10BD00BF5B
:104A500000380240105100080000024000040240EB
:104A600000080240000C0240001002400014024006
:104A700000180240001C02400020024008B5FFF769
:104A8000A3FF00F095F808BD08B500F025FAFFF780
:104A9000CBFAFFF7DDFE08BD704700BF0F4B1A6C65
:104AA00042F001021A641A6E42F001021A661B6E8D
:104AB0000B4A936843F0010393604FF08043532205
:104AC0009A624FF0FF32DA6200229A615A63DA602A
:104AD0005A6001225A611A60704700BF00380240D4
:104AE000002004E008B54FF080421369D168C9B2D4
:104AF0000B40D943116113F0020F00D108BD3023E0
:104B000083F31188FFF7BEFA002383F31188F5E7DA
:104B10000B4A136843F4807313600A4B1B6F03F452
:104B20004073B3F5007F05D0064B4FF480321A670F
:104B300000221A67024A536823F4007353607047D7
:104B4000007000400038024008B5184B1A696FEA3F
:104B5000C2526FEAD2521A611A69C2F308021A618C
:104B60001A695A694FF0FF3058615A69002159613A
:104B70005A691A6A62F080521A621A6A02F0805206
:104B80001A621A6A5A6A58625A6A59625A6A1A6CDE
:104B900042F080521A641A6E42F080521A661B6EFE
:104BA000FFF7B6FF00F076F908BD00BF00380240FD
:104BB0003B4B4FF080521A643A4A4FF44041116027
:104BC0001A6842F001021A60354B1B6813F0020F9D
:104BD000FAD0334A936823F003039360304B9B6809
:104BE00013F00C0FFAD12E4B1A6802F0F9021A607A
:104BF00000229A601A6842F480321A60284B1B68BF
:104C000013F4003FFAD0264A536F43F00103536771
:104C1000234B5B6F13F0020FFAD0214B224A5A60EC
:104C20001A6842F080721A601E4B5B6813F4804F62
:104C3000FAD01B4B1B6813F0007FFAD0184B1B4AAD
:104C40009A601B4B1A681B4B9A421FD01A4B40F2BA
:104C500005721A60184B1B6803F00F03052BF9D17E
:104C60000F4A936843F0020393600D4B9B6803F077
:104C70000C03082BF9D10A4B5A6C42F480425A6457
:104C80005A6E42F480425A665B6E70470B4B1A684C
:104C90000B4B9A42DAD1084B40F205121A60D9E761
:104CA00000380240007000400854400700948838E3
:104CB000002004E011640020003C024000ED00E010
:104CC00041C20F4108B5074A536903F0010353611C
:104CD0002BB1054B1B6813B1034A50689847FFF787
:104CE000D1F808BD003C0140E84C002008B5074A57
:104CF000536903F0020353612BB1054B9B6813B159
:104D0000034AD0689847FFF7BDF808BD003C014052
:104D1000E84C002008B5074A536903F004035361C7
:104D20002BB1054B1B6913B1034A50699847FFF734
:104D3000A9F808BD003C0140E84C002008B5074A2E
:104D4000536903F0080353612BB1054B9B6913B101
:104D5000034AD0699847FFF795F808BD003C014029
:104D6000E84C002008B5074A536903F0100353616B
:104D70002BB1054B1B6A13B1034A506A9847FFF7E2
:104D800081F808BD003C0140E84C002010B51A4BEA
:104D90005C6904F478725A6114F0200F05D0174B47
:104DA0009B6A13B1154AD06A984714F0400F05D09A
:104DB000124B1B6B13B1114A506B984714F0800FC4
:104DC00005D00E4B9B6B13B10C4AD06B984714F473
:104DD000807F05D0094B1B6C13B1084A506C984773
:104DE00014F4007F05D0054B9B6C13B1034AD06CC3
:104DF0009847FFF747F810BD003C0140E84C002001
:104E000010B51F4B5C6904F47C425A6114F4806F46
:104E100005D01C4B1B6D13B11A4A506D984714F402
:104E2000006F05D0174B9B6D13B1164AD06D984794
:104E300014F4805F05D0134B1B6E13B1114A506EF2
:104E4000984714F4005F05D00E4B9B6E13B10D4ACA
:104E5000D06E984714F4804F05D00A4B1B6F13B1E6
:104E6000084A506F984714F4004F05D0054B9B6FCC
:104E700013B1044AD06F9847FFF704F810BD00BF84
:104E8000003C0140E84C002008B5FFF72BFEFEF780
:104E9000F9FF08BD08B506210846FFF71FF80621EF
:104EA0000720FFF71BF806210820FFF717F8062157
:104EB0000920FFF713F806210A20FFF70FF8062153
:104EC0001720FFF70BF806212820FFF707F8072126
:104ED0001C20FFF703F808BD08B5FFF735FE00F00A
:104EE00005F8FFF7D9FDFFF7FBFC08BD002307E03D
:104EF000054A002142F8331002EBC302516001332E
:104F00000F2BF5D9704700BFE84C00200B46014637
:104F1000184600F009B80000024B0A46014618681E
:104F2000FFF7A8BB1C23002010B5054C13462CB17D
:104F30000A4601460220AFF3008010BD2046FCE780
:104F400000000000024B01461868FFF799BB00BF44
:104F50001C23002010B501390244904201D10020E9
:104F600005E0037811F8014FA34201D0181B10BDD2
:104F70000130F2E72DE9F041A3B1C91A17780144D5
:104F8000044603F1FF3C8C42204601D9002009E091
:104F90000578BD4204F10104F5D10CEB0405D618E7
:104FA000A54201D1BDE8F08115F8018D16F801ED9B
:104FB000F045F5D0E7E700006F72672E6172647507
:104FC00070696C6F742E41522D46343037536D61C9
:104FD000727442617400000040A2E4F164689106BA
:104FE0000000000041A3E5F265699207000000009F
:104FF0004261642043414E496661636520696E6485
:1050000065782E0080000000008000000000800015
:105010000000000000000000F91C00089D260008A8
:10502000ED250008351D0008411D0008B91E0008C7
:10503000051D0008151D0008091D0008111D0008A8
:105040000D1D0008711E0008191D0008852A0008A2
:10505000D12A0008291D00088D1E0008000000004C
:1050600000000000F91C0008FD290008212A0008A2
:10507000252A0008F92A0008352A0008051D00081D
:10508000292A0008091D00082D2A00080D1D000806
:10509000312A0008FD290008852A0008D12A0008C5
:1050A000FD290008FD29000863300000A850000811
:1050B000904A0020A04C002000400000004000006A
:1050C000004000000040000000000100000002005D
:1050D00000000200000002000000020000000200C8
:1050E00000000200000002000001002000FF01009B
:1050F0000100000000000220000002000200000089
:105100006D61696E0000000069646C65000000005C
:105110000000802A00000000AAAAAAAA0000002419
:10512000FFFF0000000000000090090000000000E8
:1051300000000000AAAAAAAA00000000FFFF0000C9
:10514000000000000000000000000005000000005A
:10515000AAAAAAA600000000FFEF000000000000BD
:10516000000000000000000000000000AAAAAAAA97
:1051700000000000FFFF0000000000000000000031
:105180000000000000000000AAAAAAAA0000000077
:10519000FFFF000000000000000000000000000011
:1051A00000000000AAAAAAAA00000000FFFF000059
:1051B00000000000000000000000000000000000EF
:1051C000AAAAAAAA00000000FFFF00000000000039
:1051D0000000000000000000000000000A000000C5
:1051E00000000000030000000000000000000000BC
:1051F00000000000000000000000000000000000AF
:10520000000000000000000000000000000000009E
:105210006E0400000000000000000F00000000000D
:1052200040420F00FE2A0100D2040000202300208B
:10523000000000000000000000000000000000006E
:10524000000000000000000000000000000000005E
:10525000000000000000000000000000000000004E
:10526000000000000000000000000000000000003E
:020000040801F1
:1000000000070020810F01080D7C0108697B0108B1
:10001000D57B0108697B0108A17B0108830F0108DA
:10002000830F0108830F0108830F0108FDC1010838
:10003000830F0108830F0108830F0108830F010854
:10004000830F0108830F0108830F0108830F010844
:10005000830F0108830F010819E9010841E901082C
:1000600069E9010891E90108B9E9010845C50108F4
:100070006DC5010899C50108C5C50108F1C501088C
:1000800019C6010845C60108C9C40108A56F0108C1
:10009000D16F0108E16F0108830F0108E1E9010850
:1000A000830F0108830F0108830F0108830F0108E4
:1000B000C9EA0108830F0108830F0108830F0108B3
:1000C000830F0108830F0108830F0108830F0108C4
:1000D000830F0108B5EA0108830F0108830F0108A7
:1000E00045EA0108830F0108830F0108830F010807
:1000F000830F0108830F0108830F010871C60108EF
:10010000830F0108830F0108830F0108830F010883
:10011000830F0108830F0108830F0108830F010873
:100120009DC60108C5C60108F1C601081DC7010822
:1001300049C70108830F0108830F0108830F0108D5
:10014000830F0108830F0108830F0108830F010843
:1001500071C701089DC70108C9C70108830F0108BD
:10016000830F0108830F0108830F0108830F010823
:10017000830F0108830F0108830F0108830F010813
:10018000830F0108830F0108830F0108830F010803
:10019000830F0108830F0108830F0108830F0108F3
:1001A000830F0108830F0108830F0108830F0108E3
:1001B000830F0108830F0108830F0108830F0108D3
:1001C000830F0108830F0108830F0108830F0108C3
:1001D000830F0108830F0108830F0108830F0108B3
:1001E0006D14010869570108597501088DB101089E
:1001F00040A2E4F164689106B8708AD8796B2BB09C
:100200009069010003BEC59300006E04FFFFFFFF6D
:10021000FFFFFFFF81F0004102E000BF83F00043D9
:1002200030B54FEA41044FEA430594EA050F08BF91
:1002300090EA020F1FBF54EA000C55EA020C7FEA55
:10024000645C7FEA655C00F0E2804FEA5454D4EBD2
:100250005555B8BF6D420CDD2C4480EA020281EA9C
:10026000030382EA000083EA010180EA020281EAD4
:100270000303362D88BF30BD11F0004F4FEA013126
:100280004FF4801C4CEA113102D0404261EB410135
:1002900013F0004F4FEA03334CEA133302D05242BB
:1002A00063EB430394EA050F00F0A780A4F1010477
:1002B000D5F1200E0DDB02FA0EFC22FA05F28018B1
:1002C00041F1000103FA0EF2801843FA05F3594197
:1002D0000EE0A5F120050EF1200E012A03FA0EFC16
:1002E00028BF4CF0020C43FA05F3C01851EBE37140
:1002F00001F0004507D54FF0000EDCF1000C7EEB5D
:1003000000006EEB0101B1F5801F1BD3B1F5001F9A
:100310000CD349085FEA30004FEA3C0C04F10104B9
:100320004FEA445212F5800F80F09A80BCF1004FE2
:1003300008BF5FEA500C50F1000041EB045141EA64
:10034000050130BD5FEA4C0C404141EB0101013C2D
:1003500028BFB1F5801FE9D291F0000F04BF01461C
:100360000020B1FA81F308BF2033A3F10B03B3F1EE
:1003700020020CDA0C3208DD02F1140CC2F10C027E
:1003800001FA0CF021FA02F10CE002F11402D8BFDC
:10039000C2F1200C01FA02F120FA0CFCDCBF41EAA8
:1003A0000C019040E41AA2BF01EB0451294330BD77
:1003B0006FEA04041F3C1CDA0C340EDC04F1140454
:1003C000C4F1200220FA04F001FA02F340EA03002B
:1003D00021FA04F345EA030130BDC4F10C04C4F171
:1003E000200220FA02F001FA04F340EA0300294651
:1003F00030BD21FA04F0294630BD94F0000F83F49B
:10040000801306BF81F480110134013D4EE77FEA7D
:10041000645C18BF7FEA655C29D094EA050F08BFC9
:1004200090EA020F05D054EA000C04BF19461046AA
:1004300030BD91EA030F1EBF0021002030BD5FEAEE
:10044000545C05D14000494128BF41F0004130BD16
:1004500014F580043CBF01F5801130BD01F000456A
:1004600045F0FE4141F470014FF0000030BD7FEADD
:10047000645C1ABF194610467FEA655C1CBF0B46D8
:10048000024650EA013406BF52EA033591EA030FEF
:1004900041F4002130BD00BF90F0000F04BF0021E7
:1004A000704730B54FF4806404F132044FF000051A
:1004B0004FF0000150E700BF90F0000F04BF002193
:1004C000704730B54FF4806404F1320410F00045F9
:1004D00048BF40424FF000013EE700BF42004FEAF4
:1004E000E2014FEA31014FEA02701FBF12F07F4371
:1004F00093F07F4F81F06051704732F07F4208BF28
:10050000704793F07F4F04BF41F40021704730B52E
:100510004FF4607401F0004521F000411CE700BF7A
:1005200050EA010208BF704730B54FF000050AE0FD
:1005300050EA010208BF704730B511F0004502D5FE
:10054000404261EB41014FF4806404F132045FEA00
:10055000915C3FF4D8AE4FF003025FEADC0C18BFA9
:1005600003325FEADC0C18BF033202EBDC02C2F19B
:10057000200300FA03FC20FA02F001FA03FE40EA2D
:100580000E0021FA02F11444BDE600BF70B54FF031
:10059000FF0C4CF4E06C1CEA11541DBF1CEA13550F
:1005A00094EA0C0F95EA0C0F00F0DEF82C4481EA77
:1005B000030621EA4C5123EA4C5350EA013518BF97
:1005C00052EA033541F4801143F4801338D0A0FB84
:1005D00002CE4FF00005E1FB02E506F00042E0FB31
:1005E00003E54FF00006E1FB03569CF0000F18BF37
:1005F0004EF0010EA4F1FF04B6F5007F64F54074DF
:1006000004D25FEA4E0E6D4146EB060642EAC62171
:1006100041EA55514FEAC52040EA5E504FEACE2EDE
:10062000B4F1FD0C88BFBCF5E06F1ED8BEF1004FE1
:1006300008BF5FEA500E50F1000041EB045170BD5D
:1006400006F0004646EA010140EA020081EA0301A1
:10065000B4EB5C04C2BFD4EB0C0541EA045170BD9D
:1006600041F480114FF0000E013C00F3AB8014F117
:10067000360FDEBF002001F0004170BDC4F1000460
:10068000203C35DA0C341BDC04F11404C4F12005E1
:1006900000FA05F320FA04F001FA05F240EA02003C
:1006A00001F0004221F0004110EBD37021FA04F672
:1006B00042EB06015EEA430E08BF20EAD37070BD2C
:1006C000C4F10C04C4F1200500FA04F320FA05F08B
:1006D00001FA04F240EA020001F0004110EBD3708D
:1006E00041F100015EEA430E08BF20EAD37070BDFD
:1006F000C4F1200500FA05F24EEA020E20FA04F3D6
:1007000001FA05F243EA020321FA04F001F0004184
:1007100021FA04F220EA020000EBD3705EEA430EF5
:1007200008BF20EAD37070BD94F0000F0FD101F024
:100730000046400041EB010111F4801F08BF013C5D
:10074000F7D041EA060195F0000F18BF704703F09B
:100750000046520043EB030313F4801F08BF013D22
:10076000F7D043EA0603704794EA0C0F0CEA1355DE
:1007700018BF95EA0C0F0CD050EA410618BF52EA98
:100780004306D1D181EA030101F000414FF000009E
:1007900070BD50EA410606BF1046194652EA4306AC
:1007A00019D094EA0C0F02D150EA013613D195EA20
:1007B0000C0F05D152EA03361CBF104619460AD168
:1007C00081EA030101F0004141F0FE4141F4700172
:1007D0004FF0000070BD41F0FE4141F4780170BD62
:1007E00070B54FF0FF0C4CF4E06C1CEA11541DBFC7
:1007F0001CEA135594EA0C0F95EA0C0F00F0A7F8C9
:10080000A4EB050481EA030E52EA03354FEA0131F5
:1008100000F088804FEA03334FF0805545EA131308
:1008200043EA12634FEA022245EA111545EA1065D0
:100830004FEA00260EF000419D4208BF964244F167
:10084000FD0404F5407402D25B084FEA3202B61A86
:1008500065EB03055B084FEA32024FF480104FF45A
:10086000002CB6EB020E75EB030E22BFB61A7546CE
:1008700040EA0C005B084FEA3202B6EB020E75EB61
:10088000030E22BFB61A754640EA5C005B084FEAC9
:100890003202B6EB020E75EB030E22BFB61A754696
:1008A00040EA9C005B084FEA3202B6EB020E75EBA1
:1008B000030E22BFB61A754640EADC0055EA060E62
:1008C00018D04FEA051545EA16754FEA06164FEAA5
:1008D000C30343EA52734FEAC2025FEA1C1CC0D151
:1008E00011F4801F0BD141EA00014FF000004FF0DE
:1008F000004CB6E711F4801F04BF01430020B4F19F
:10090000FD0C88BFBCF5E06F3FF6AFAEB5EB030C56
:1009100004BFB6EB020C5FEA500C50F1000041EB53
:10092000045170BD0EF0004E4EEA113114EB5C0420
:10093000C2BFD4EB0C0541EA045170BD41F48011F3
:100940004FF0000E013C90E645EA060E8DE60CEAFB
:10095000135594EA0C0F08BF95EA0C0F3FF43BAF18
:1009600094EA0C0F0AD150EA01347FF434AF95EACF
:100970000C0F7FF425AF104619462CE795EA0C0FB3
:1009800006D152EA03353FF4FDAE1046194622E780
:1009900050EA410618BF52EA43067FF4C5AE50EA5A
:1009A00041047FF40DAF52EA43057FF4EBAE12E74A
:1009B0004FF0FF3C06E000BF4FF0010C02E000BF2B
:1009C0004FF0010C4DF804CD4FEA410C7FEA6C5C0E
:1009D0004FEA430C18BF7FEA6C5C1BD001B050EAB1
:1009E000410C0CBF52EA430C91EA030F02BF90EA9C
:1009F000020F0020704710F1000F91EA030F58BF5B
:100A0000994208BF90422CBFD8176FEAE37040F0BC
:100A1000010070474FEA410C7FEA6C5C02D150EA5A
:100A2000013C07D14FEA430C7FEA6C5CD6D152EA15
:100A3000033CD3D05DF8040B704700BF84461046DA
:100A400062468C461946634600E000BF01B5FFF7D9
:100A5000B7FF002848BF10F1000F01BD4DF808EDA9
:100A6000FFF7F4FF0CBF012000205DF808FB00BF7A
:100A70004DF808EDFFF7EAFF34BF012000205DF8D4
:100A800008FB00BF4DF808EDFFF7E0FF94BF012021
:100A900000205DF808FB00BF4DF808EDFFF7CEFF22
:100AA00094BF012000205DF808FB00BF4DF808ED61
:100AB000FFF7C4FF34BF012000205DF808FB00BF32
:100AC0004FEA410C7FEA6C5C02D150EA013C0AD14A
:100AD0004FEA430C7FEA6C5C02D152EA033C02D13C
:100AE0004FF0000070474FF0010070474FEA41029D
:100AF00012F5001215D211D56FF47873B3EB625270
:100B000012D94FEAC12343F0004343EA505311F096
:100B1000004F23FA02F018BF404270474FF0000028
:100B2000704750EA013005D111F0004008BF6FF066
:100B3000004070474FF00000704700BF4FEA41028D
:100B4000B2F1E04324BFB3F5001CDCF1FE5C0DD92B
:100B500001F0004C4FEAC0024CEA5070B2F1004F75
:100B600040EB830008BF20F00100704711F0804F78
:100B700021D113F13872BCBF01F00040704741F43D
:100B800080114FEA5252C2F11802C2F1200C10FA41
:100B90000CF320FA02F018BF40F001004FEAC12325
:100BA0004FEAD32303FA0CFC40EA0C0023FA02F3C9
:100BB0004FEA4303CCE77FEA625307D150EA01339F
:100BC0001EBF4FF0FE4040F44000704701F000406F
:100BD00040F0FE4040F40000704700BF7BB972B99E
:100BE0000029BEBF00204FF0004106E008BF0028EA
:100BF0001CBF6FF000414FF0FF3000F0BFB9ADF106
:100C0000080C6DE904CE002909DB002B1ADB00F08B
:100C10004DF8DDF804E0DDE9022304B070474042FE
:100C200061EB4101002B1BDB00F040F8DDF804E034
:100C3000DDE9022304B0404261EB4101524263EB23
:100C400043037047524263EB430300F02FF8DDF893
:100C500004E0DDE9022304B0404261EB410170474A
:100C6000524263EB430300F021F8DDF804E0DDE9D4
:100C7000022304B0524263EB4303704753B94AB9AD
:100C8000002908BF00281CBF4FF0FF314FF0FF3094
:100C900000F074B9ADF1080C6DE904CE00F006F86F
:100CA000DDF804E0DDE9022304B070472DE9F047E8
:100CB000089D04468E46002B4DD18A42944669D940
:100CC000B2FA82F252B101FA02F3C2F1200120FA23
:100CD00001F10CFA02FC41EA030E94404FEA1C4871
:100CE000210CBEFBF8F61FFA8CF708FB16E341EA6D
:100CF000034306FB07F199420AD91CEB030306F1F3
:100D0000FF3080F01F81994240F21C81023E634413
:100D10005B1AA4B2B3FBF8F008FB103344EA0344B7
:100D200000FB07F7A7420AD91CEB040400F1FF33CC
:100D300080F00A81A74240F207816444023840EA09
:100D40000640E41B00261DB1D4400023C5E9004342
:100D50003146BDE8F0878B4209D9002D00F0EF80C5
:100D60000026C5E9000130463146BDE8F087B3FAF8
:100D700083F6002E4AD18B4202D3824200F2F980E0
:100D8000841A61EB030301209E46002DE0D0C5E9E3
:100D9000004EDDE702B9FFDEB2FA82F2002A40F02F
:100DA0009280A1EB0C014FEA1C471FFA8CFE012632
:100DB000200CB1FBF7F307FB131140EA01410EFBD6
:100DC00003F0884208D91CEB010103F1FF3802D27D
:100DD000884200F2CB804346091AA4B2B1FBF7F077
:100DE00007FB101144EA01440EFB00FEA64508D99A
:100DF0001CEB040400F1FF3102D2A64500F2BB80D7
:100E00000846A4EB0E0440EA03409CE7C6F1200725
:100E1000B34022FA07FC4CEA030C20FA07F401FA6B
:100E200006F31C43F9404FEA1C4900FA06F3B1FBF4
:100E3000F9F8200C1FFA8CFE09FB181140EA014159
:100E400008FB0EF0884202FA06F20BD91CEB0101F6
:100E500008F1FF3A80F08880884240F28580A8F14E
:100E600002086144091AA4B2B1FBF9F009FB1011A0
:100E700044EA014100FB0EFE8E4508D91CEB01013E
:100E800000F1FF346CD28E456AD90238614440EAE1
:100E90000840A0FB0294A1EB0E01A142C846A64661
:100EA00056D353D05DB1B3EB080261EB0E0101FAEA
:100EB00007F722FA06F3F1401F43C5E90071002647
:100EC0003146BDE8F087C2F12003D8400CFA02FC9D
:100ED00021FA03F3914001434FEA1C471FFA8CFEAD
:100EE000B3FBF7F007FB10360B0C43EA064300FB9D
:100EF0000EF69E4204FA02F408D91CEB030300F13B
:100F0000FF382FD29E422DD9023863449B1B89B2F1
:100F1000B3FBF7F607FB163341EA034106FB0EF37A
:100F20008B4208D91CEB010106F1FF3816D28B4227
:100F300014D9023E6144C91A46EA004638E72E46F3
:100F4000284605E70646E3E61846F8E64B45A9D2EB
:100F5000B9EB020864EB0C0E0138A3E74646EAE75A
:100F6000204694E74046D1E7D0467BE7023B614408
:100F700032E7304609E76444023842E7704700BF71
:100F800002E000F000F8FEE772B6374880F3088808
:100F9000364880F3098836483649086040F2000038
:100FA000CCF200004EF63471CEF200010860BFF3BF
:100FB0004F8FBFF36F8F40F20000C0F2F0004EF68B
:100FC0008851CEF200010860BFF34F8FBFF36F8FDF
:100FD0004FF00000E1EE100A4EF63C71CEF2000137
:100FE0000860062080F31488BFF36F8F0DF040FA7D
:100FF0000DF032FB4FF055301F491B4A91423CBF68
:1010000041F8040BFAE71D49184A91423CBF41F8E8
:10101000040BFAE71A491B4A1B4B9A423EBF51F890
:10102000040B42F8040BF8E700201849184A9142D3
:101030003CBF41F8040BFAE70DF01EFA0DF060FB1F
:10104000144C154DAC4203DA54F8041B8847F9E7F9
:1010500000F0FCF9114C124DAC4203DA54F8041BB9
:101060008847F9E70DF006BA0007002000230020AA
:101070000000010808ED00E000010020000700204A
:10108000A867020800230020E8240020E8240020AC
:10109000E8A30020E0010108F0010108F0010108C7
:1010A000F00101082DE9F04F2DED108AC1F80CD0A8
:1010B000C3689D46BDEC108ABDE8F08F002383F322
:1010C00011882846A04700200CF09EFCFEE70CF09B
:1010D0003DFB00DFFEE7000010F8012B11F8013B9B
:1010E000012A28BF9A42F7D0D01A7047034613F856
:1010F000012B002AFBD1181A0138704701F0FF01BB
:10110000102A2BDB10F0070F08D010F8013B013A32
:101110008B422DD010F0070F42B3F6D1F0B441EA64
:10112000012141EA014122F007047FF0000700237A
:10113000F0E80256083C85EA010586EA010685FAD0
:1011400047F5A3FA87F586FA47F6A5FA87F68EB92A
:10115000EED1F0BC01F0FF0102F0070232B110F84D
:10116000013B013A83EA010313B1F8D10020704733
:1011700001387047002D06BF35460338073815F093
:10118000010F07D1013015F4807F02BF013015F443
:10119000C03F0130F0BC0138704700BF704700000D
:1011A00070B50446183004F03FFC04F13C0000F038
:1011B000A9F9154B1549196004F1500000231426B4
:1011C0009DB206FB05120133127C002AF8D1104BA8
:1011D0001D80104B1A6812B10F4806F01BFD1860F5
:1011E00004F58053012104F581505A6383F83210CD
:1011F000183005F03FFF094B1A680AB10848ECE7C0
:101200001C60204670BD00BFF43500206015020848
:10121000F0350020B835002080140208E8240020B2
:101220009B14020838B51A4D04460DF0D7F80DF09E
:10123000E9F8286820231A46006C4FF4E13102F0E7
:1012400099F928684FF4807380224FF4E131C06C23
:1012500002F090F9204600F02DF90DF0D3F8204669
:1012600001F08EF804F1180004F09AFC0DF0CAF8B1
:1012700005F036F82B68D86A03685B68984710B1A8
:10128000044805F013FFBDE8384006F0EDBC00BF90
:1012900008250020BC1402080148FFF7C3BF00BFA7
:1012A0000C2500202DE9F341144C154EDFF8608029
:1012B000144F20460DF088F8134A0146121B1348BC
:1012C00001F020F90CF066F90446A4B1206AE16946
:1012D0000191B04214BF251AA8EB06050DF074F871
:1012E000019902462B46384601F00CF920460CF0D5
:1012F00061F90446E9E702B0BDE8F0810001002091
:1013000000070020E614020800070020DC14020891
:101310000023002010B50F4C03F0C4FC2368986A2A
:1013200003680522DB69002198472368986A0368EF
:1013300064211B6998472368986A036828215B68C1
:1013400098472368986A0368BDE810401B6900212C
:10135000184700BF0825002038B5054606F084FC74
:101360002C4A1368C31AB3F57A7F044608D92A4B6E
:1013700010601B7823B9294A536983F48053536161
:1013800004F0DEFC264A136841F28831E31A8B42EE
:1013900006D9016821B114600289224801F0B2F82F
:1013A0006B7ADA070AD5204A136841F28831E31ACA
:1013B0008B4203D928461460FFF774FF6B7A9B07B2
:1013C0000CD4284600F0A8F8184A1368E31A132B27
:1013D0001DD82846BDE8384001F016B906F044FC97
:1013E00043F698239842ECD91148FFF793FF114830
:1013F0000CF0C2FFBFF34F8F0F49104BCA6802F4C5
:10140000E0621343CB60BFF34F8F00BFFDE7146072
:10141000DFE700BFEC24002000230020000802408A
:10142000F4240020F8140208F0240020F8240020FE
:101430000C250020010007B000ED00E00400FA05D3
:101440000148FFF789BF00BF0C25002038B5054BC8
:101450001C6823680A461D68034B01462046A847BE
:10146000002038BD08250020FC24002010B50A4CBF
:101470002046FFF795FE094A094920460DF064FB16
:1014800006F062F8074B084A1860BDE810400749AB
:10149000074801F08FBF00BF0C250020A078002076
:1014A0009D11010808250020411401089912010826
:1014B000FC24002013B5044603F0ACFF03F032F91E
:1014C000204603F027FF18B1B4F90030022B0BD0EF
:1014D00004F012FA02F0F8FD02230DF10601204695
:1014E000ADF8063004F0BCF902230DF106012046E8
:1014F000ADF8063004F0AAF902B0BDE8104003F0E0
:1015000093BC000010B50349044603F0B7FE204623
:1015100010BD00BF341602082DE9F0412DED028BFD
:1015200090F93C60002E86B0044640F39680856CAE
:10153000F5B9B00001F0EEFDA064002800F08D8048
:101540004B4B84F84C60D3F80080D8F8100094F925
:101550003E100368A66C5B6851FA85F19847EFB2BC
:10156000013546F8270094F84C20EBB29A42ECD8AB
:1015700006F07AFBD4ED106A9FED3E6A636C86EE4E
:10158000267AC31A07EE903AF8EE677AF4EEC77A35
:10159000F1EE10FA61D460644FF4836001F0B4FDA1
:1015A00005464FF4047001F0B5FD064645B180B91B
:1015B000284606B0BDEC028BBDE8F04101F0ACBDA1
:1015C00000284AD006B0BDEC028BBDE8F04101F026
:1015D000A7BD94F84C309FED288A2B724FF000087D
:1015E00094F84C305FFA88F7BB4211D9A36C53F8DA
:1015F000270050B10368DB68984730EE488A05EB56
:10160000870787ED038AB0EE408A08F10108E7E713
:1016100005F20C42194B136005F5826231461360E6
:1016200094F83D3085F815340122284601F06EF813
:101630000023049380B244F624631822CDE90260AB
:10164000CDE90032204608A3D3E9002300F04AF98F
:10165000284601F061FD3046B4E706B0BDEC028BD0
:10166000BDE8F081AFF3008082484875FC497F7D7A
:101670000825002000007A44000000000000C07F20
:10168000BFF34F8F0549064BCA6802F4E06213436B
:10169000CB60BFF34F8F00BFFDE700BF00ED00E060
:1016A0000400FA0513B51022002104468DF8072026
:1016B0000DF07CFA054B1B68D86A03680DF1070230
:1016C0001B6B2146984702B010BD00BF08250020C3
:1016D000F0B58BB0174604460E4606F0C5FA05462F
:1016E00002F0B2FC03464FF4C87005F5167504F518
:1016F0008054B3FBF0F202FB103315FA83F3E3627C
:10170000FD7E35B91D4805F0D1FC84F830500BB092
:10171000F0BD384605A901F075FA07460028F6D154
:1017200001A8FFF7BFFF9DF8165001A92A460DF149
:1017300017000DF01DFA28B1114805F0B7FC84F828
:101740003070E4E70F2D0AD8E36A84F83050A3F52F
:101750001673E36229460B4805F0A8FCD7E79DF80D
:1017600014100029D3D030460AF05AF89DF81420FE
:1017700094F83210044805F099FCC8E78416020872
:10178000AF160208D0160208F216020807B5104676
:1017900001A901F0E5F858B9074B9DF804101B6842
:1017A000D86AA1F1FF02036851421B685141984772
:1017B00003B05DF804FB00BF0825002038B50846DB
:1017C00015461C460AF034F860B99DF81030022B1B
:1017D00007D1012C05D11BA3D3E90023C5E90023C0
:1017E000012038BD0B2C0BD884B1601E0A280DD8FF
:1017F000DFE800F00E0C0C0C160C0C0C0C1E1A0082
:10180000282C09D040F24C439C4215D00020E8E738
:101810000EA3D3E90023E1E70EA3D3E90023DDE71C
:101820000EA3D3E90023D9E70EA3D3E90023D5E71C
:101830000EA3D3E90023D1E70EA3D3E90023CDE71C
:10184000AFF30080401DA12026812A0B9E6AC4218F
:10185000818A46EE26417272DF25D7B7F017304AEB
:1018600039059E56D5A4D139F922B6A7CDD269EB58
:10187000C51A133B03806A5575F3008713B59DF8AD
:101880001040CDE9003413460A460146806AFFF74E
:1018900095FF02B010BD000070B500F580560D46F2
:1018A000B46A74B90C2101200CF05EFCB06208B976
:1018B000002070BD056084600430FAE72646A46805
:1018C00024B12368AB42F9D1201DF2E70C2101209D
:1018D0000CF04AFCB0600028EAD00560B3689C6058
:1018E000B068E9E72DE9F04190B000F58151BDF80D
:1018F000587004461646183140F2434201A89846F3
:1019000001F096FD012F0ED146EA07412046FFF770
:10191000C3FF054670B9002401A801F0A5FD2046CB
:1019200010B0BDE8F08104F1580009F081FF0028F3
:10193000EAD1F0E73822002102A80DF037F902239E
:101940008DF808309DF85C308DF82030189B099395
:10195000BDF86430ADF82830CDE90468ADF81870F2
:10196000079506F083F90D4BC01841F10001CDE950
:101970000C0104F1580002A909F05CFF084B002893
:10198000D5BF9A881A6801321218D4BF9A801A609B
:101990000028D4BF00240124BEE700BF40420F004E
:1019A0006835002030B58FB014460D46382200212E
:1019B00068460DF0FBF8DDE91223CDE90223BDF8FE
:1019C0005030ADF8103004F119030593A37E8DF863
:1019D0001830159B0793BDF85830ADF8203006F04D
:1019E00045F90D4BC31841F100016A46CDE90A31B2
:1019F0002846E17E09F062FF084B0028D5BF9A888F
:101A00001A6801321218D4BF9A801A600028D4BF15
:101A1000002001200FB030BD40420F00683500208B
:101A2000F0B591B005460E46104608A9144601F0DF
:101A3000B1F938BB9DF82030012B07D103F05CFFD2
:101A400002F042FB03F0F0F903F0E4FC1022002165
:101A500006AF0CA80DF0AAF8012239460CA88DF8A3
:101A6000382001F0BBF90A23029307A3D3E900232E
:101A700080B2CDE90370CDE90023314622462846E5
:101A8000FFF790FF11B0F0BDCDD269EBC51A133B43
:101A90002DE9F041ADF5487D66AC05460E4617468A
:101AA00000214FF4C47220460DF080F806F0DCF8F7
:101AB0002F4B4FF47A72B0FBF2F0186093E80700F6
:101AC00084E8070001F01CFB037C237401F018FB81
:101AD000437C63740323A374264B5A6962610DF53A
:101AE000DD709A68DB68A261E361FFF7DBFD46F613
:101AF0000463EA682384204B002A18681F4B29DD01
:101B0000CDE900320DF2CB211D4BC06A502201F00D
:101B1000CDFD50210DF2CB200DF01EFD0DF11C0866
:101B200084F8320141460122204600F033FF0123B0
:101B300002930DA3D3E9002380B2CDE90380CDE960
:101B4000002331463A462846FFF72CFF0DF5487D25
:101B5000BDE8F081009350220A4BC06A0DF2CB2100
:101B600001F0A4FDD5E700BF9E6AC421818A46EE3C
:101B70005C350020F0010108082500201717020835
:101B800010170208171902082DE9F0411546ADF5A6
:101B9000866D06460F460CF035FC08A9284601F074
:101BA00033F90446002840F09F8001464FF4D0727C
:101BB000A4A80CF0FBFF9DF8B880B8F1100F7ED8F8
:101BC00008F1FF330F2B2BD842460DF1B9010DF26E
:101BD000D1300CF0DDFF424651490DF1B9000DF056
:101BE00093FC0246B0B94F480DF11F0102F088FF87
:101BF0000446002C63D09DF8B83073B39DF82830AC
:101C00005BB39DF81F20013A032A6DD8DFE802F08C
:101C10001C2E384122460DF11F010DF2D130E5E7AF
:101C2000BDF82000479447AA0DF11F0103F0DCFA2C
:101C30000446002843D0012300930DF2D132112332
:101C400047A902F099FED4E7012B4DD10C9B8DF8EA
:101C50001C3147A9204603F0E5FD9DF81F30013BEC
:101C6000032B41D8DFE803F01C444A4F012B3BD142
:101C70000C9BADF81C3147A9204603F00BFEECE7A6
:101C8000012B31D10C9B479347A9204603F024FE3A
:101C9000E3E7022B28D10CA9204603F095FDDCE7F1
:101CA00001238DF8903294F90030DA17CDE9A6328D
:101CB0005C210DF2D1300DF04FFC8DF8D00347AC14
:101CC00001222146A4A801F0C7F90B23029312A315
:101CD000D3E9002380B2CDE90340CDE900233946A2
:101CE0002A463046FFF75EFE0DF5866DBDE8F081B1
:101CF00001238DF89032B4F90030D6E701238DF836
:101D000090322368D1E702238DF890322368A6939E
:101D1000CEE700BFAFF30080D5A4D139F922B6A732
:101D200038170208411702082DE9F04FDFF8D8A054
:101D30008BB0804608F15809484609F0FBFD05467E
:101D4000002858D00024007E0694CDE90744ADF861
:101D5000244001F0F3FA2A7E8DF8240005F11001E9
:101D600007A80CF015FF2B6843F00043069305F01D
:101D70007DFF224B0390C218DAF804000E4641F1B1
:101D8000000308F5805760B30168009409690D46A7
:101D900006A9A847A04224DCDAF8040003689B6A7D
:101DA0009847D0E90A23CDE9042305F05FFFDDE978
:101DB0000423801A61EB0301114B834274EB01038E
:101DC0000FD397F83130072B12D90E4A87F83140DC
:101DD0009388013393804846039A334609F0B8FD4F
:101DE00009E0484609F0AAFD002387F83130A1E751
:101DF000013387F831300BB0BDE8F08F40420F005F
:101E00007F841E0068350020883500202DE9F041D0
:101E10004FF00053DFF8E0801B684345FCB00546F7
:101E20000C46164604D03148DC2200210CF0BEFEE0
:101E30004FF0005749A9C7F80080304600F02EFF48
:101E4000002849D19DF824313B750BB9F37E3B75D1
:101E50009DF8252126480DF593710CF099FE20463A
:101E600009F0E6FC4FF0005307AF587581220021BE
:101E700028A80CF09BFE3946012228A800F054FF48
:101E80002823029317A3D3E9002380B2CDE903707E
:101E9000CDE90023214632462846FFF783FD154F42
:101EA0003326013E16F0FF06284608D0FFF73CFF18
:101EB0003B68986A036801215B689847F1E7FFF780
:101EC00029FA204609F0B4FC40F0304040F40020EC
:101ED0000CF052FAFFF7D4FB7CB0BDE8F08100BFF4
:101EE000AFF3008026417272DF25D7B704000020CF
:101EF00016000020082500209AAD44C5F0B5044620
:101F000089B008460E46154609F092FC68B92B7E4A
:101F1000022B1FD1EB8A012B1CD12A4631462046C9
:101F200009B0BDE8F040FFF7D3BBEB8A0B2B0BD811
:101F300083B1013B0A2B0DD8DFE803F00E0C0C0C2B
:101F40001E0C0C0C0C463E00282B0DD040F24C42CF
:101F5000934241D009B0F0BD2A463146204609B02F
:101F6000BDE8F040FFF794BD2A463146204609B04F
:101F7000BDE8F040FFF74ABF07AF1E4805F096F8EE
:101F80000122394606A88DF8182000F0DDFD052352
:101F9000029316A3D3E9002380B2CDE90023CDE953
:101FA00003702A4631462046FFF7FCFC05F05CFE34
:101FB00004F580546063CDE72A463146204609B0D7
:101FC000BDE8F040FFF7E0BD2A463146204609B0A3
:101FD000BDE8F040FFF724BD2A463146204609B04F
:101FE000BDE8F040FFF7D2BBAFF30080F017304AF6
:101FF00039059E564C1702080A460146806AFFF7CB
:102000007DBF000049421B4B112912D8DFE801F0C7
:102010000911110D1111111111111519151D21257C
:10202000292D9A6801329A6070479A8901329A8103
:102030007047DA890132DA8170475A8B01325A834C
:1020400070471A8B01321A8370471A8A01321A823A
:1020500070475A8A01325A8270479A8B01329A83AA
:1020600070479A8A01329A827047DA8A0132DA829C
:10207000704700BF683500202DE9F04F374E97B00C
:102080000023CDE90B330A93ADF83430736804466E
:10209000002B5FD0324D01274FF0000A4FF0000BAC
:1020A00070688DF814704FF000088DF81580036883
:1020B000CDE900AB0DF11502D3F8089005A9434610
:1020C000C8479DF81430002B44D0414620220EA86A
:1020D0000CF06CFD7068036806AAD3F814800AA996
:1020E0000DF11603C047002834DD9DF8340001F0DF
:1020F00041F90BA902468DF8500012A80CF048FDDA
:1021000004F158080A9B0E930EA9DDE90623404608
:1021100009F04CFE10F10D0F014603D02046FFF7E9
:1021200071FFBDE70E9809F031FE03900E9809F09B
:1021300027FE039BCDE9000708AA41462046FFF78A
:102140003DFB18B12B8A01332B82A9E76B8B01333E
:102150006B83A5E717B0BDE8F08F00BF883500207E
:102160006835002007B500F15801684609F0D2FD36
:10217000BDF8040064235843BDF80030B0FBF3F011
:1021800080B203B05DF804FBF0B597B0044605F0EB
:102190006BFD4FF47A73B0FBF3F0434B434D1B6878
:1021A0002860D86A03685B6D98474FF6FF739842C2
:1021B00028BF184628810EA90122284600F09CFC61
:1021C0000EAB80B20293182240F255130025CDE9E0
:1021D000003203902EA3D3E9002304952046FFF795
:1021E00081FB637A59074ED501220EA93048314F41
:1021F00000F05AFB0EAB80B202931F264FF4AB7374
:10220000CDE90036039024A3D3E9002304952046AA
:10221000FFF768FB786803689B6A9847002832D00C
:102220003A788DF8382002680F924268ADF8402065
:102230008268ADF84220C268ADF844200269ADF86A
:1022400046204269ADF8482082691392C269ADF810
:102250005020026AADF8522007AF436AADF85430FF
:10226000012239460EA800F0C9FA40F2571380B295
:10227000CDE902700093049509A3D3E900230196E8
:102280002046FFF72FFB17B0F0BD00BFAFF3008073
:10229000F1C6A7C1D068080FD1F886A9B8E33A768D
:1022A000753CA33CAE0C08CE082500205C35002010
:1022B0006835002088350020F0B506468DB05830CE
:1022C00009F0B6FA2C4D20B100232B7001200DB07F
:1022D000F0BD05F0C9FC2B7804463BB13046FFF752
:1022E00041FF01210246254804F0E0FE01F0ACFE6A
:1022F0004FF4C87306F58057B0FBF3F202FB1303EB
:1023000004F5167010FA83F000238DF8183097F852
:102310003030F86223B901228DF8182087F8323066
:1023200008A8FFF7BFF997F83010C1F11004E4B224
:10233000062C28BF062408AB224619440DF11900CB
:102340000CF026FC013406AB002502931822012371
:10235000E4B2CDE90032049505A3D3E90023039448
:102360003046FFF7BFFA87F830502846AFE700BF86
:10237000401DA12026812A0B002300205C170208A3
:1023800070B5244D244E4FF4807386B0AB80044664
:1023900005F06AFC4FF47A73B0FBF3F028606288B2
:1023A000B4F902307F2A98BF33700DF11701002372
:1023B00004F108008DF8173003F034FA41F23810B8
:1023C00000F0A2FE054608B104F044FA134B1D606C
:1023D000134B00225D601A702DB12B6861685B6839
:1023E0000122284698470F4B009304F1580004F14E
:1023F00088010D4B01944FF47A62039009F0E4F9DF
:102400003178039821B106B0BDE8704009F008BAF0
:1024100006B070BD5C3500209D3500209035002051
:10242000883500207D180108F91F01082DE9F04FBB
:102430000628ADF5217D0C4698BF3049DFF8C0A0D5
:1024400098BF11F8009013464FF0000288BF9146E4
:10245000469200214FF4B27247A807930CF0A6FBF6
:10246000079B22464FF4B47146A804F00FFE21A743
:10247000D7E9006720EAE0754FF004084FF0000B41
:1024800095B37C22002127A80CF090FB5A2D2C46F6
:1024900028BF5A2446AB22468DF8BD402D1B5C4414
:1024A00003EB0B010DF1BE001FFA84FB08AC8DF8A5
:1024B0009C900CF06DFB0122214627A800F04EFBFA
:1024C0000023049380B243F6FF731822CDE9003253
:1024D000CDE9024032463B46504608F1FF38FFF74F
:1024E00001FA18F0FF08CBD10DF5217DBDE8F08F82
:1024F000AFF30080759D040C8EA454D61818020802
:102500000C2500200FB407B504AA072052F8041BBD
:102510000192FFF78BFF03B05DF804EB04B0704746
:1025200037B50446583009F013FA2046FFF71AFE73
:10253000462802D92A4804F0B9FD2046FFF724FEB8
:1025400094F90850002D38D0002304F10800EDB2B2
:1025500001A98DF8043003F065F92A2D214C0AD128
:10256000214D2846FFF7CEFF2368986A036864214F
:102570005B689847F5E72B2D04D11C48FFF7C2FF95
:102580001B4B98474FF4FA6101A800F037FF24680D
:10259000A06A03684FF47A715B689847E06A036841
:1025A0009B6A984718B1012816D0124800E01248DB
:1025B000FFF7A8FF01A800F02DFF104B00225A7171
:1025C00005F052FB47F23053984207D90C4803B04C
:1025D000BDE830400BF0D0BE0A48E9E703B030BD9B
:1025E0009417020808250020B2170208C317020832
:1025F00038ED00E0FE170208D31702085C35002012
:10260000263A09B0E81702082DE9F341044605F01F
:102610002BFB38490B68C31A322B05461BD9364BA6
:102620001B78C3B1354802780123934023F4AA43B1
:1026300023F055031B041B0C002B0EBF01260026A4
:102640004FF4805343EA067301322D4E02F01F020D
:10265000B36102700D6004F5805605F005FBF36A66
:10266000984202D92046FFF727FE264A1368EB1A44
:10267000B3F57A7F07D3156005F0F8FA02460B46EA
:102680002046FFF74DFF05F0EBFA04F58155DFF822
:1026900078800746183505F0E3FAC01BB0F57A7F5D
:1026A00017D2D8F80030986A03684FF480619B68AD
:1026B000984740F2D772294601A800F0B9FE20469B
:1026C000FFF732FB2046FFF7D7FC01A800F0CCFE55
:1026D000E1E7736B5BB105F0C7FA736BC01AB0F535
:1026E0007A7F04D92046FEF715FEFEF7C9FF02B037
:1026F000BDE8F08198350020002300209C350020A3
:102700000008024094350020082500202DE9F743F9
:102710000C4606464FF40472002120460CF046FA9F
:10272000334638220021204609F0ACFA337A8DF87E
:10273000053008220DF105033821204609F0A2FAE0
:1027400006F10C09402500279DF805309F4205F150
:10275000100843D306F5816329462046102209F06C
:1027600091FA414606F20A431022204609F08AFAFD
:1027700006F20C4393ED000A09F0D4FA05F12001AA
:10278000ADF806000DF106031022204609F07AFA92
:1027900006F5826393ED000A09F0C4FA0DF1060311
:1027A000ADF8060005F130012046102209F06AFA62
:1027B00006F2144305F140012046012209F062FAB5
:1027C000204606F21543082205F1410109F05AFAA4
:1027D00005F15000C00803B0BDE8F083B9EC010A70
:1027E00009F0A0FA2946ADF806000DF10603102203
:1027F000204609F047FA01374546A5E770B50C4673
:10280000192605463246002120460CF0CFF92B460A
:1028100020460822002109F035FA2B1D20462022EF
:10282000082109F02FFA05F108032046102228217B
:1028300009F028FA05F10A0320461022382109F090
:1028400021FA05F10C0320461022482109F01AFA5A
:1028500005F10E0320461022582109F013FA05F164
:10286000100320461022682109F00CFA05F1140328
:1028700020462022782109F005FA05F118032046A8
:102880001022982109F0FEF905F11A0320461022C2
:10289000A82109F0F7F9204605F11C031022B82100
:1028A00009F0F0F9304670BD70B50C461C2605469F
:1028B0003246002120460CF079F92B462046202292
:1028C000002109F0DFF92B1D20461022202109F0FC
:1028D000D9F905F1080320462022302109F0D2F968
:1028E00005F10C0320461022502109F0CBF905F127
:1028F0000E0320461022602109F0C4F905F11003EF
:1029000020461022702109F0BDF905F1120320467E
:102910001022802109F0B6F905F114032046102297
:10292000902109F0AFF905F1160320461022A021ED
:1029300009F0A8F905F1180320461022B02109F08A
:10294000A1F905F11A0320461022C02109F09AF9D5
:102950002046AB191022D02109F094F9304670BD01
:1029600013B50446007F10B1A38A012B0CD80023B5
:10297000009108221946204609F046F8237FA08AD4
:1029800023B9B0FA80F0400902B010BD013818BF79
:102990000120F9E72DE9F3470D4604460021904652
:1029A000284640F279120CF001F92346202200213A
:1029B000284609F067F9231D02222021284609F044
:1029C00061F9631D03222221284609F05BF9A31D4A
:1029D00003222521284609F055F904F108031022A5
:1029E0002821284609F04EF904F110030822382165
:1029F000284609F047F904F111030822402128462E
:102A000009F040F904F1120308224821284609F090
:102A100039F904F1140320225021284609F032F933
:102A200004F1180340227021284609F02BF904F123
:102A300020030822B021284609F024F904F12103DB
:102A40000822B821284609F01DF904F12207C02602
:102A50003B46314608222846083609F013F9B6F5F8
:102A6000A07F07F10107F3D194F832308DF80730D9
:102A700031460DF107030822284609F003F9002624
:102A800004F1330A9DF807304FEAC6099E4209F562
:102A9000A47720D394F83231502B28BF50238DF8DF
:102AA0000730B8F1000F08D139460DF107030722AE
:102AB000284609F0E7F809F24F17002604F233140C
:102AC0009DF807309E4207EBC6010DD30731C808B9
:102AD00002B0BDE8F0870AEB060308223946284613
:102AE00009F0D0F80136CDE7A3190822284609F0ED
:102AF000C9F80136E4E7000013B504460846002192
:102B000001602346C0F803102022019009F0BAF8B2
:102B10000198231D0222202109F0B4F80198631DB9
:102B20000322222109F0AEF80198A31D03222521DA
:102B300009F0A8F8019804F108031022282109F0EF
:102B4000A1F8072002B010BD08B5034608460021D1
:102B50000170012209F096F8012008BD2DE9F3412A
:102B60000D4604460021164628467B220CF01EF82E
:102B7000234603220021284609F084F863781F2B9E
:102B800028BF1F238DF8063005220DF1060303210F
:102B9000284609F077F801239DF80620DF0003F1AD
:102BA0000108013B9A421CD894F821305A2B28BFC7
:102BB0005A238DF807303EB939460DF10703072235
:102BC000284609F05FF80737002622349DF80730C1
:102BD0009E4207EBC6010DD30731C80802B0BDE81D
:102BE000F08104EB080308223946284609F04AF828
:102BF0004346D1E7A3190822284609F043F80136D5
:102C0000E4E70000F7B5047F05460E462CB1838A41
:102C1000122B02D9012003B0F0BD00231946072270
:102C20000096284608F0F0FE731C00930122002352
:102C30000721284608F0E8FED4B9B31C009305220A
:102C400023460821284608F0DFFE0D24B378102B18
:102C5000E0D83746B278BB1B934210D32B7FA88AAB
:102C60000734E408B3B9844294BF00200120D2E7BE
:102C7000AB8ADB00083BDB08B3700824E6E7FB1CEB
:102C80000093214600230822284608F0BDFE0834A0
:102C90000137DFE7201A18BF0120BCE7F7B5047F32
:102CA00005460E462CB1838ACA2B02D9012003B0F7
:102CB000F0BD0023194600960822284608F0A4FE1D
:102CC000731CD4B90822009311462346284608F005
:102CD0009BFE10247378C82BE8D8012372785F1C00
:102CE000013B934210D32B7FA88A0734E408B3B981
:102CF000844294BF00200120D9E7AB8ADB00083B67
:102D0000DB0873700824E5E7F319009321460023DC
:102D10000822284608F078FE08343B46DEE7201AF1
:102D200018BF0120C3E70000F7B50D460446002197
:102D30001646284681220BF039FF2346082200213F
:102D4000284608F09FFF94F901206378002AB8BF55
:102D50007F238DF807309EB90DF107030722082164
:102D6000284608F08FFF0F27002602349DF8073011
:102D70009E4207EBC60105D30731C80803B0F0BD7A
:102D80000827F1E7A3190822284608F07BFF01363F
:102D9000ECE7000037B50446007F0D4610B1A38A6A
:102DA000072B15D800231946009508222046083520
:102DB00008F02AFE0123009530220821204608F061
:102DC00023FE237FA08A2BB906288CBF0020012078
:102DD00003B030BD073818BF0120F9E738B50C46FD
:102DE000002121600546C4F8031003463022204626
:102DF00008F048FF204605F108030122302108F0C1
:102E000041FF072038BD00002DE9F04390F81C80F9
:102E100085B006460D46B8F1000F06D0838AE02B38
:102E200003D9012005B0BDE8F083002319460D2227
:102E30000095304608F0E8FD0DF10F0300930322E2
:102E400000230D21304608F0DFFD9DF80F30042BE4
:102E5000E7D82B72013B032B03D8DFE803F02530C2
:102E60003B461024B8F1000F5FD105F198030093A1
:102E7000214643460722304608F0C6FD073495F840
:102E800098305C2BCDD82F4695F898207B1B934229
:102E900052D3337FB08A0734E408002B58D18442E0
:102EA00094BF00200120BDE705F1100300934022EC
:102EB00001231021304608F0A7FD5024D2E705F188
:102EC00010030093202201231021304608F09CFDBE
:102ED0003024C7E705F110030093082200231021D6
:102EE000304608F091FD1824BCE705F1100300936B
:102EF000082200231021304608F086FD2B7C802B11
:102F00008FD8002705F111092B7CFC009F4204F1AA
:102F10001804A7D209EB07030093082200232146D7
:102F2000304608F071FD0137EEE7B38AC4EBC30306
:102F3000DB0885F89830A2E707F199030093214652
:102F400000230822304608F05FFD083401379BE774
:102F5000201A18BF012065E7F7B50C4613780968F9
:102F60008DF8063015460DF106030322064608F0DB
:102F700089FE2168033121602B78013B032B0CD89B
:102F8000DFE803F0020D161F05F10803402230466A
:102F900008F078FE23684033236003B0F0BD05F1EC
:102FA00008032022304608F06DFE23682033F3E743
:102FB00005F108030822304608F064FE2368083350
:102FC000EAE72B7A802B28BF80238DF80730082270
:102FD0000DF10703304608F055FE236808332360DF
:102FE000002709359DF807309F42D6D2EB1921689A
:102FF0000822304608F046FE236808332360013774
:10300000F0E7000073B50C46137809688DF80730B7
:1030100015460DF107030222064608F033FE21682B
:10302000023121602B78012B03D0022B0BD002B090
:1030300070BD05F108034022304608F023FE2368E6
:1030400040332360F3E705F108032022304608F0FF
:1030500019FE23682033F4E773B50D4604460021BA
:103060001646284640F273120BF0A0FD05232246B7
:1030700001A928460193FFF76FFF019B04F190021D
:10308000053301A928460193FFF766FF019B04F56C
:103090009072063301A928460193FFF7B3FF019B05
:1030A00004F59872063301A928460193FFF7AAFF99
:1030B00094F840315C2B28BF5C238DF803304EB967
:1030C0000DF1030301990722284608F0DBFD019B5F
:1030D00007330193002604F241149DF8033001994F
:1030E0009E4203D30731C80802B070BDA31908225D
:1030F000284608F0C7FD019B083301930136ECE731
:1031000000487047681802080121884238BF084605
:103110000BF02AB8FFF7F8BF08B10BF029B87047D9
:10312000FFF7FABF10B4026854681A4623465DF8E8
:10313000044B18470020704701207047002070475B
:103140000020704700207047704700000020704743
:1031500000207047704700007047000037B50546F3
:103160000C468322011D01A800F062F9611EC9B25C
:1031700002299EBF05EBC1010023C1E9073301A865
:1031800000F072F903B030BD2DE9F7431E461B88ED
:103190005B070546884620D4011D422201A800F0A5
:1031A00047F92C4605F118094C4513D0E3696BB17A
:1031B0002B6828465B6C98473388276AC1B243F076
:1031C0000403E0694246B8470834EDE7236A002B60
:1031D000EED1F9E701A800F047F9012003B0BDE8FE
:1031E000F08300007FB56D4685E806000446011DAA
:1031F000712203A81E4600F01BF921460022C8696F
:10320000D3B288B9086A78B995E8030004EBC20222
:103210001C32013382E803000124337003A800F05C
:1032200023F9204604B070BD0132032A01F10801E0
:10323000E5D10024F2E700002DE9F04F2DED028BDF
:103240008BB004468B465322011D01A8BDF858805F
:103250009FED258B00F0ECF8254604F118090027B6
:1032600008F0040AA94536D0EB690BB92B6A63B1A3
:10327000BAF1000F0BD1236820465B6C9847434698
:10328000C1B25A46D5E90706B0470835EAE7002F2C
:10329000FBD18DED028BADF810705B4605AA0BF1EA
:1032A000080C18685968174603C7083363453A463F
:1032B000F7D1186838609B88BB8004F0D7FC0423E2
:1032C000ADF810302368CDE902019B6C02A92046BD
:1032D00098470127D9E701A800F0C6F801200BB0F4
:1032E000BDEC028BBDE8F08F000000000000000084
:1032F00030B503680968DD0FB5EBD17F23F060447A
:1033000021F060424FEAD1700BD0002BB8BFA40C63
:103310000029B8BF920C944202D034BF0120002093
:1033200030BD944205D1C1F38070C3F380738342F2
:10333000F6D194422CBF00200120F1E7082817D9CC
:103340000C280CD910280CD914280CD918280CD901
:1033500020280CD930288CBF0F200E207047092060
:1033600070470A2070470B2070470C2070470D20D3
:1033700070470000082817D909280CD00A280CD05B
:103380000B280CD00C280CD00D280CD00E2814BF04
:103390004020302070470C207047102070471420C8
:1033A0007047182070472020704700004368184776
:1033B0008368184710B5024C8260C0E9004110BD17
:1033C00000190208007B00F0010070477047000000
:1033D0008160828070470000826838B504465AB127
:1033E000037B13F0010507D143F0010303739047FA
:1033F000237B65F30003237338BD000010B5044B35
:103400001B680446986A03681B699847204610BDEC
:103410000825002010B5054B1B680446986A036810
:1034200000211B699847204610BD00BF08250020D9
:10343000F8B50C4B01601E680446B06A03681B6C4B
:1034400017469847054610B1F36AA3F84270206802
:1034500003689B6898471DB1F36A0022A3F84220D5
:103460002046F8BD0825002010B504460068036812
:10347000DB689847204610BDC181B1FA81F0400950
:1034800070470000C08970477047000000207047F7
:103490007047000070470000002070470020704710
:1034A000704700004FF4B450704700000020704790
:1034B00000207047002070470020704700207047B0
:1034C000007B70477047000007B503688DF8071050
:1034D000DB6801220DF10701984703B05DF804FB9A
:1034E00008B5036801225B6A98470028D4BF002012
:1034F000012008BD07B503680DF10701DB69984796
:1035000020B19DF8070003B05DF804FB4FF0FF30D9
:10351000F9E7000013B5044608460191FDF7E6FD02
:1035200023680199DB680246204602B0BDE81040DE
:103530001847000004F09ABB10B444682CB9036823
:103540005DF8044BD3F88030184700205DF8044B39
:103550007047000082681AB90368D3F890301847A2
:103560000020704782681AB90368D3F8943018476E
:103570000020704730B4456825B90468E46FA4465C
:1035800030BC604730BC704700231A46FFF7F2BFDB
:1035900010B484680CB19C4206D103685DF8044BFA
:1035A000D3F8843092B2184700205DF8044B70477E
:1035B0000023FFF7EDBF0000013901298CBF002077
:1035C000012070470020704700207047002070479E
:1035D0007047000000230B70704700007047000028
:1035E000704700000020704700207047002070479F
:1035F000704700004368C26893423CBF8268D15460
:10360000436801334360012070470000F8B5054668
:103610000C468F180026BC4207D02B6814F8011BFB
:103620009B68284698470644F5E73046F8BD0000F9
:10363000002070470020704700207047002070472E
:1036400038B590F89C308B4204460D460CD080F87B
:103650009C1004F009FB2368C4F8A0005B682046B6
:10366000984708B984F84D5038BD00007FB50D4625
:103670001446194600267AB1531E0B4A6846CDE916
:103680000026089ACDE9025300F08EF80198844292
:1036900004D92E5404B070BD1346EEE7002CF9D0C7
:1036A0002C4404F8016CF5E72419020808B410B59D
:1036B00085B007AC54F8043B00940394FFF7D6FFA1
:1036C00005B0BDE8104001B07047000070B5044679
:1036D00002F036FB5E224FF4000102F01DFB0D4E9E
:1036E0000D4B1D6833783BB9E86A04222146483007
:1036F00004F0BEFA01233370EB6A2A2283F84620D5
:10370000EB6A93F89C301BB90448214604F082FA16
:1037100070BD00BF9E350020082500200819020852
:1037200007B503680DF10701DB69984720B19DF8E3
:10373000070003B05DF804FB4FF0FF30F9E700002D
:10374000F8B506460F4614460025AC420AD0336849
:1037500030469B699847431C01D12846F8BD7855EF
:103760000135F2E72046F9E70EB403B503AA036872
:1037700052F8041B5B680192984702B05DF804EBB5
:1037800003B0704700F010B813B504460846019125
:10379000FDF7ACFC23680199DB680246204602B0C5
:1037A000BDE81040184700002DE9F04F2DED028BC9
:1037B00006468DB0904691F80090B9F1000F00F0E8
:1037C000DE82B9F1250F08D04B1C039333684946BC
:1037D0009B68304698470399EDE791F801908B1C60
:1037E000B9F1250F0393F1D00025AA462C461F2CD2
:1037F0003BD8B9F12B0F2DD01CD8B9F1200F2BD00D
:10380000B9F1230F2ED0A9F13003DBB2092B36D842
:1038100060064BBF05EB85050AEB8A0A03EB4505FD
:1038200003EB4A0A4EBF05F0FF050AF0FF0A44F019
:10383000200407E0B9F12D0F11D0B9F1300FE2D11A
:1038400044F00104039B13F8019B0393B9F1000FAB
:10385000CDD126E044F0020444F00404F2E744F041
:103860000804EFE744F01004ECE77F2CCBD92306E3
:1038700017D5B9F16C0F14D144F48074E2E7B9F1B3
:103880002E0F05D1620600F17A8244F04004D9E798
:10389000B9F16C0F02D144F08004D3E7B9F1680F9D
:1038A000D0D0A9F14503022B61D809F1200944F0D9
:1038B00010045FFA89F908F1070828F00708F8E80A
:1038C0000201FDF73BF914F0400F08BF062524F074
:1038D000C004B9F1650F08EE100AA4B250D144F04B
:1038E000400427060DD59FED977AF0EEC87AF4EEE6
:1038F000C77AF1EE10FAC2BF4FF63F73234043F090
:10390000400414F0800346D03B2DA94628BF4FF059
:103910003B0909F101095FFA89F9072717220021FC
:1039200006A802930BF042F94A46394606A8B0EEC3
:10393000480A04F031FB9DF81830019303F00902A6
:10394000012A029B83462FD0A0072FD414F0040F26
:103950000CBF00222022019911F00C0758D0002A38
:1039600040F0AB82BAF1030F50D8174637E0A9F107
:103970006503022B00F25B8124F01004A4B29AE7E5
:10398000B9F1660F02D144F08004AAE7002DA8D057
:10399000013DEDB2A5E70A2D83BF0A2599462F46C2
:1039A0002F4698BF9946B9E72D22D4E72B22D2E7BC
:1039B0000427AAEB07072107FFB20AD43368029253
:1039C0009B6820213046013F984717F0FF07029A75
:1039D000F4D122B1336811469B6830469847019B69
:1039E000594D13F0080F594B08BF1D46013D04F017
:1039F000100415F8011F002900F0B5800CB1203922
:103A0000C9B2336830469B689847F2E70327D0E78E
:103A1000CDF808B0002B36D0019BD944DB065FFA05
:103A200089F907D59DF81930312B04BF09F1FF3909
:103A30005FFA89F94FFA89F3002B44DDB9F1080FD9
:103A400028BF4FF0080914F0800304931ABF2BEA33
:103A5000EB730133052302B101330DB1691C0B4433
:103A60009A45C4BFAAEB0303DFB214F0090F2FD1AC
:103A700077B3336805929B6820213046013F984711
:103A8000FFB2059AF4E76006DDD45D4504DB1BF167
:103A9000040FA8BF44F080046B1C06A90B4435B189
:103AA00013F80119302902D1013DEDB2F7E72106E3
:103AB000C9D505F101095D455FFA89F906DDA5EB78
:103AC0000B05EDB2BFE74FF00109BCE70025BAE7EF
:103AD00022B1336811469B6830469847220708D4C4
:103AE0003FB1336830219B683046013F9847FFB2B1
:103AF000F6E7049B002B47D02BEAEB74ABEB040AF0
:103B000006AB9A44ABEB09096D42A34517DBA1450F
:103B100015DA9AF80110013CA54219DC002900F0E1
:103B2000D281336830469B689847631C04D1336860
:103B30002E219B68304698470AF1010AE5E73021BB
:103B4000E9E700BF7F96184B541902085019020884
:103B5000A34507D19DF81930352B0FD802D1019B11
:103B6000DD060BD559B9002F3FF435AE336820215F
:103B70009B683046013F9847FFB2F4E73121336834
:103B80009B6830469847EEE79DF8191031291EBF13
:103B9000019B03F0EF030193336830469B6898471D
:103BA000E5B9336814F0100F14BF452165219B68F7
:103BB00030469847BBF1000F29DACBF1000302939E
:103BC0002D21336830469B6898473021029B092B92
:103BD00023DD01310A3BC9B20293F7E733682E2196
:103BE0009B68304698470235EDB24FF002094B46CC
:103BF0000CAA1A44336812F8181C9B6809F10109D1
:103C00005FFA89F930469847A945F0D1C9E702D152
:103C1000019BDC06D1D42B21D3E7336830469B6867
:103C200098470299336830319B68C9B2A9E7B9F166
:103C3000630F37D0B9F1730F4FD0B9F1640F63D16F
:103C400024F0900714F4807FBFB20DF118097BD0E7
:103C500008F1070222F007029046516858F8080B55
:103C6000002904DA404261EB410147F080070A2352
:103C70004A4600F07BF9A0EB0900C4B27B0640F194
:103C80009F8027F00109AC421FFA89F980F0D280A9
:103C900007F01403102B03D127F011071FFA87F93F
:103CA000AB468FE058F8043B8DF8183001250DF134
:103CB0001809200701D4AA451CD84D445746A945E8
:103CC0003FF451AF336819F8011B9B6830469847A1
:103CD000002FF4D0013FFFB2F1E758F8049B14F035
:103CE000400F14BF29464FF0FF3148460BF034FC1B
:103CF0000546DEE7336820219B6830460AF1FF3A2B
:103D000098475FFA8AFAD6E7B9F1690F98D0B9F106
:103D1000750F27D124F01004A7B20A2317F4807F6F
:103D2000DBB20DF1180944D008F1070828F00708A4
:103D3000F8E802014A4600F019F9A0EB090027F063
:103D40008007C4B2BFB299E758F8040B0028B8BF87
:103D500040424FF00A024946B8BF47F0800700F0E2
:103D6000B7F888E724F00607B9F1700FBFB214D096
:103D70000AD8B9F1580F13D0B9F16F0F17D00DB0A1
:103D8000BDEC028BBDE8F08FB9F1780FF7D1F906E1
:103D900001D547F004071023C0E747F01007F6E706
:103DA000E20601D547F006074FF40473B6E708238F
:103DB000B4E758F8040B1A46494600F089F8BCE706
:103DC000A346B94619F0100F41D00CAB234413F8A9
:103DD000193C302B30D129F016091FFA89F919F056
:103DE000080744D119F0010F35D0DA4545D904EB65
:103DF0000A05A5EB0B05EDB2336819F0100F9B68AF
:103E00003FD030213046984719F0040F08D033686E
:103E100019F0020F9B6814BF58217821304698474B
:103E20003368AC429B6839D230213046013D984717
:103E3000EDB2F5E7A346C5E719F0040F02D10BF187
:103E4000010B01E00BF1020B5FFA8BFBC7E719F0E6
:103E5000860FC4D0F3E73368DA459B680FD9202179
:103E600030460BF1010B98475FFA8BFBF3E7DA451D
:103E700005D9AAEB0B07FFB2BEE72546BCE7002732
:103E8000BAE719F0860FCBD019F0020F14BF2B211F
:103E9000202119F0800F18BF2D21BFE7651E06AB4A
:103EA00053FA85F5336815F801199B68013CE4B2B3
:103EB00030469847002CF5D155E6BAF1040F3FF68D
:103EC00077AD002786E5A3457FF44DAE42E600BFFF
:103ED000082A30B505D10346C008FCD130330B7039
:103EE0000DE0102A0DD100F00F0202F13003392B42
:103EF00088BF02F13703000901F8013BF3D10846FE
:103F000030BD03460022DCB223F00103023342F14C
:103F10000002580840EAC270C31842EB5202180966
:103F200040EA0270C01842EB1212030A43EA02632D
:103F3000181842EB1222030C43EA02431B1842EB0F
:103F40001242D31842F100001B0943EA0073C3EB8D
:103F50004315C3EB85053034020904EB450453EAED
:103F6000101001F8014BCED1C9E70000082B30B585
:103F70000AD10346C00840EA4170C90850EA01046A
:103F8000F7D13033137013E0102B13D100F00F046E
:103F900004F13003392B4FEA101088BF04F13703C6
:103FA00040EA0170090902F8013B50EA0103EDD132
:103FB000104630BD20F00104023441F100036108D5
:103FC00041EAC3710C1943EB5303210941EA037120
:103FD0000C1943EB1313210A41EA03610C1943EB5B
:103FE0001323210C41EA0341091943EB13435918E8
:103FF00043F10003C5B2080940EA0370C0EB401466
:10400000C0EB84043035190905EB440550EA13135D
:1040100002F8015BCED1CBE770EE600ADFED057AE6
:10402000F0EEE00AF4EEE70AF1EE10FA4CBF0120E0
:104030000020704700000034884203DB90420146B4
:10404000A8BF114608467047094A136849F269003B
:1040500099B21B0C00FB01331360064B186844F245
:10406000506182B2000C01FB0200186080B2704700
:1040700008230020042300207047000038B505689D
:1040800004462DB1284603F019FE2846FFF744F8F0
:10409000204638BD13460246014801F08DBC00BFE2
:1040A000EC35002013B50422054B0193044601466C
:1040B0000DEB0200FFF7EEFF024B1C8002B010BDBB
:1040C000FFFF3F00E035002007B5502304228DF8A4
:1040D0000430412300210DEB02008DF8053006234A
:1040E0008DF806308DF80710FFF7D4FF0420FFF796
:1040F000D9FF03B05DF804FB00EB0212907B20B9FE
:104100001BB19289120758BF3F209840084470475E
:10411000430608D4000A08D0054B1B88184214BF78
:10412000012000207047002070470120704700BF29
:10413000E435002010B50B4B1A880B4B01301B687F
:1041400080B2142404FB0033824207D9DC898C42FC
:1041500003F1140304D0013080B2F5E7002010BD54
:104160000120FCE7F0350020F435002082898368C7
:10417000D20648BF1B6818467047000082898368D2
:10418000D20648BF1B6818467047000007B50423D5
:1041900000220DEB03010B48019201F0D5FB9DF8C5
:1041A0000430502B07D19DF80530412B03D19DF8E9
:1041B0000630062B01D0FFF787FF012003B05DF822
:1041C00004FB00BFEC35002082894368920705D5C7
:1041D0001B68181E18BF01200B6070470120FBE709
:1041E00037B58B891446DA070D4605D523684A682A
:1041F00013442360012012E09B07FBD50A4B1B6888
:10420000142201A902FB0030FFF7DEFF48B101993B
:1042100022686B680A44D3581BB15B1A236003B051
:1042200030BD0020FBE700BFF43500202DE9F04F42
:104230008BB01F469DF85480069114235343059379
:1042400008F10603DBB2054616464FF0000B079354
:104250005FFA8BFA07EB0A1999F80F40002C4CD043
:10426000062C28D1B8F10B0F21D84846FFF77EFF66
:104270000446C8B1169B099309AA49463046FFF780
:10428000AFFF88B11499434652463846FFF734FFD2
:10429000099B0293079B0699CDE90003324623460A
:1042A0002846FFF7C3FF18B90BF1010BD0E7002038
:1042B0000BB0BDE8F08F1499434652463846FFF7DD
:1042C0001BFFB0EB953FEFD1C5F30423A342EBD125
:1042D0000B4C059B206809A91844FFF775FF0028BF
:1042E000E2D0D9F80430099A1344169A1344069A76
:1042F00013602068059B1844DAE72046D8E700BF22
:10430000F43500202DE9F04F1F4B5FFA80F8B3F829
:1043100000A0C0F3403348EA03281C4B1E680F4638
:1043200087B00546C0F3042B00211FFA81F9CA4566
:1043300027D9F3894345344620D1337C062B0FD14E
:104340003046FFF71BFFC8B10023CDE901330093CE
:104350004A46034639462846FFF768FF044609E007
:104360009B450BD105A93046FFF72EFF0028F5D05D
:10437000059B3B60204607B0BDE8F08F0131143645
:10438000D3E70024F6E700BFF0350020F435002025
:104390002DE9F04F98468DB0142353430693484BB4
:1043A0009DF85890DDF868B004461868069B0E46E4
:1043B00018440AA91746FFF707FF00287DD00023FD
:1043C000079309F10603DBB209939DF81CA006EBE5
:1043D0000A15EB7B002B70D0062B3BD12846FFF74C
:1043E000C5FE0890002831D0B9F10B0F65D8179B96
:1043F0000B930BAA29463846FFF7F2FE30B39BF821
:104400000030012B59D85A1C0BEB83038BF800208A
:1044100041465D6052464B463046FFF76DFE1B9AA3
:104420000899CDE904B2199A0392189A02920B9A4C
:104430000192099A009203463A462046FFF7A8FFE8
:1044400000BB9BF80030013B8BF80030079B013329
:104450000793BAE7179A686810440A9A1044A04272
:1044600013D14B46524641463046FFF745FE189B56
:104470001B9A1860199B1D6000231370104B18685D
:10448000069B18440DB0BDE8F08F052BDED1031D4F
:104490009C4203D000F108039C42D7D11B9B201AF9
:1044A0008008187052464B4641463046FFF724FEBE
:1044B000189B1860199B1D60E0E70020E2E700BF31
:1044C000F43500202DE9F04F8BB00025DFF8A4A0D3
:1044D000079306460F4690461560254B1B881FFA2A
:1044E00085FB5B4541D9DAF80000142303FB0B047C
:1044F00009A9204694F81090FFF766FE98B3B9F129
:10450000060F17D12046FFF739FE014658B3149B1A
:104510000593079B0297CDE903830023CDE9003380
:104520005A463046FFF734FF0446E0B120460BB050
:10453000BDE8F08F0998B04204D1149A00233B6083
:104540001370F3E7B9F1050F0DD1031D9E4203D09F
:1045500000F108039E4206D1149B301A800818709F
:1045600000233B60E2E70135B7E70024DEE700BF48
:10457000F0350020F43500202DE9F04798460D88ED
:10458000234B0446C5F30809186809EB890588B070
:1045900000EB850507A92846119E95F810A017463F
:1045A000FFF712FE20B90025284608B0BDE8F087C5
:1045B0000021BAF1060FC8F8001013D12846FFF702
:1045C000DDFD0028EFD0109B0091CDE90383CDE9FC
:1045D00001170B46059601464A462046FFF7D8FECE
:1045E0000546E1E70798A04202D139603170DBE768
:1045F000BAF1050FD7D1031D9C4203D000F1080387
:104600009C42D0D1241AA408002334703B60CBE72D
:10461000F43500200138C0B204289ABF014B185C61
:10462000002070477C1902082DE9F04F2DED028B18
:1046300083B000240093931DDBB208EE103A0546C8
:104640000E461746A246A0464FF0010BE0B201010C
:1046500005EB001090F80F90B9F1000F5AD0837B52
:104660003F2B02D92E4803F0D5FA17B1002B08BF13
:104670003F23C3F1200EA3F1200C2AFA03F208FA1B
:104680000EFE28FA0CFC42EA0E0242EA0C0212F07C
:10469000010FC3F1200CA3F12002E3D10BFA02F2C7
:1046A0002BFA0CFC42EA0C020BFA03F3B9F1060FE9
:1046B00043EA0A0A42EA080813D10B2FD2D8FFF7BF
:1046C00055FD814658B16858FCF710FD009B184411
:1046D000C3B218EE102A31464846FFF7A5FF013451
:1046E000B4E74846FFF796FF01900028BAD0685813
:1046F000FCF7FCFC009B1844C0B2B9F1050F04BFE5
:104700000230C0B21028019BACD83088043003447A
:104710003380E4E703B0BDEC028BBDE8F08F00BF4F
:10472000581902082DE9F04F85B00423DFF898905E
:10473000ADF80E3000244FF0140A214B1B881FFAED
:1047400084F8434539D9D9F800300AFB08F15D18DF
:104750002F7CB5F80EB0062F23D1B8F1000F02D18F
:10476000184803F057FA28460193FFF707FD06465D
:10477000A8B1019B5858FCF7B9FC0022C3B20DF157
:104780000E013046FFF750FF59464046FFF7D2FC76
:104790000028E5D1062F02D0AB899B07E0D4013475
:1047A000CBE73846FFF736FF0028D9D0BDF80E30EA
:1047B00004331844ADF80E00E6E705B0BDE8F08F0D
:1047C000F035002058190208F4350020437803F032
:1047D0001F021F2A0FD00278C3F3401342EA0323BB
:1047E00040F2FF12934206D000680138C31C94BF08
:1047F0000020012070470120704700002DE9F3419F
:10480000224FDFF8908006460D4604247B88A342A1
:1048100037D904230DEB03012246384601F094F802
:104820009DF80510737881EA0302D20618D196F834
:1048300000C09DF80400C3F34013C1F340124CEADA
:10484000032340EA022293420AD13268019B53407B
:1048500013EA080F04D12C80012002B0BDE8F081DA
:1048600001A8FFF7B3FF20B1094B2C801C8000206A
:10487000F3E701F01F00FFF7CDFE031D1C44A4B2B7
:10488000C4E74FF6FF732B80F1E700BFEC35002043
:10489000E035002000C0FFFF70B50C4620461146F1
:1048A00015461E460AF058FE831CAB420AD85F220A
:1048B000225422180330A84206F1580656709CBFB5
:1048C0000022E25470BD00002DE9F74FDDE90D54E0
:1048D00007468A46164609689DF830809B46224660
:1048E0009DF83C30009328460AF022FE4FF0000964
:1048F0009BF800105FFA89F29142019212D9214689
:1049000028460AF029FEC0B28442019A07D90BEB6F
:1049100082025168221A096828440AF009FE09F146
:104920000109E5E7E6B1214628460AF015FEC3B2C3
:104930009C4204D93168E21AE8180AF0F9FD009B9C
:1049400013B9B8F1000F13D0F37B052B10D14346F8
:1049500022462946384603B0BDE8F04FFFF79CBF1A
:10496000009B13B9B8F1000F02D09AF81030ECE7B1
:1049700003B0BDE8F08F0000F0B58BB007AC1F4668
:104980000023C4E9013307930DF11303CDE900437C
:10499000154606AB05AA0646FFF7EEFD014610B91F
:1049A00028700BB0F0BD9DF84030069A0195CDE916
:1049B00002739DF81330009330462346FFF784FFBF
:1049C000EFE700002DE9F04F984689B014234B43E0
:1049D000DFF828A1039204460E4604934FF0000925
:1049E0005FFA89F52B0108EB0515059395F80FB0D3
:1049F000BBF1000F7FD0BBF1060F58F803702AD12E
:104A00003846FCF773FB3946024620460AF05AFD49
:104A1000002869D12846FFF7A9FB0746002863D084
:104A2000039B079307AA29463046FFF7D9FB0028C6
:104A30005AD0059B58F80300FCF758FB129B0093D3
:104A4000079A3B4631462044FFF7BCFF00284BD075
:104A500009B0BDE8F08F394620460AF019FD88B943
:104A6000DAF80000049B07A91844FFF7ADFB002803
:104A70003AD0129B83F800B06868079B1844039BE8
:104A80001844E5E7BBF1050F2ED1102138460AF096
:104A900063FD5FFA80FB5A46394620460AF034FD32
:104AA00010BB14F90B305F2B1ED10BF1010B14F866
:104AB0000B30583B022B17D8DAF80000049B07A9EB
:104AC0001844FFF781FB78B16868079B129A184475
:104AD000039B18440423137014F90B30592B06D090
:104AE0005A2B06D0582BB3D009F1010978E70430CE
:104AF000AEE70830ACE75846AAE700BFF43500201F
:104B00002DE9F04F8BB0DFF8C8B00291044617468C
:104B100000252E4B1B881FFA85FA534552D91422C3
:104B200053465343DBF8002002EB0309D35899F8AE
:104B30001080B8F1060F33D11021184603930AF004
:104B40000BFD039B5FFA80F84246194620460AF0A7
:104B5000DBFC0646002833D14846FFF70FFB03462F
:104B600070B3029A009204EB080032465146FFF7F8
:104B700029FF804620B37FB10DF11303009306AAED
:104B800007AB05A9CDE9076605960996FFF79AFCDC
:104B9000069B0BB19B893B8040460BB0BDE8F08F74
:104BA000194620460AF074FC50B9029B07A983F805
:104BB00000804846FFF708FB20B1DDF81C80EBE7DA
:104BC0000135A6E74FF00008E6E700BFF03500200A
:104BD000F4350020F0B5304D87B040F2A5120290B8
:104BE0008DF80C1006460C4601A8291DFEF720FC86
:104BF000052204A9286803F0A7F9074601A8FEF7D3
:104C000033FC052F06D1049BB34203D19DF8143029
:104C1000A3423ED0214E224F4FF4B072314601A83C
:104C2000FEF706FC286803F0B3F8042821D92868A9
:104C3000052202A903F022F9431F5C425C4101A84E
:104C4000FEF712FC2CBB3C68E36A93F89C3093B9E6
:104C5000A06A036801211B699847A06A03684FF4A2
:104C6000FA719B689847A06A036800211B699847FE
:104C7000D2E70024E3E7A06A03681B6C984700288A
:104C8000E6D001F05DF840F2FA424FF4801101F0F5
:104C900043F807B0F0BD00BFBC350020C035002090
:104CA000082500202DE9F341154E164FC92406F1C1
:104CB0000408013CA4B2FCB140F24B12414601A8E9
:104CC000FEF7B6FB306803F049F8054601A8FEF789
:104CD000CBFB042D10D93D68A86A03680A211B6923
:104CE0009847A86A03680A215B689847A86A03681E
:104CF00000211B699847DCE702B0BDE8F08100BFE6
:104D0000BC3500200825002000B58BB00023CDE97C
:104D10000733049309930DF10D03009305AA07AB24
:104D200004A9FFF7CFFB10B3059B23B3DB7BC2893C
:104D30008DF8182003F01F03C2F300221B0243EA80
:104D40004233049A43EA82339DF818200DF10E0194
:104D5000134306A80693FFF751FD40B19DF81930A3
:104D600003F01F03052B03D09DF80D3003B1002085
:104D70000BB05DF804FB037CD9E70000F0B5144FDD
:104D80003B8889B006460D46FBB10DF10B030024AC
:104D9000009304AA05AB03A9CDE905440394079445
:104DA000FFF790FB88B10B4B38881B68A2B290428A
:104DB0000BD91A46013411688E4203F10C03F5D168
:104DC000137A2B70012009B0F0BD0020FBE700BF73
:104DD000E8350020DC35002013B50DF1070104464D
:104DE000FFF7CCFF10B92046FFF78EFF02B010BDD1
:104DF0000138032816D8DFE800F002080E13FDEE94
:104E0000C07A17EE903A0B707047BDEEC00A10EEF4
:104E1000103A0B807047BDEEC00A81ED000A704762
:104E200081ED000A7047000030B5224B1A7885B03A
:104E300072B901221A70204B204A1B680292986AAC
:104E40001F4A0368039204AA12E906009B6A984766
:104E50001C4D04246B88A34229D9042322466946A9
:104E6000284600F071FD6846FFF7B0FC18B1164BFC
:104E70001C8005B030BD009801A9FFF743FA60B16E
:104E80009DF8010000F01F00FFF7C4FB221D034640
:104E9000019992B2284600F057FD9DF8010000F0FC
:104EA0001F00FFF7B7FB04300444A4B2D2E7002090
:104EB000DFE700BFEA350020082500209F350020ED
:104EC00059570108EC350020E035002037B503685C
:104ED00003F0004303600A4B1B880C4613B9002003
:104EE00003B030BD074D01A92868FFF76DF9002810
:104EF000F5D014B12B681B7C23700198F0E700BF3C
:104F0000F0350020F43500202DE9F04F8FB09B469E
:104F10009DF870300B93142343439DF860901A9DC5
:104F20000A93074688460892002307939DF81CA021
:104F300008EB0A16F47B002C00F0BC80B089FFF768
:104F4000E7F8002800F0B380062C2FD13046FFF799
:104F50000DF90446002800F0AA80199B0D930DAAB4
:104F600031463846FFF73CF9002800F0A0804B4658
:104F7000524659464046FFF7BFF81D9A05920B9AD4
:104F800004921B9ACDE902520D9A019209F1060290
:104F9000D2B2034600922146089A3846FFF7B4FF82
:104FA000002800F084800FB0BDE8F08F089B1B78CC
:104FB0000993002B3CD02B8867F308032B805246C3
:104FC0004B4659464046FFF797F83B4B03EA4030C3
:104FD0002B6823F0FF4323F4FF0323F4FC4318431F
:104FE0001B9B286003B11C70344B18680A9B0DA9E9
:104FF0001844FFF7E9F8002859D00D9A7368134454
:10500000199A98180B9A002ACDD02D4A1278002AA6
:10501000C9D0F27B012AC6D1B2895207C3D5199AE9
:105020009B56002BBFD1EB7843F08003EB70BAE7BF
:105030004B46524659464046FFF75EF82B68C3F38D
:105040005133984233D1089A0123137095F90330F4
:10505000002B06DAEB78099A62F3C713EB7010465F
:10506000A1E7052C23D16B78C3F34302022A1ED893
:10507000013262F344036B701B9B13B11B9A042330
:1050800013700E4B18680A9B0DA91844FFF79CF883
:1050900068B170680D9C95F801B0199B2044CBF362
:1050A000430B18440BF1FF3B00EB8B007BE7079BA6
:1050B00001333AE7204676E700E0FF7FF435002031
:1050C0000C2300202DE9F04F8BB0DFF8EC90048822
:1050D000079200228DF82720B9F800201F46C4F35C
:1050E00008039A4205460E461C4662D9DFF8CC807A
:1050F0001BB2D8F8001003EB83039A0001EB830383
:105100001B7C052B18D14378C3F34301022915D822
:10511000013161F3440343700EB104233370D8F8B6
:10512000001068780A44C0F34300431E506800EB47
:1051300083000BB0BDE8F08F062B04D001340123AF
:10514000A4B28DF827304FF0140B4FF0000AB9F8D5
:105150000030A3422DD9D8F800200BFB04229089FF
:10516000FEF7D6FFB8B1117C062917D11046FFF71C
:1051700005F8014678B1079B0597CDE90363CDE9B2
:1051800001A5CDF800A000230DF127022046FFF76E
:10519000BBFE0028CDD10134A4B2D8E72B68C4F3FC
:1051A000080403F0004323432B6006B131705068BC
:1051B000BFE70020BDE700BFF0350020F435002038
:1051C00073B505460C461646334601220DF107011C
:1051D0002846FFF777FF28B19DF80730042BF3D856
:1051E00004B1237002B070BDF8B514460746002222
:1051F00020460E46FFF76AFE002540B1BD4206D0AC
:10520000002231462046FFF7DBFF0135F5E7F8BD08
:10521000013903290BD8DFE801F00204060800F089
:105220000DBB00F043BB00F061BB00F0DDBA9FEDA9
:10523000010A70470000C07F70B50E4B1E880E4BF0
:105240001B68002294B2A64209D91C460132256887
:10525000854203F10C03F5D194ED010A70BD8B89F1
:105260001B0649BF8B6891ED020AC01A90ED000A37
:10527000F4E700BFE8350020DC3500202DE9F041DF
:1052800005460F464FF000085FFA88F307EB03115D
:10529000CC7BDCB1042C0BD84E682E443046FFF793
:1052A000CBFF31462046FFF7A3FD08F10108EBE7ED
:1052B000052CFAD14C682C442046FFF7BDFF84ED45
:1052C000000A84ED010A84ED020AEEE7BDE8F081F0
:1052D00070B50E4B1E880E4B1B68002294B2A6427E
:1052E00009D91C4601322568854203F10C03F5D12A
:1052F00094ED010A70BD8B891B0649BF8B6891ED47
:10530000020AC01A90ED000AF4E700BFE835002059
:10531000DC3500202DE9F0418AB00023CDE90733C8
:10532000039309930DF10903009304AA07AB03A9A2
:105330000446FFF7C7F8054620B9002630460AB0F4
:10534000BDE8F081049B002B3AD0DB7BEA898DF825
:10535000142003F01F03C2F300221B0243EA42336E
:10536000039A43EA82339DF814200DF10A01134396
:1053700005A80593FFF742FA064658BB06A928463A
:10538000FEF722FF0028D9D09DF815700499DDF8AA
:10539000188007F01F07B9B19DF81C3093B1089A27
:1053A000012B556802D0099B5B681D442046FFF71E
:1053B00043FF4968414429443846FFF719FDBDE7DA
:1053C000037CC3E73546F1E729462046FFF780FF17
:1053D0004146F1E79DF815009DF8093000F01F02E5
:1053E000052A0FD0002BA8D100F01F00FFF712F9FB
:1053F000BDF80A200432034692B22146044800F068
:10540000A3FA9BE7002BEFD0A4EB8304ECE700BFEB
:10541000EC3500202DE9F04385B0FEF7B7FE134EC2
:10542000134F00254FF014083288ABB29A4219D9B5
:105430001C463B6808FB043494F81090B9F1040F43
:105440000ED803A92046FEF7BFFE48B1039801908D
:105450002146FFF73DFF019801464846FFF7C8FC8B
:105460000135E1E705B0BDE8F08300BFF03500206D
:10547000F43500202DE9F347DFF88C901F4940F602
:1054800078226846FDF7D4FFB9F800702FB11C4BA5
:105490001A881C4B1B889A4228D0194E194D052496
:1054A0004FF00008B9F800701FB132882B889A427B
:1054B0001CD0013C14F0FF0418D00022114601A8B2
:1054C0003788CDF80480FFF701FD4FF0000A1FFA7E
:1054D0008AF30AF1010A28B10022114601A8FFF758
:1054E0006FFEF4E7A9F800302F80DBE76846FDF790
:1054F000BBFF384602B0BDE8F08700BFA0350020F2
:10550000DA350020E6350020E2350020024A138813
:1055100001331380704700BFDA3500202DE9F041D8
:105520002DED028B90B00023CDE9083305930A934B
:105530000DF1110300930E4608AB06AA05A9044617
:10554000FEF7C0FF0546D8B10699F1B1CA7BEB89D9
:105550008DF81C3002F01F02C3F300201302059ADD
:105560009DF8117043EA403343EA82339DF81C20D2
:105570001A43C3F30423052B079200F0868037B14A
:1055800010B0BDEC028BBDE8F081027CDFE7012B9F
:1055900005D121B18B895B0701D5FFF7B7FF2746FE
:1055A00077E0BDF812204FF6FF739A420AD14C4BB8
:1055B00083F800804B4B4C491B68986903681B6853
:1055C0009847DDE79DF81D1001F01F01042925D93A
:1055D0009DF81D00BDF81220444900F01F00FFF7A0
:1055E00019F84988131808338B424AD20432104400
:1055F00080B2FEF757FD9DF81D0000F01F00FFF779
:1056000009F8BDF812100431024689B23846FEF797
:1056100041FDBDF81210042207A85EE02046FFF706
:10562000F7FD0699F0EE408A71B12046FFF704FEBF
:10563000B0EE408AF0EE400AB0EE680AFEF7ECFCED
:1056400038B1002EC4D19BE729462046FFF740FE23
:10565000EEE7002EBCD19DF81D3003F01F03032B95
:10566000B6D09FED230A38EEC88AF0EEE88A68EEDD
:10567000808AB0EEC88AB4EEE88AF1EE10FAA7D5B7
:105680007EE7174B01221A7094E7002F87D0A4EB16
:10569000870711234FF00108CDE902380BAB0193C6
:1056A0009DF81130009329462046069A08ABFFF773
:1056B0000BF90DF1120107A8FFF7A0F800283FF43D
:1056C00070AF9DF81D0000F01F00FEF7A3FFBDF8AE
:1056D00012100431024689B23846FEF7DBFC4FE770
:1056E000D8350020082500206C190208EC35002070
:1056F00017B7D1387FB5164D2E1D40F27F123146B7
:1057000001A8FDF795FE286802F028FB042812D9AD
:105710002868052202A902F033FC431F5C425C4169
:1057200001A8FDF7A1FE44B19DF80C1002980122DA
:10573000FFF7F4FEE1E70024F2E7064B1B68986AE6
:1057400003685B6B984708B1FFF794FE04B070BD27
:10575000BC35002008250020FFF7CCBF10B504465B
:10576000FDF7DAFC204610BD38B51148114D01F0A7
:1057700081FC114A11490E4809F0E6F92846002338
:1057800040F8043B01F076FC1420FDF7BDFC044614
:1057900010B19B2102F080FA0949074A05482C60A4
:1057A00009F0D2F9BDE838400648002100F0B6B84B
:1057B000A0350020BC350020A078002079400108E9
:1057C0007D400108EC350020D1ED007A90ED007AA3
:1057D000F4EE477AF1EE10FA04D0C0ED007A012120
:1057E000FFF7F8B97047000090ED000A704700001D
:1057F00091F9001090F900309FED097A01705B1A61
:1058000007EE903AF8EEE77AF0EEE77AF4EEC77A30
:10581000F1EE10FA4CBF01210021FFF7DBB900BF08
:105820000000003491F9002090F90010914203D05B
:1058300002700121FFF7CEB97047000090F90030E7
:1058400000EE103AB8EEC00A7047000038B50446C2
:105850000D46FFF7C1FA10B9B5F90030238038BD05
:10586000B1F90010B0F900309FED097A01805B1AA0
:1058700007EE903AF8EEE77AF0EEE77AF4EEC77AC0
:10588000F1EE10FA4CBF01210021FFF7A3B900BFD0
:1058900000000034B1F90020B0F90010914203D0AB
:1058A00002800121FFF796B970470000B0F900307F
:1058B00000EE103AB8EEC00A7047000038B5044652
:1058C0000D46FFF789FA08B92B68236038BD000040
:1058D0000B680360704700000A6801688A4203D0C1
:1058E00002600121FFF776B97047000090ED000AD1
:1058F000B8EEC00A7047000008B5064B1B6858692F
:1059000003685B68984720B9BDE80840024801F089
:10591000CDBB08BD082500208419020830B500233E
:10592000084A0170438014788C4204BF44889588EB
:1059300003F1030304BF64194480242B02F106021F
:10594000F1D130BDA41902082DE9F84F184EDFF847
:10595000649007468A461D4606F1480831783B7830
:10596000994204D1B488944209D8121B92B20636E7
:10597000B045F3D1B5FA85F04009BDE8F88F12FAC9
:1059800085F3A342D9F8003058697388C8BFA41AB8
:105990001A440368D4BFACB2A4B2D3F808B092B230
:1059A00023465146D8472D1BE4D0A2440022DEE70F
:1059B000A4190208082500202DE9F84F184EDFF839
:1059C0006490074692461D4606F1480832783B78B7
:1059D0009A4204D1B4888C4209D8091B89B2063690
:1059E000B045F3D1B5FA85F04009BDE8F88F11FA5A
:1059F00085F3A342D9F8003058697388C8BF641A88
:105A000019440368D4BFACB2A4B2D3F80CB0524668
:105A1000234689B2D8472D1BE4D0A2440021DEE7FB
:105A2000A41902080825002010B5044B0449186089
:105A30000446FFF723FC204610BD00BFF8350020C8
:105A4000401A020890F8233063B9012380F823300C
:105A5000054800684FF40073006C80224FF4E13178
:105A6000FDF788BD704700BF08250020002850DDE5
:105A70006F2846D01BDC132845D00EDC431E082BB4
:105A800011D8082B33D8DFE803F041053236323223
:105A9000323239004FF416607047392839D0642803
:105AA0003AD026283AD04FF47A7358437047B0F56D
:105AB000FA7F36D010DCB0F5807F34D006DC732856
:105AC00034D0E628EFD14FF461307047B0F5E67F6F
:105AD000E9D14FF4E120704740F2DC53984228D0DE
:105AE000B0F5FA6F27D040F29933984225D0B0F53F
:105AF000FA6FD8DD70474FF4965070474FF4165048
:105B000070470F4870474FF4964070474FF49660C7
:105B100070474FF4614070470A4870474FF4164091
:105B20007047094870474FF47A3070474FF4E130BE
:105B3000704706487047064870474FF46120D9E720
:105B4000FCB10100A086010020A1070060E316005F
:105B500080841E000068FFF789BF00000E4B70B5FF
:105B60001D68CBB2092B0C4612D8103355F82320F0
:105B700000EBC103116810464E6B9988B04750B9CD
:105B8000A8690649036822461B68BDE870401847AB
:105B900000231B68FFDE70BD08250020EC190208F9
:105BA0002DE9FF41FF23804603A921308DF80C30F9
:105BB000FFF738FE4046FFF745FF564B1B68019341
:105BC00008F1080401267327019A06F1100352F820
:105BD0002350E6717DB3B1B24046FFF7BFFF94F9A1
:105BE00006300133332B00F28C80DFE803F0241AF7
:105BF0001A1A2C3335353D478A338A528A8A245AF9
:105C00008A8A698A8A4C8A7D8A8A8A8A8A248A8AC6
:105C10008A8A8A8A8A8A8A8A8A8A1A8A8A8A8A8A54
:105C20008A242046FFF796FF4FF4807301468022B6
:105C30002846FDF79FFC0136042E04F10804C3D169
:105C400004B0BDE8F081092303A920460393FFF7C0
:105C50003FFEF0E73923F7E72046FFF77BFF1023ED
:105C600001464FF48072E3E703A920460397FFF74C
:105C70002FFE80231A464FF4E131D9E703A92046CD
:105C80000397FFF725FE2046FFF764FF80230146B8
:105C9000CDE7092303A9A01D8DF80C30FFF7A8FD5F
:105CA000C9E703A920460397FFF712FE2046FFF736
:105CB00051FF1E2301461A462846FDF75BFC0DE006
:105CC0002046FFF747FF802301461A462846FDF786
:105CD00051FC2B680121DB6C284698472B6800217A
:105CE000DB6B28469847A6E703A920460397FFF7F2
:105CF000E5FD2046FFF72EFF102301464FF400720A
:105D0000DAE72046FFF726FF01462846FDF73CFC70
:105D100091E700BF0825002010B5036802811943F0
:105D20004368016001334360044B1B68DC6AA16275
:105D3000D96A40688885DB6ADA8510BD08250020AD
:105D400000487047FC35002008B50449FBF7C4F94A
:105D50000028034818BF002008BD00BFA01A020891
:105D6000105502082DE9F0418846FFF7EDFF054682
:105D700008B9002409E08668701C08F0C7F90446D9
:105D80000028F6D026B9C8F800602046BDE8F081AA
:105D90004FF4A16008F0BAF9064618B9204608F099
:105DA000E7F9E6E70022114600F040F92B6933607D
:105DB0006A68F46113447360AB68B361304600F005
:105DC00045F90746304608F0D3F9002FE6D1AA6816
:105DD0002146384602F06CFAEB689842DED1AB6897
:105DE000C8F80030D1E7000008F0C2B9F0B50D46A0
:105DF000164689B020220021044608F0D7FE2A4624
:105E00007019824207D012F8011B34F811300133A7
:105E100024F81130F5E72146002321F802396A46BB
:105E200004F11E0031F8027F22F8023B81423B441C
:105E3000F8D10023B3420ED0E95C51B108AA02EBBD
:105E4000410131F8202C501C103221F8200C24F88C
:105E500012300133EEE709B0F0BD000010B5D0E913
:105E600000329342044603D25A1C0260187810BDD7
:105E700083683BB190F8292022B99847031E01DBC3
:105E8000D8B2F4E7012384F829300020EFE70000BE
:105E900010B503695A1E0446026123B9FFF7DEFFFD
:105EA0000723E0602361E0684308E36000F001003D
:105EB00010BD00002DE9F0410746164661B10125ED
:105EC00005FA01F80024454507D23846FFF7E0FF00
:105ED00000B12C446D00F6E70C463019BDE8F081A6
:105EE0002DE9F843002380460E468F1C01F120095E
:105EF0001D4640465C00FFF7CBFF4F4504440FD0E2
:105F000037F8023B5A19E31A08D52544B5F5907FB6
:105F100006D2103536F81500BDE8F8831546E8E7D7
:105F20006FF00200F8E700002DE9F04F0E46D3B005
:105F30000521904640F201120446FFF7BBFF012203
:105F4000052105462046FFF7B5FF04221146074606
:105F50002046FFF7AFFF13228246002102A808F077
:105F600025FEDFF8C4B04FF00009D1450BD0002268
:105F700003212046FFF79EFF1BF8013B02AA09F10F
:105F80000109D054F1E7132202A93046FFF72EFF92
:105F900005EB07094FF0000ACA4538D231462046C2
:105FA000FFF79EFF00280ADB112829D012282BD0EA
:105FB00010281ED1BAF1000F04D16FF0020053B0C7
:105FC000BDE8F08F02AB5344032213F8013C0221D9
:105FD00020460193FFF76EFF0AEB000BCB4502460C
:105FE000EBD8019B194602AB03EB0A0008F0DEFD7B
:105FF00004E002AB0AF1010B03F80A00DA46CBE732
:10600000032211460023E3E70B220721FAE72A4681
:1060100002A93046FFF7EAFE02AB40463A4659195C
:10602000FFF7E4FE0020CAE78055020810B5002300
:106030004FF0FF34C0E90133C0E90F1280F8293076
:1060400003610363C4624364436310BD2DE9F047F9
:106050009F4DA04EA04F0446E36A013340F0948068
:106060002046FFF715FF0022206302212046FFF79C
:1060700021FF0128E0627BD10023A4F84830A4F876
:106080004A30A4F84C30A4F84E30A4F85030A4F8AC
:106090005230A4F854301823A4F856309823A4F8AA
:1060A00058307023A4F85A3004F168024FF480731A
:1060B00022F8023B01339BB2B3F58C7FF8D104F197
:1060C0009802002322F8023B0133902BFAD14FF4BF
:1060D0008C72A4F8B82140F21912A4F8BA214FF436
:1060E0008D72A4F8BC2140F21B12A4F8BE214FF41B
:1060F0008E72A4F8C02140F21D12A4F8C2214FF400
:106100008F72A4F8C42140F21F12A4F8C62104F52E
:10611000E47222F8023B01339BB2B3F5807FF8D1E1
:1061200000232022A4F8B222A4F8A832A4F8AA32AC
:10613000A4F8AC32A4F8AE32A4F8B03204F532724E
:1061400022F8023B0133202BFAD1636B002B40F085
:106150008A8004F148012046FFF7C2FE94F82930F6
:10616000BBB9FF2859DCE3695A1CE261C0B240E0C8
:10617000022809D104F52A7204F148012046FFF7EC
:10618000D3FE002840F09E80E36A2BB1013B012B37
:10619000DBD96FF0020095E0D4F834A0BAF1000F1B
:1061A0001CD12046FFF75AFE81462046FFF756FED7
:1061B00009EB00292046FFF751FE80462046FFF7F5
:1061C0004DFE08EB002383F47F4383F0FF039945E2
:1061D000DFD109F101006063C4F810A0636B013BDB
:1061E0006363002B69D02046FFF738FEE3695A1C31
:1061F000E2611870E26B4AB1636C591C6164D0545F
:10620000D4E910329A4201D100236364A0690138B5
:10621000A06100287FF420AF54E0B0F5807F4CD01F
:106220006FF48073184435F81020315C2046FFF776
:1062300041FE04F52A7160632046FFF751FE0028F5
:1062400040DB264B37F81020195C2046FFF732FE62
:10625000E36B002B29D0226C904235D8636C181A5E
:1062600048BF8018A063E16BE369A26BF9B1581CC9
:10627000E0618A5C1A70E36B5BB1626CA16B501CCD
:106280006064595C9954D4E910329A4204BF0023E7
:106290006364A36B226C01339342A36301D1002397
:1062A000A363636B013B6363B0E74042DAE79A5C48
:1062B0001A70E3690133E361F3E7236B002B3FF4CA
:1062C000CFAE0120BDE8F0876FF00400FAE700BF11
:1062D000245502086055020894550208D05502085A
:1062E00010B4064B064A1B680649986903681C6887
:1062F000537E127EA4465DF8044B604708250020BB
:10630000F0010108F0550208002070470E20704788
:1063100000F5805090F8F000C0F340007047000096
:1063200000F588507047000000F5805090F9F800A3
:106330007047000000F58050C0F8F410012070474D
:106340002DE9F3470C68BDF8288014F00054074687
:106350000D4696469C4640F08F800E7B082E00F23C
:106360008B8000F58059D9F800610136C9F80061C9
:10637000302686F31188C66BD6F808A01AF0806F15
:1063800017D1B468240113D4B46814F080546FD1C9
:10639000D9F808510135C9F80851D9F80C51002D28
:1063A00068D1CDF80080FCF747FF84F311885CE0EA
:1063B00001242B6804F11802002B4FEA0212BABF25
:1063C000DB0043F004035B05B3502B6813F0804FF0
:1063D00023B218BF06EB031106EB03131EBFD1F85F
:1063E000802142F00202C1F880212A7BC3F8842177
:1063F00006EB0416AA68C6F88C216A68C6F88821DC
:10640000D3F8802142F00102C3F8802141F29001CB
:1064100007EB44120A4401EB44113944C2E900EC91
:1064200063012A46083105F10C0052F8044B41F88B
:10643000044B8242F9D13B4412880A8003F5805311
:1064400008F0030293F8AC1021F00B010A4383F823
:10645000AC20002383F31188CDF800807246634698
:1064600029463846FCF7E8FE012002B0BDE8F08777
:1064700002249EE7204698E74FF0FF30F5E7000042
:106480002DE9F04F90F83830032B40F098800E2A19
:1064900000F29580002900F09480302383F3118866
:1064A000C46BD4F8003243F00103C4F80032C46B6B
:1064B000D4F8003223F47C53C4F80032C46BD4F80F
:1064C000003243F46063C4F80032C36B3E4CC3F83F
:1064D0001442C46B0023C4F80432C46B6FF07845D7
:1064E000C4F80C5200F5805494F8F8509D4218BF3F
:1064F0000E25DAB9C36B05F1480143F83120C36BAF
:1065000003EBC1035A60C26B012303FA05F5C2F81D
:106510001C52C26BD2F8003223F00103C2F80032E1
:10652000002383F311880120BDE8F08F4FF00108AC
:1065300001F10409EF189A42D0F83CA008FA07FECE
:1065400036DD51F833B059F833C0BBF1000F02DB30
:10655000BCF1000F27DB4FEACB044FEACC0644F036
:1065600004041BF0804F07F1480718BF44F00204F1
:106570004AF83740C46BBCF1000FB8BF46F00406C0
:1065800004EBC7041CF0804F18BF46F0020666609B
:10659000C66BD6F81C424EEA0404C6F81C4201330E
:1065A0000E2BC7D1B5E74FEA4B544FEA4C56D8E70C
:1065B000DAF81C4224EA0E04CAF81C42EFE7002075
:1065C000B2E70846B0E700BFAAAAAA0A13B500F5C9
:1065D00080540191D4F8840001F0DAFB1F280BD914
:1065E0000199D4F88400202201F048FCA0F1200396
:1065F0005842584102B010BD0020FBE708B53023D7
:1066000083F3118800F58050D0F8840001F094FBEA
:10661000002383F3118808BD00220260828142605A
:106620008260704710B500220023C0E900230023D8
:10663000044603810C30FFF7EFFF204610BD000039
:106640002DE9F04300F580570D4697F8F03013F030
:10665000040FC3F3800108BF114661F3820387F87A
:10666000F03000EB451303F58553083389B01B79EF
:10667000D907DDE9108904464FEA45163BD5002AC3
:106680003BD0180739D404EB45156846FFF7CAFF1D
:1066900005F58453183303AA05F58555186859681C
:1066A0009446ACE803000833AB426246F6D1186862
:1066B000CCF800009B88ACF804300123ADF808301A
:1066C0002368CDE900899B6C694620469847A31949
:1066D00003F5855308331A7911070ED442F00802E6
:1066E0001A71D7F80C3104F589540133C7F80C310D
:1066F000C4E9028901E0002AE9D109B0BDE8F083CC
:106700002DE9F0479A4688B00746884691463023DF
:1067100083F3118807F580546846FFF783FFD4F8A8
:10672000840001F01BFB1F282BD9D4F88400202201
:10673000694601F025FC202823D103AD444605AB72
:106740002E4603CE9E4220606160354604F1080467
:10675000F6D130682060B388A380DDE90023C9E961
:106760000023BDF80830AAF80030002383F3118815
:1067700053464A464146384608B0BDE8F047FCF764
:1067800003BD002080F3118808B0BDE8F087000049
:106790002DE9F84F2B4B044640F8043B0F4600F020
:1067A00069FC1822002104F11C0008F0FFF92046C2
:1067B000254B40F8403BFFF72FFF04F15000FFF757
:1067C00031FF04F1700804F5835546461035304614
:1067D0002036FFF727FFAE42F9D104F580554FF47C
:1067E00080534FF00009C5E91D39C5F870800123B9
:1067F000C5F8846004F5885804F58556C5F87C9082
:1068000085F8803085F88830103608F110084FF090
:10681000000A4FF0000B46E908ABA6F11800FFF79D
:10682000FBFE203646F8289C4645F4D185F8F870E2
:1068300017B1064801F0EEF9054BE3632046BDE8C9
:10684000F88F00BFAC18020828560208005602084C
:106850000064004010B5044B197804464A1C1A70B5
:10686000FFF796FF204610BD0C3600202DE9F047BB
:10687000002950D0294B2A4FB7FBF1F599428CBF24
:106880000A231123581EB5FBF3FC03FB1C53C4B2AF
:106890002BB102280346F5D80020BDE8F0870CF1A3
:1068A000FF36B6F5806FF7D2C4EBC40E0EF10303CA
:1068B0004FEAE309C3F3C703A4EB030809F1010A94
:1068C0004FF47A755FFA88F009FB05555AFA88F893
:1068D000B5FBF8F5B5F5617FC1BF0EF1FF33C3F32A
:1068E000C703E01AC0B25C1C50FA84F40CFB04F439
:1068F000B7FBF4F4A142CFD1013BDBB20F2BCBD8D5
:106900000138C0B20728C7D80021107116809170D5
:10691000D3700120C1E70846BFE700BF3F420F0028
:1069200080DE800270B505460E464FF47A74EB6B3C
:106930005B6803F00103B34207D04FF47A7007F0AD
:1069400081F8013CF3D1204670BD0120FCE7000036
:10695000F0B5C26B936913F0700F1ED000230F4E79
:10696000936141F2A80500F5805400EB43122A44DC
:1069700011794F070ED589070CD5C16B56F82370D6
:106980008F60117941F004011171D4F814210132A2
:10699000C4F814210133032BE7D1F0BD14560208CB
:1069A00073B51D46C36B16469A68D207044609D5CF
:1069B0009A6801219960C2F34002CDE90065002187
:1069C000FFF73EFEE36B9A68D1050BD59A684FF44A
:1069D00080719960C2F34022CDE900650121204613
:1069E000FFF72EFEE36B9A68D2030BD59A684FF43B
:1069F00080319960C2F34042CDE900650221204612
:106A0000FFF71EFE04F58053D3F8F40038B1D3F835
:106A100030210132C3F8302103681B6998472046B2
:106A200002B0BDE87040FFF793BF0000F8B5044620
:106A3000C66B002940F08D8006F10C073868850789
:106A400000F090803868C00641BF04F58055D5F845
:106A500020010130C5F8200106EB011506EB0111FC
:106A6000D5F8B00110F0040FD5F8B0011ABFC00876
:106A700040F00040400D2064D5F8B0C11CF0020F7A
:106A80001CBF40F080402064D5F8B40100F00F0036
:106A900084F84C00D1F8B80184F84400D1F8B8016A
:106AA000000A84F84500D1F8B801000C84F84600CB
:106AB000D1F8B801000E84F84700D1F8BC0184F881
:106AC0004800D1F8BC01000A84F84900D1F8BC01A3
:106AD000000C84F84A00D1F8BC11090E84F84B1060
:106AE0003821396004F15C0004F1400104F14C05E7
:106AF00051F8046B40F8046BA942F9D10988018070
:106B0000C4E9142321460023A4F8583051F8503B1F
:106B100020469B6C984704F58053E8B1D3F81821C0
:106B20000132C3F8182193F8F020D3F8F40042F0B2
:106B3000040283F8F02038B1D3F830210132C3F8D1
:106B4000302103681B6998472046BDE8F840FFF7ED
:106B5000FFBE06F1100771E7D3F81C210132C3F81C
:106B60001C21E0E7F8BD000010B5044601F07EF8F6
:106B700002460B4652EA030102D0013A63F10003D8
:106B80000449086820B12146BDE81040FFF74EBF18
:106B900010BD00BF083600202DE9F041302181F3FF
:106BA0001188DFF85C8000F584511031002441F237
:106BB000A80E00F5805C00EB441575442E7977072C
:106BC00013D4F60611D5D1E9007697429E410CD236
:106BD000C66B58F82470B7602E7946F004062E7103
:106BE000DCF810510135CCF810510134032C01F1BF
:106BF0002001E0D1002383F31188BDE8F08100BFBC
:106C00001456020808B5302383F31188FFF7A0FE5D
:106C1000002383F3118808BD2DE9F041C36B0546BD
:106C2000986800F0E050B0F1E05F0F4623D000B369
:106C3000302383F3118805F584541834002641F27B
:106C4000A80805EB461343441B791A0706D50136FD
:106C5000032E04F12004F4D1012007E05B07F6D4F1
:106C600021463846FCF744FB0028F0D1002383F38B
:106C70001188BDE8F0810120FBE7000008B5302352
:106C800083F3118800F58050D0F8840001F066F895
:106C9000002383F3118843090CBF0120002008BDA5
:106CA000F8B51D46002313700F4606461446FFF73D
:106CB000E5FF80F00100387025B129463046FFF726
:106CC000ABFF2070F8BD00002DE9B8410C46154619
:106CD0001F46804600F0CAFF0B462178024609B9DC
:106CE000287850B14046FFF757FFFFF78BFF3B4630
:106CF0002A462146FFF7D4FF0120BDE8B8810000F5
:106D000070B5302686F31188174B1A6C42F000726A
:106D10001A641A6A42F000721A621A6A22F0007249
:106D20001A62002383F3118800F5805494F8F03040
:106D300013F0010516D1A9B186F3118803211320A0
:106D400005F082FF0321142005F07EFF03211520AA
:106D500005F07AFF94F8F03043F0010384F8F03046
:106D600085F3118870BD00BF003802402DE9F0475F
:106D700000F5805588B095F8F830012B0446884618
:106D8000164600F28A80864F57F8232042B947F80A
:106D9000230000F0DDFB95F8F83000EB8300C463BE
:106DA000D7F800A0C4F8348084F83860BAF1000F36
:106DB00065D095F8F830012B71D001212046FFF7FE
:106DC0009FFF302383F31188E26B136823F00203E3
:106DD0001360E26B136843F001031360E36B002759
:106DE0005F6187F3118801212046FFF79BFD002892
:106DF00000F09680D5F8840000F09EFF04F58459D9
:106E0000BA4609F1100920220021684607F0CEFE9B
:106E100002A8FFF701FCCDF818A06A4609EB0703AA
:106E20000DF1180E9446BCE80300F4451860596053
:106E3000624603F10803F5D1DCF800001860203742
:106E40009CF804201A71602FDDD195F8F0306FF3B3
:106E50008203002785F8F0306A4641462046ADF8A7
:106E60000070ADF802708DF80470FFF7FFFCE36B63
:106E700048BB4FF400421A6008B0BDE8F08741F209
:106E80003810FCF741F9814610B15146FFF780FCFC
:106E9000C7F80090B9F1000F8BD10020ECE73868FB
:106EA00003689B6B98470146002886D13868FFF736
:106EB00027FF3868036832465B68414698470028D8
:106EC0007FF47BAFE9E761221A609DF802309DF8FC
:106ED00003201B06120402F4702203F040731343D4
:106EE000BDF80020C2F3090213439DF804201205E7
:106EF000022E02F4E0020CBF4FF0004100211343C8
:106F0000E26B0B43D361E36B13225A61E26B1368AC
:106F100023F00103136039462046FFF703FD08B94B
:106F2000E36BA6E795F8F83093BBE16BD1F800224C
:106F300042F00102C1F80022E16BD1F8002222F4F4
:106F40007C5222F00E02C1F80022E16BD1F800223F
:106F500042F46062C1F80022E26BC2F81432E26BC4
:106F6000C2F80432E26B41F6FF71C2F80C12E26B18
:106F7000C2F84032E26BC2F84432E36B0122C3F83C
:106F80001C22E26BD2F8003223F00103C2F8003277
:106F900095F8F03043F0020385F8F0306CE700BF5D
:106FA0000836002008B500F061FE50EA01030246F1
:106FB00002D0421E61F10001044B186810B10B466B
:106FC000FFF7EEFCBDE8084005F04CB9083600209C
:106FD00008B50020FFF7C8FDBDE8084005F042B93C
:106FE00008B50120FFF7C0FDBDE8084005F03AB93B
:106FF000036800211B68184708B5043006F094FAAE
:10700000012008BD043006F085BA00002DE9F843E0
:1070100006460D4621B9043006F05AFA012424E050
:1070200003685B6898470028F8D100F01FFE104BFA
:107030008846D3F800904FF47A7107464D43D9F84B
:1070400028000368C8219B689847336830465B680E
:10705000984704460028E1D100F008FEC01B61EB10
:107060000801A84271F10003E9D32046BDE8F88386
:107070000825002010B5044B044640F8043B06F0F8
:10708000E5F9204610BD00BF7C56020813B5054C3B
:107090000093246813460A460146E06AFCF7E6FAC4
:1070A00002B010BD08250020FAF720B80FB407B5CC
:1070B000054B04A91B6851F8040B0191984703B0D4
:1070C0005DF804EB04B07047102300207047000007
:1070D00013B50468009224690B46A04702B010BDA6
:1070E00070470000002070470020704713B56C46C1
:1070F00084E8060000F1140394E8030083E8050027
:1071000002B010BD0020704713B56C4684E806003D
:1071100000F10C0394E8030083E8050002B010BD01
:107120000023C0E90333704782B002AB03E90600D5
:1071300002B07047704700000020704770470000A1
:1071400013B50468009224690B46A04702B010BD35
:1071500000207047002070477047000000207047F3
:107160000020704782B002A901E90C0002B070470C
:107170000F2070470F207047012070470020704794
:107180007047000000207047704700007047000003
:107190000120704701207047012070472830704758
:1071A00082B002A9002001E90C0002B07047000083
:1071B00070470000704700007047000070470000F3
:1071C000084606F071BE0000084606F035BF000014
:1071D00073B51E460C461546011D102201A8FCF78A
:1071E00027F932462946204606F0B2FE044601A899
:1071F000FCF73AF9204602B070BD000013B50D222D
:107200000C46011D01A8FCF713F9204606F064FEA8
:10721000044601A8FCF728F9204602B010BD000082
:1072200006F040BE084606F037BE0000084606F0ED
:1072300011BE000010B5064B044640F8803B00F03C
:107240003DFD04F16C0000F039FD204610BD00BF8B
:10725000C45D020808B53020FBF756FF70B100236B
:10726000C0E90333C0E905330371037A022262F3F4
:1072700002030372024B0360024B836208BD00BF2E
:107280003C570208205A020810B4BDF8044001948B
:107290005DF8044B00F0CCBB10B4BDF80440019481
:1072A0005DF8044B00F06EBB00F086BB00F0B6BB8F
:1072B00010B5044B03600446406A08B1FBF730FF89
:1072C000204610BDA856020810B50446FFF7F0FF8F
:1072D0002046FBF721FF204610BD000010B51D4BD6
:1072E000036000210446017100F5705090B0F02257
:1072F000083007F05BFC04F573503830FFF7BAFE36
:10730000022006F0C9FD144B0A94CDE90B34134B4F
:10731000CDE90D34124B0F9310A9024611E9030079
:1073200005AB83E80300DDE90C0103AB83E8030050
:10733000DDE90A0101AB83E803000A4B009304F581
:107340007450234604F10801243000F0C7FF2046A2
:1073500010B010BD7C58020899720108A97201088A
:10736000AD720108897201081B4A1C491C4B10B5FB
:1073700002611C4A42611C4A826102641B4A4264E7
:107380001B4A82641B4AC161C2641B491B4A0162D9
:1073900002651B491B4A416242651B491B4A036047
:1073A000816282651A4B1B491B4A4360C162C265F8
:1073B0001A4B1B491B4A8360016300231A4902666A
:1073C0001A4AC360044641634266C36300F020FC6E
:1073D000174B2360204610BD047800201036002093
:1073E00000570208C0390020D03700203039002073
:1073F0004039002050390020183600206039002024
:10740000FC360020703900202477002080390020CD
:107410001C7700202837002090390020207700209A
:1074200014230020A039002074360020B039002039
:10743000DC57020808B5302383F31188074B1B681B
:107440009A68996B8A4201D0824200D29860986310
:1074500006F09AF9002383F3118808BD70360020E6
:107460002E4D2F4E2B6008B52E4BF2681A60B420BB
:1074700006F0D0FA03F00CFD06F08CFF2A4B1C68D6
:107480004FF4E131206CFCF77FF8206903681B683A
:107490009847A06A03681B6898470A20FFF7CAFF4D
:1074A00006F0D0FF40B12148132106F0DBFF1F4951
:1074B0004C22881807F06CFB1D4B286801229A7338
:1074C00003681B6898471B4B1B6813B11B6ADB07DB
:1074D00001D506F083FFE06A03685B68984738B11E
:1074E000FEF72EFC4FF497724FF40061FEF714FC88
:1074F0000F4801F0EFFEA06A0D4C03681B6B984724
:10750000F3680D4ADA61B42006F084FA286803684B
:107510005B689847204601F0DDFEF7E790360020D3
:1075200070A0002070360020082500202C37002095
:1075300024770020A478002094560208014B186894
:10754000704700BF70360020004870479436002016
:10755000004870479436002038B53F4D3F4C00211D
:10756000284602F08BFA3E492246284607F0ECFAFC
:107570003C483D4D00F096FE3C4800F093FE3C48F0
:1075800000F090FE3B4800F08DFE3B4800F08AFE84
:107590003A4800F087FE3A4800F084FE394800F08F
:1075A00081FE394800F07EFE384B394A1A60394B6B
:1075B000394A1A602846394B40F8843BFFF75AFD98
:1075C0002846374D3749224607F0BEFA2846FFF7CE
:1075D00085FE224634492846344D07F0B5FA344832
:1075E00003F002FE2846334B40F8043B24220021DE
:1075F00007F0DCFA05F13400FFF73CFD4FF0FF33F4
:107600002D49EB642246284607F09EFA2B4B2C4866
:107610002C4D30221A714FF47A72DA804FF4FA62EC
:107620001A81294A1A6001F0F9FD284B002283F8DB
:107630009C202846264A1A60264B40F8043BFFF758
:1076400019FD22462846244907F07EFABDE8384055
:107650002248FFF789BE00BFD0370020A078002065
:1076600035720108303900200478002040390020AC
:107670005039002060390020703900208039002006
:1076800090390020A0390020B03900201C7700205C
:107690000C57020820770020A05702086C5B0208F4
:1076A000C0390020B1710108B571010818360020F9
:1076B000103600208C5B0208B9710108FC360020EE
:1076C0002477002074360020405902082837002013
:1076D000E85F0208B8570208BD710108943600201F
:1076E00070470000037933B108304FF470530860DD
:1076F00013600120704718467047000000F5745071
:10770000243000F0CDBF000010B50446007958B118
:1077100004F5405400F0A8FAD4F8203DC01AB0F5A2
:10772000FA6F2CBF0020012010BD000008B5FEF745
:1077300007FBA2224FF40031FEF7EEFA002008BD4D
:10774000F8B5064602B3CC0801390A44C2F3CC05A9
:107750000127A54218D3B4F5F06F10D2630906EBE8
:10776000830303F5405304F01F02D3F8081C07FA03
:1077700002F20A43C3F8082C0134A4B2E9E7FFF788
:10778000D5FF0028EAD1F7E7F8BD000000F5405327
:10779000022110B503220446A3F8181D0648FFF77E
:1077A00085FC04F57450243000F0B6FF10B903488E
:1077B00000F030FA10BD00BFE0570208065802087A
:1077C00010B50179044679B900F57050F0220830FF
:1077D00007F0ECF92046FFF7D9FF02212171034899
:1077E000BDE81040FFF762BC10BD00BF245802087E
:1077F000B3F5705FF8B507460E4614461D460DD822
:10780000C3F570539A4209D80834FFF7D9FF2A46C6
:1078100039193046BDE8F84007F0BAB9F8BD0000A4
:10782000B3F5705F2DE9F34105460E4690461C46C0
:1078300023D8C3F5705399421FD801F108070744B4
:1078400022463946404607F093F9B0B12846FFF783
:10785000B7FF05F57351F122383101A8FBF7E8FDB8
:1078600022464146384607F093F92846A2B23146EF
:10787000FFF766FF01A8FBF7F7FD02B0BDE8F08156
:1078800037B505460C4601A80121FBF7B7FDE1001D
:1078900005F5745089B20822243000F027FE044612
:1078A00001A8FBF7B7FD204603B030BD2DE9F74F27
:1078B000037904464BB300F5705300F57356083353
:1078C000383653F8042B42B9B342FAD100F0CCF960
:1078D00004F54054C4F8200D17E00025012204F5FA
:1078E0004051C5F34A134FEA830901EB830305F0C6
:1078F0001F07D3F8083C02FA07F71F421FFA85FA60
:1079000006D10135B5F5F06FEBD103B0BDE8F08FCE
:10791000ED004FF488723146083501A8FBF788FD69
:1079200043F610526359A35004EB050B04EB020815
:10793000DBF80430C8F8043001A8FBF795FD237983
:10794000022BE2D151462046FFF79AFF0028DCD0F7
:107950004FF49C72314601A8FBF76AFD0822594694
:10796000404607F005F940B94C4404F54054D4F8BA
:10797000083C23EA0703C4F8083C01A8FBF774FDA0
:10798000C3E7000038B51C460A4B1B6815465A6B06
:1079900000F54053B3F8180D136801441B681046F6
:1079A0009847BDF810204119204607F0F1F8012052
:1079B00038BD00BF082500202DE9F743DFF85890B7
:1079C00006460F4605244FF47A7101A8FBF716FD11
:1079D000D9F8008006F54053D8F83400B3F8181DE4
:1079E00003683944DB689847054630B101A8FBF7C6
:1079F00011FD284603B0BDE8F083D8F828000368DD
:107A000001215B689847013C01A8FBF703FD14F0D6
:107A1000FF04D8D1EDE700BF08250020034B1B6809
:107A2000DB6A93F89C0080F0010070470825002075
:107A30002DE9F04F2DED028B08EE103A2C4BD3F8C8
:107A40000090044604F54053D9F834000F46B3F8CB
:107A5000181D036885B01B68BDF840B039449046D6
:107A60009847052500EB080A012103A8FBF7C6FC8F
:107A7000D9F83400036818EE102A1E6951465B4697
:107A8000B047064640B103A8FBF7C4FC304605B03A
:107A9000BDEC028BBDE8F08FD9F828000368012106
:107AA0005B689847013D03A8FBF7B4FC15F0FF05A0
:107AB000DAD12046FFF7B2FF0028E7D000F0D4F873
:107AC00004F5405241F28831D2F81C3DC31A8B4272
:107AD000DCD9C2F81C0D04F57450243000F00AFE05
:107AE0005B460090424639460248FFF7DFFACDE791
:107AF000082500204458020870B51D46164B1B6827
:107B000013B11B6ADB0725D5144B1E68F46A94F881
:107B10004630C3B9124BA4F84400DB6884F8461021
:107B2000E26163B19A6884F84720D96939B194F960
:107B3000483023B9042204F1480000F099F8094BB9
:107B40005B68C4E90835F06A1321BDE87040043071
:107B500006F082BC70BD00BFA4780020082500207C
:107B600070A0002000ED00E000B59BB0EFF30981AC
:107B70006822684607F00CF8EFF30581074BC9B29D
:107B80009A6BD86A986A986A986A986A986A9B6A9F
:107B9000059B7B20FFF7B0FFFEE700BF00ED00E094
:107BA00000B59BB0EFF309816822684606F0F0FF4C
:107BB000EFF30581064BC9B29A6B986A986A986A86
:107BC000986A986A9B6A059BBF20FFF795FFFEE7BE
:107BD00000ED00E000B59BB0EFF309816822684634
:107BE00006F0D6FFEFF30581064BC9B25A6B986ACF
:107BF000986A986A986A9B6A059BE320FFF77CFF66
:107C0000FEE700BF00ED00E0FEE70000FEE7000039
:107C1000704700000FB483B504AC0F4F54F8048BC9
:107C20000E4EFEF78DF84FF4A5722021FEF774F882
:107C300042F21075214640460194FFF735FA384666
:107C4000FFF734FA3368986A036829465B689847F7
:107C50004FF4FA75EEE700BFA06002080825002087
:107C60004FF08043586A704706F0FCBA06F0DEBA5F
:107C7000F8B50D46074611462846164607F06CFC37
:107C8000864204468CBF421C02462946384606F00E
:107C90007FFF2046F8BD000070B500260446C0E90D
:107CA000026601200D4606F05FFAB04208BF354675
:107CB000206065602674204670BD000010B5037C0E
:107CC000044613B9006806F053FA204610BD0000C0
:107CD00070B5057C04460E46DDB9BFF35B8FC56009
:107CE000BFF35B8FBFF35B8F8560BFF35B8F436830
:107CF0008B420CD0006806F03BFA3146012006F0BA
:107D000033FA206010B96560284670BD66600125B1
:107D1000FAE70025F8E7000038B505460C4644B1FF
:107D200021462846FFF7D4FF20B904EB4404A408F9
:107D3000F5E7204638BD00000023BFF35B8FC3602A
:107D4000BFF35B8FBFF35B8F8360BFF35B8F7047C5
:107D5000BFF35B8F0068BFF35B8F704770B505465C
:107D60000C30FFF7F5FF05F1080604463046FFF733
:107D7000EFFFA04206D930466D68FFF7E9FF2544C2
:107D8000281A70BD3046FFF7E3FF201AF9E700001C
:107D900070B50546406898B105F10800FFF7D8FFB7
:107DA00005F10C0604463046FFF7D2FF8442304608
:107DB00094BF6D680025FFF7CBFF013C2C44201ACF
:107DC00070BD000038B50C460546FFF7C7FFA0425E
:107DD00010D305F10800FFF7BBFF04446868B4FB4B
:107DE000F0F100FB1144BFF35B8F0120AC60BFF3E7
:107DF0005B8F38BD0020FCE72DE9F04114460746B3
:107E00000D46FFF7C5FF844228BF0446D4B1B846EB
:107E100058F80C6B4046FFF79BFF30442860404603
:107E20007E68FFF795FF331A9C4203D86C600120EF
:107E3000BDE8F0816B60A41B3B68AB602044E86048
:107E40000220F5E72046F3E738B50C460546FFF774
:107E50009FFFA04210D305F10C00FFF779FF044407
:107E60006868B4FBF0F100FB1144BFF35B8F0120A5
:107E7000EC60BFF35B8F38BD0020FCE72DE9FF41CC
:107E8000884669460746FFF7B7FF6C4606B204EB23
:107E9000C6060025B44209D06268206808EB0501D7
:107EA00006F076FE636808341D44F3E72946384639
:107EB000FFF7CAFF284604B0BDE8F081F8B50546D3
:107EC0000C300F46FFF744FF05F108060446304624
:107ED000FFF73EFFA042304688BF6C68FFF738FFCF
:107EE000201A386020B130462C68FFF731FF20445B
:107EF000F8BD000073B5144606460D46FFF72EFF89
:107F0000844228BF04460190DCB101A93046FFF746
:107F1000D5FF019B33B93268C5E90233C5E90024B6
:107F200001200CE09C4238BF0194286001986860F1
:107F30008442F5D93368AB60241AEC60022002B0A9
:107F400070BD2046FBE700002DE9FF410F46694662
:107F5000FFF7D0FF6C4600B204EBC0050026AC4230
:107F600009D0D4F8048054F8081BB819424606F02A
:107F70000FFE4644F3E7304604B0BDE8F081000050
:107F800038B50546FFF7E0FF044601462846FFF7EF
:107F900019FF204638BD00002DE9F74F10EE103ACA
:107FA000009210EE102A072928BF0721C3F31604F8
:107FB0004FEAD37812024FEAD35307460E4603F036
:107FC000FE0340F1A6800133DBB2FF2B32D044F434
:107FD0000004DA0859495A4811F90290594951F8F0
:107FE000225003F00703A4FB0554C3F10F02113321
:107FF000B2F1200104FA03F325FA02F558BF44FA5E
:1080000001F145EA03054FF0000B58BF0D43144141
:1080100045F6F321CDF804B04FF0300A2A1A64EB8C
:108020000103002B0DDB0AF1010A4FFA8AFA15460B
:108030001C46F3E714B948F00408C8E748F00808FC
:10804000C5E700230A22F8F7C9FD019BD3B9BAF1AD
:10805000300F06D109F1FF394FFA89F92A46234634
:10806000E5E7009BF3B1009A09F101035BB2013A25
:10807000012BACBFD218013202F0FF039E420093E5
:1080800028BF1E460BF10103BAF1390FDAB257FAD5
:1080900083FC0ADC0123964207F802A0019319D958
:1080A0009346B9E70136F6B2ECE7A2EB0B003921B3
:1080B0003844CDF800C006F079FDDDF800C0634615
:1080C00030201946013B0A78013252B23A2A13D0C5
:1080D0000A700CE00A22A0FB0206400840EAC670C3
:1080E000281A02FB016164EB6104002CE7DA87F8CF
:1080F00000800FFA89F01DE0BB4208D1312309F15D
:1081000001090B704FFA89F948F01008EFE7587031
:10811000D7E7002B7FF45BAF002C7FF45AAF3846D3
:1081200048F00208721C00F8018BD2B2302106F030
:108130003DFD204603B0BDE8F08F00BF185902088E
:1081400000407A10985802087047000070470000FD
:108150000020704770470000704700007047000023
:1081600003689B6B184700000368DB6B184700002F
:1081700070470000002070477047000000207047E3
:108180009FED010A704700BF0000C8420020704701
:1081900000207047002070477047000000207047A3
:1081A00000207047002070477047000070470000B3
:1081B0007047000000230B600120704700207047CB
:1081C00000207047704700007047000070470000B3
:1081D00070470000704700007047000000207047A3
:1081E0007047000000207047704700007047000093
:1081F0000020704700207047002070477047000043
:108200000020704770470000704700007047000072
:108210007047000070470000704700003220704730
:10822000704700000F299CBF00EB4100428170475E
:108230000F299ABF00EB410040894FF461707047ED
:10824000102A0B4628BF102200F10A0152001846DE
:1082500006F09EBC03790BB10022027118467047EC
:1082600003685B681847000003791BB90123037199
:1082700018467047002070477047000010B504464C
:10828000FAF74AFF204610BD704700007047000013
:10829000002070470020704701207047104670474B
:1082A00000207047014B0360704700BF405A02082E
:1082B00030B5094D0A4491420DD011F8013B5840A8
:1082C000082340F30004013B2C4013F0FF0384EA31
:1082D0005000F6D1EFE730BD2083B8ED82B010B585
:1082E000044602A8C4E9001240F8043F03C804F1A0
:1082F000080383E80300DDE9050104F1100383E8C6
:108300000300DDE9070104F1180383E80300DDE958
:10831000090104F1200383E803002046BDE8104072
:1083200002B0704710B50A4492B2914208D0046876
:108330004B1C615C9BB209B1002010BD1946F4E7EB
:108340000120FAE70378FF2B06D0FE2B06D0FC2B8A
:1083500014BF04200320704701207047022070479B
:1083600010B4BDF804400194D0E90004A4465DF8BF
:10837000044B60472DE9F043054685B08946042447
:1083800000F110074FF002086B68023BA3423BD993
:10839000CDF8008003AB224649463846FFF7E0FFA0
:1083A00040B19DF80C3003F00303012B08D0032BE0
:1083B00002D063B1002000E0EC6205B0BDE8F083BC
:1083C0009DF80D305B0904EBC3040A34DCE7BDF80B
:1083D0000C309DF80D20C3F38A035209DB000132F3
:1083E0009BB2D60003EBC202B2F5705FE2DC2A68F2
:1083F000009613444946A21C3846FFF7B1FF0028F7
:10840000D8D002363444BFE7EC620120D5E7000043
:1084100010B4BDF804400194D0E90004A4465DF80E
:10842000044B6047F0B5026B87B004466AB990F818
:108430002850039285F001050426009605AB2946D5
:108440001030FFF78DFF039A08B900202DE0059B3F
:10845000174923F0FF038B4203D0012384F8343003
:10846000F3E705A8FFF76EFF0128F6D1114B05933E
:1084700004F1080794F82810009605AB38460392DB
:10848000FFF7C6FF0028E0D00B4B0593039A009638
:1084900005AB29463846FFF7BBFF0028D5D043F689
:1084A0002063C4E90B6384F8285007B0F0BD00BF17
:1084B000005B6851FC5B6851FE5B68517FB5044608
:1084C000D0E906030D461646984758B156B1064BFB
:1084D000039304230093002203AB294604F1080010
:1084E000FFF796FF04B070BDFF5B68512DE9F047C0
:1084F00090F8343094B005460F461646002B3FD115
:108500004FF00108002E7BD06B68EA6A9A1A2B6B39
:108510003F2E03F1420394BF344640249A42E4B212
:1085200032D39DF80C3068F301038DF80C30BDF8A0
:108530000C30C7F3CA01073461F38C03C4F3C404DD
:10854000ADF80C30621EA946C3F3072362F347134C
:108550008DF80D3059F8083BE40003EBC1012246C9
:108560000DF10E004FF0020A06F012FBEA6A95F8D0
:108570002810CDF800A003AB4846FFF749FF98B993
:10858000002014B0BDE8F0872846FFF74BFF002815
:10859000C7D1D5E9080398470028F1D0284600F054
:1085A00069F80028BDD1EBE7EA6A95F82810009435
:1085B0000DF10E0302324846FFF72AFF0028DFD0F4
:1085C0009DF80C30EA6A95F82810CDF800A06FF3FA
:1085D00001038DF80C30484603ABFFF719FF002864
:1085E000CED0EB6A02332344EB6207F00703E41AB0
:1085F000E4B2B442C5DC2744341BBFB2A6B281E763
:108600000120BEE737B505464FF47054402C224692
:10861000C4F57051A8BF402289B292B22846CDE974
:108620000012FFF77FFEDDE9001218B1403CEDD1EA
:10863000012004E02846FFF759FF0028F6D103B0D7
:1086400030BD0000002310B580F8343003630446C9
:10865000FFF7D8FF60B194F828100122514020465E
:10866000FFF72CFF20B12046BDE81040FFF7DABE2F
:10867000002010BD38B590F83550044645B1FDF7DF
:108680005FFB91224FF40011FDF746FB002038BD3F
:10869000012380F83530FFF7D5FF84F83550F6E731
:1086A0007FB50025042680F8345080F82850C66233
:1086B0002A4629460446FFF701FF10B9002004B0FE
:1086C00070BD94F82820013A18BF012201212046EC
:1086D000FFF7F4FE0028F1D0054B039394F828101F
:1086E000009603AB2A4604F10800FFF791FEE6E787
:1086F000FE5B685110B50446D0E90803984740B1C5
:108700002046FFF7CDFF20B12046BDE81040FFF71F
:1087100079BF002010BD00002DE9F04F074687B05B
:1087200005464FF4705257F8100BDFF81CB10021CA
:1087300006F03CFA0DF1100A0026D14604230093FE
:108740000022534631463846FFF70AFED04604461B
:1087500030B90024204607B0BDE8F08F0126EDE7D0
:108760004046FFF7EFFD0138D8F80020C0B20228DC
:108770000AF1040A22F0FF0201D85A4504D0284623
:10878000FFF78EFF0446E5E7002EE7D04846FFF7E7
:10879000D9FD07468DF80C0005A8FFF7D3FD8742E9
:1087A00080468DF80D0003D1012FE8D1002608E0A6
:1087B000032FFBD0032804D0022FF7D0831E5E4284
:1087C0005E4106AB334413F80C9CA9F10203012B64
:1087D00005D831462846FFF7CDFD0028CFD086F0DA
:1087E000010106AB0B4413F80C3C023B012B04D8EF
:1087F0002846FFF7BFFD0028C1D00023B9F1030FC1
:1088000085F834302B6315D0032F06D101220021C7
:108810002846FFF753FE00289BD0B8F1030F06D17E
:10882000012211462846FFF749FE002891D0002377
:108830002B638FE786F0010685F828602846FFF74E
:10884000E1FE0028E0D19AE7005B685190ED120A42
:108850007047000090ED130A70470000B0F8540014
:1088600070470000B0F856007047000090ED040A11
:108870007047000010B52DED028B044682B000F168
:108880002001782201A8FAF7D3FD237D53B994ED96
:10889000028A01A8FAF7E8FDB0EE480A02B0BDEC82
:1088A000028B10BD07EE903A94ED067AD4ED076A7C
:1088B000F8EEE77A002387EE278AA361E3610023BD
:1088C000237586EEA77A84ED028A84ED037AE0E7C9
:1088D000F7B506460F4640F2063200F1840101A8C2
:1088E000FAF7A6FD0025331D53F8042B9AB938205A
:1088F000FAF70AFC044628B10D4B0360878020304C
:10890000FEF7B8FB06EB85056C6001A8FAF7ACFD35
:10891000204603B0F0BD0135102DE5D1054B0649C9
:108920001B68986903681B6898470024EDE700BF3F
:108930004C5B020808250020D85A0208FF2937B5E9
:1089400005460C4626D0B0F904308B421FD067296B
:108950000BD0052909D0062907D0012905D0022905
:1089600003D0032901D0042914D1EB2205F1200101
:1089700001A8FAF75DFD00230022AC80AB61EB613A
:108980002A752B61AB60EB6001A8FAF76DFD012041
:1089900003B030BD0020FBE7F8B50F4B83421AD17E
:1089A0000E4B0F4E1C686021204605F005FD04F1BA
:1089B000600520460023316830F8027BCA583A44EB
:1089C000CA500433182BF6D10C34A542F1D1054A14
:1089D000136808331360F8BDC09C0020B0780020F5
:1089E000A8780020AC7800202DE9F0412E4B2F4EC6
:1089F0001B680446D86A036800229B6C6021984774
:108A0000306000284CD0182005F080FB284B1860FF
:108A1000002845D00021274804F1580504F04CF9FE
:108A20002C220021284606F0C1F8012384F8583092
:108A30000623A4F85A30204BE3654FF4A003A36744
:108A40004FF08043A366DFF878E0002318464FF02C
:108A5000070C1EF83320092A18D802EB42010CFA41
:108A600001F7216F3943216703EB830101338A400A
:108A7000062B40EA0200ECD1C4F8800032680D48B1
:108A800029460823BDE8F04104F024B9A2F10A0107
:108A9000E76E01EB41010CFA01F13943E166E3E7CE
:108AA0000648FFF7B7F800BF08250020B07800207F
:108AB000A8780020C09C002099890108F05A02087B
:108AC000145B0208FFF790BF10B5B0F90420094805
:108AD000002300EBC3014C78944204D1FF2A02D05A
:108AE00091ED010A10BD0133062BF2D19FED020A70
:108AF000F8E700BF145B02086740533A10B504461C
:108B00002DED028BFFF7E0FF236820461B68B0EED7
:108B1000408A984728EE000ABDEC028B10BD000089
:108B200010B503680446DB6898472046FFF7CCFF82
:108B3000D4ED037A20EE270A10BD000010B50446DC
:108B40002DED028BFFF7C0FF236820465B68B0EE77
:108B5000408A984728EE000ABDEC028B10BD000049
:108B600010B52DED028B82B0044600F12001FB22EE
:108B700001A8B0EE408AF0EE608AFAF759FCF0EEF8
:108B8000087AF4EEE78AF1EE10FA5CBFB1EE040A5F
:108B900028EE000A237DD4ED077A94ED067A84ED61
:108BA000048A58BFC0EE286A03F10103DBB22375C3
:108BB0004CBF38EE270A36EEA70A38EE077AFE2BAE
:108BC00084ED067A84ED070A0BD1F6EE007A27EEE3
:108BD000277A20EE270A7F2384ED067A84ED070AA0
:108BE000237501A8FAF740FC02B0BDEC028B10BD62
:108BF00038B51346302282F3118819B1002383F36C
:108C0000118838BD09480A4C0A4601682568895808
:108C1000B1FBF5F199500432182AF6D10068002111
:108C200005F0C4FF00232360E9E700BFA878002017
:108C3000AC7800202DE9F04F2DED028B83B000AF12
:108C40000B1E7B600CBF4FF006084FF000086B4610
:108C5000A3EB88039D46E9464A460446FFF7C8FF52
:108C60009FED1C8A0025EBB298452CD91A4B261D86
:108C700004F1440A03EBC50B56F8040B98B17B686A
:108C8000ABB99BF80110B0F904C0614511D1FF29BF
:108C900009D059F82530D4ED120A07EE903AB8EE13
:108CA000670AFFF75DFF5645E6D10135DBE7FF2197
:108CB000E9E7BCF1670FF6D194ED140ADFED070A7E
:108CC00080EE080AEDE70C37BD46BDEC028BBDE82F
:108CD000F08F00BF6740533A145B020800000000A9
:108CE000B0F854305BB133F0200308D0084B1B6858
:108CF000DB6A93F89C30002B0CBF00232023B0F8D4
:108D00005620A0F854301A43A0F85620704700BFF0
:108D10000825002010B50446FEF7A2FF636C42F25E
:108D20000F72C31A934208D960642046FFF7D8FF38
:108D30000021BDE81040FFF77DBF10BD7047000067
:108D400000207047B0F94C0070470000B0F94E00A9
:108D500070470000012380F85430704780F85510A8
:108D60007047000090F8543013B190F8300070470D
:108D70001846704737B590F8543004460D46ABB1ED
:108D800090F83030122BA8BF122399420EDA00F16E
:108D90003401612201A804EB4504FAF749FB01A85C
:108DA000A488FAF761FB204603B030BD0024FAE73F
:108DB00037B590F854500446A5B100F134014A2269
:108DC00001A8FAF735FBD4E90A51226D0023994234
:108DD00008BF9542C4E90A2301A814BF0125002554
:108DE000FAF742FB284603B030BD000073B590F897
:108DF000544005460E468CB1122A28BF122200F1BB
:108E00003401144601A87122FAF712FB6200291DF1
:108E1000304605F0BDFE01A8FAF726FB204602B059
:108E200070BD000070470000407B704701617047D3
:108E300010B5074B074ADB680446DA61A37B33B9F8
:108E400023684FF47A719B6820469847F6E710BD77
:108E500070A00020B45B020838B50D4B0D4ADB68EA
:108E60000446DA612368A27B9B6862B10A4D2368DD
:108E700020469B684FF47A7198472B6858690368BD
:108E80001B699847F3E742F2107120469847E9E7DB
:108E900070A000201B5802080825002013B50446C6
:108EA0000121C83004F07CFC04F1D400012104F05D
:108EB00077FC1A4B0094B5224FF4FE61184804F079
:108EC00033FD184BC4F8B0000094B5224FF47C7108
:108ED000154804F029FD154BC4F8B4000094B122E4
:108EE0004FF4BE61124804F01FFD124BC4F8B800E5
:108EF00000943A224FF41F610F4804F015FD0F4B08
:108F0000C4F8BC0000943B224FF4BE610C4804F04E
:108F10000BFDC4F8C00002B010BD00BFF5930108FE
:108F200078920020318E0108988800200D91010868
:108F3000A882002089940108B8780020598E010881
:108F4000888C002070B5437D04460D464BB90368FC
:108F50001B6C984728B1B620FEF76CFA40F201135B
:108F6000A3822368294620469B68BDE870401847C5
:108F700008B5FEF7E3FA034BDB681B1A5842584169
:108F800008BD00BF70A000202DE9F04704460D4643
:108F9000FEF76CFEDFF8689006460F46FEF766FEA9
:108FA000801B4FF0000361EB07014FF47A72F7F773
:108FB00065FEA84271F1000320D223684FF47A7154
:108FC0009B6820469847A388AB42E7D82368204691
:108FD0001B6C98470028E1D0D9F80080D8F82C30D5
:108FE000FC2293F94CA083F84C2023682046DB6CCC
:108FF0009847D8F82C3083F84CA0CFE7BDE8F0872D
:109000000825002008B5302282F311888368002BE0
:1090100001DC04F0EBFB04F0B7FB002383F31188C1
:1090200008BD0000F7B5044600F1C8066D4630469D
:1090300085E8060004F0D0FB94F86430DDE9000711
:10904000224604EBC30C62450DD0516A814208D11F
:10905000916AB94205D1304603B0BDE8F040FFF750
:10906000D1BF0832EFE7072B0AD895E8030004EBDD
:10907000C3022432013382E8030084F86430EAE753
:10908000034B04491B68986903681B689847E2E72B
:1090900008250020BC5B020808B50E4B1B68586A07
:1090A0000368DB6C0C4698470B4B0C48002C08BF40
:1090B000184605F061F972B6BFF34F8F0849094BA6
:1090C000CA6802F4E0621343CB60BFF34F8F00BF66
:1090D000FDE700BF08250020020007B0010007B02F
:1090E00000ED00E00400FA0510B5836904461BB9E1
:1090F000BDE8104004F0B4BFFEF7B6FDA369C01A86
:10910000E3699842F4D8012010BD000038B50D4B3A
:109110000D4ADB680446DA612368A27B9B685AB17A
:109120000A4D236820469B684FF47A7198472B6854
:10913000186AFFF777FEF4E744F620612046984767
:10914000EAE700BF70A00020D45B020808250020D9
:1091500008B5437B13B10348FEF75CFD012343735D
:1091600008BD00BFDC5B020804F07CBB084604F0CD
:1091700083BB000029B10A2938BF0A21084604F040
:1091800061BC704710B503681B6C0446984740B13A
:10919000637D33B100236375B420BDE81040FEF752
:1091A00049B910BDF7B5044600F1D4066D46304606
:1091B00085E8060004F010FB94F8A830DDE900070C
:1091C000224604EBC30C62450DD0916E814208D15A
:1091D000D16EB94205D1304603B0BDE8F040FFF78B
:1091E00011BF0832EFE7072B0BD895E8030003F116
:1091F0000D0204EBC202013382E8030084F8A830B8
:10920000E9E7044B04491B68986903681B689847A1
:10921000E1E700BF082500201C5C020810B5084BE0
:109220000446402240F8243B002105F0BFFC4022C8
:10923000002104F1680005F0B9FC204610BD00BF14
:10924000485C020810B50B4C1046002314F813209C
:109250008A4209D104EB4303FF225B7802211844C0
:10926000FAF7EAFEC0B210BD01330E2BEED13A2060
:10927000F9E700BF9C5C0208F0B585B0074602AD77
:10928000082085E806001E4604F040FF0446D8B1D9
:1092900095E803009DF9302084E803009DF82C1028
:1092A0003846FFF7CFFF0A9D094B009405F2F715EA
:1092B0000246314625F0070004F084FF054628B930
:1092C000204604F055FF284605B0F0BD0120FBE71D
:1092D000DD94010810B5044605F094F8FEF7C4FCCF
:1092E000C4F8AC0010BD000070B503681B6C0446E8
:1092F0000D46984738B12046FFF7ECFF4DB9236A79
:1093000013B90023A36170BD013B2362002BFAD186
:10931000F7E7FEF7A9FCA36943B1E269C11A8A42E3
:1093200004D913441B1A9D4238BF1D46236AC4E961
:10933000060501332362236820469B69BDE870401F
:109340001847000010B5114805F03EF83F2807D82F
:10935000FCF7F6FC4FF6FF724FF40001FCF7DCFC63
:1093600004F018F9044678B1006A05F02DF83F289A
:1093700006D8FCF7E5FC228F4FF40001FCF7CCFC8B
:10938000204604F017F9EDE710BD00BF00010020F2
:10939000D0E9000318470000F8B590F8653004469E
:1093A00003F0FF051BBB012300F1C80680F8653000
:1093B000304604F011FA304694F86470FFF722FE4C
:1093C00004F12406AF4207DD736813B13046FFF79E
:1093D000DFFF01350836F5E7236903B19847044BF1
:1093E0001B681869FFF796FC002384F86530F8BD08
:1093F0000825002010B5104B104ADB680446DA61DE
:109400002368A27B9B6822B94FF47A712046984763
:10941000F6E723684FF47A719B6820469847204608
:10942000FFF7BAFF236820465B6998470028F0D011
:109430002046FFF74FFFECE770A00020345C0208E5
:10944000F8B590F8A930044603F0FF05DBB9012315
:1094500000F1D40680F8A930304604F0BDF930465A
:1094600094F8A870FFF7CEFD04F16806AF4207DD5F
:10947000736813B13046FFF78BFF01350836F5E707
:10948000002384F8A930F8BD70B5124B124ADB688E
:109490000446DA612368A27B9B6822B94FF47A7193
:1094A00020469847F6E7002623684FF47A719B68B8
:1094B000204698472046FFF7C3FFFEF7D5FB831BE6
:1094C000B3F57A7F0546EFD92046FFF73BFF2E46DE
:1094D000EAE700BF70A000203C5C020810B504461B
:1094E000FFF756FF2046BDE8104004F041BE0000E3
:1094F00090F801017047000003695B7923B9406B64
:109500000A23B0FBF3F070474FF448307047000077
:10951000406B7047037D03B1437D184670470000E0
:1095200010B5054B1B689B690A4619684C680146D3
:109530001846A047012010BD0825002090F8E9201A
:10954000034602F0FF0012B193F8E800C0B2704782
:109550000020704700207047F8B590F80031476B45
:109560001E330C4600EBC30150F833504E6877B100
:1095700003695B795BB903685B6998472044054BD5
:10958000B3FBF7F35843281A054666F10006284650
:109590003146F8BD80969800C089704708B5803084
:1095A000FEF7DCFB003818BF012008BD90F8E8305A
:1095B0003BB1054BC26CDB689A4202D16C30FEF7BE
:1095C000CDBB0020704700BF70A0002013B540F253
:1095D0007F22044600F1D0016846F9F729FF4FF4D5
:1095E000207204F1B80101A8F9F722FF002384F8E2
:1095F000E83084F8E93023695A7912B9186803F021
:1096000049FD002104F16C00FEF762FB002104F12A
:109610008000FEF75DFB01A8F9F726FF6846F9F721
:1096200023FF02B010BD000008B580F84411806A25
:10963000082103F0B9FE012008BD000090F8E920E0
:10964000034602F0FF001AB103F18000FEF7A0BB51
:10965000704700002DE9F843174604460D46FEF713
:1096600003FBDFF85C90064600EB07082368204602
:109670005B699847A84218D24FF4806003F068FEF7
:10968000D9F80C30A4F854502365FEF7EDFA821B8C
:10969000BA420AD2A8EB00034FF47A71A3FB01137C
:1096A0004FF4806003F0A0FEE0E7236820465B698A
:1096B000984785428CBF00200120BDE8F88300BF99
:1096C00070A0002038B50446302383F311880B07BF
:1096D00007D5FCF735FB40F232324FF00061FCF762
:1096E0001BFBD4F8B4301A68136823F01F0313600F
:1096F000D4F8B42011680D6815F00105FBD151684C
:10970000527A3D2393400B60FEF7AAFA0221C4F877
:109710000401A06A03F032FE85F3118838BD000011
:1097200070B503695A790446002A46D11D68036A58
:10973000002B08BF0021036880F80111DB6A9847FD
:1097400000283AD094F80131032B36D8DFE803F033
:109750000239366A206A88B1012600F00F013246CC
:1097600006FA01F120F00F0003F0F6F8236A23F067
:109770000F0203F00F039E40B6B25683012384F814
:109780000231302383F31188D5F854325A6912F428
:10979000407F0FD0DA6822F40052DA60D5F8542204
:1097A000536923F440735361D5F85422D36843F4CA
:1097B0000053D360002383F3118870BD0023C4E9F4
:1097C0004133206A012600F00F01324606FA01F10A
:1097D00020F00F0003F0C0F8236A23F00F0203F01B
:1097E0000F0306FA03F39BB2538384F8026130231C
:1097F00083F31188D5F854325A6902F44072B2F5F5
:10980000007FD7D0DA6822F40052DA60D5F854220B
:10981000536943F400735361D5F85422536923F418
:109820008073C0E723682046DB6BBDE870400021F1
:109830001847000010B50446C06940B100F00F039E
:1098400001210022994020F00F0003F085F8A06963
:1098500050B100F00F030121BDE8104000229940F3
:1098600020F00F0003F078B810BD000038B5036990
:109870005A7904460D46002A37D10173186803F05F
:1098800009FC012D32D0022D34D01DB9A38F23F451
:10989000B053A387236904F13801186803F0ECFB87
:1098A00094F85C3133B12369186804F5A47104306D
:1098B00003F034FD002D14BF0123002384F85C3134
:1098C00009D0236918684FF40062202304F5A471BD
:1098D000043003F00FFD237D3BB123691B68D3F8EF
:1098E0005422D36823F02003D36038BDA38F43F400
:1098F000B053CEE7A38F23F4007343F4A053C8E71B
:10990000037D82B0C3B103691B68D3F85422136886
:109910009BB2ADF80430BDF80430DB060CD55368BB
:109920009BB2ADF80630BDF80630D0F8B0301A68FA
:10993000136823F00103136002B0704738B5036960
:109940005A7904460D46DAB9186803F0A3FB012DD5
:10995000D4F8203115D0022D18D0D4F82031E38767
:10996000236904F13801186803F086FB237D3BB1BD
:1099700023691B68D3F85422D36823F02003D360F3
:1099800038BD23F40053C4F82031E6E743F4005314
:10999000F9E7000003695B791BB9806A042103F0D1
:1099A00003BD7047F7B590F8E93004460E461746F8
:1099B00003F0FF05BBB100F198014FF4427201A81A
:1099C000F9F736FD3A46314604F18000FEF756FAC3
:1099D00094F8443105461BB1A06A042103F0E4FC6D
:1099E00001A8F9F741FD284603B0F0BD70B590F825
:1099F000013105460C46D3B9406AB8B1012600F0E2
:109A00000F0106FA01F120F00F00324602F0A4FF28
:109A10006D6A05F00F0184EA060001F11003984019
:109A20008C4025F00F050443AC61304670BD00202A
:109A3000FCE7000070B590F8013105460C46D3B93B
:109A4000006AB8B1012600F00F0106FA01F120F01A
:109A50000F00324602F080FF2D6A05F00F0184EA04
:109A6000060001F1100398408C4025F00F050443D7
:109A7000AC61304670BD0020FCE70000164B10B50D
:109A80000360164B80F832102C2201FB0233036175
:109A90004FF461430446436300216C30FEF7FCF849
:109AA000002104F18000FEF7F7F804F19800FDF7BB
:109AB000E1FA04F1B800FDF7DDFA04F1D000FDF79A
:109AC000D9FA002394F8322084F80131044B43F88A
:109AD0002240204610BD00BFC45D0208385D020868
:109AE000689A002013B5094C23686BB900930849A4
:109AF000084B3C224FF49E6004F064FB2060236816
:109B000013B90548FEF786F802B010BD949A0020FC
:109B1000B85C0208F9A70108C05C020830B5836A86
:109B200085B004462BBB144B22691B685579D86A53
:109B300013790093114A124B04F12C01002D08BF38
:109B4000134606220391F9F7B1FD94F844310399C5
:109B50000094002B18BFB5220A4B08BF3C224FF4DB
:109B60004C7004F02FFBA062A36A13B90648FEF7FD
:109B700051F805B030BD00BF08250020E75C0208A1
:109B8000E05C020805A70108EF5C020838B5D0F8D0
:109B9000B4500446B5B9302383F3118800690A4AEA
:109BA000407B23460C2102F047FEC4F8B40085F345
:109BB0001188D4F8B4301A6823691B68D3F854327A
:109BC0000433936038BD00BFC5960108FFF7DEBFC0
:109BD00038B503699D6890F8583083F0010380F828
:109BE000583090F8583000EB830304464021D86D7C
:109BF00004F0E2FB94F85830D4F8B02004EB83036F
:109C00001268DB6DD360D4F8B0301B6840225A6014
:109C1000D4F8B0306D061A6845F4826545F0060543
:109C20001560D4F8B0301A68136843F0010313606C
:109C300038BD00002DE9F04104468AB090461F4629
:109C40000E4671B957EA02030BD190F8E93043B1DF
:109C500090F8E8302BB1554BDB68C3640AB0BDE81F
:109C6000F081FFF73FFF23691A68002AF6D05B797D
:109C70004FF4C870B6FBF0F0B0F5007F38BF4FF47A
:109C80000070002B0CBF4FF400734FF4806385B25B
:109C90009F4238BF1F464FF49472454504F1D001EE
:109CA00004A838BF4546F9F7C3FB236F9D4207D090
:109CB000002384F8E830294604F16C00FEF72CF804
:109CC000236F1B09C4F89430B6B1636BB3425ED006
:109CD000374B1B689B696663A34258D004F16C053F
:109CE0002846FEF73BF8D4F818311844C4F8180198
:109CF0002846FEF721F8012694F82831E3B9E389D4
:109D0000D90519D4E26D52B923699B793BB1284B2F
:109D10001B68D86A036840219B6C9847E065226EF7
:109D200052B923699B793BB1214B1B68D86A036800
:109D300040219B6C98472066636E73B923691B7B37
:109D40005BB1E28912F4007207D1194B1B68D86A23
:109D5000036840219B6C9847606694F82831C3B132
:109D60000023A382B4F86820636BB2F57A7F21D90F
:109D7000B3F5E13F21D80023637523691A7BE2B173
:109D8000587B01F0B3F8C0B10023637515E00026DD
:109D9000B2E7E26D1AB1236E003B18BF01232375B1
:109DA000636E003B18BF01236375DBE770A00020E2
:109DB00008250020B3F5E13FDFD940F2671204F136
:109DC000B80105A8F9F734FBD4F884309F4207D0D6
:109DD000002384F8E930394604F18000FDF79CFF48
:109DE0001EB104F18000FDF7A7FF23695B79002B0A
:109DF00040F09280636B002B00F08E8094F8EA6054
:109E000094F8EA30F6B203F0FF05DBB9237DB3B175
:109E1000302383F311882069534AC07923460C21EB
:109E200002F00AFDC4F8B00085F31188D4F8B03010
:109E30001A6823691B68D3F85432043393600123F2
:109E400084F8EA30637D0BB3D4F8EC30F3B9474BB8
:109E50000694CDE907341420454B0993F9F754F9DA
:109E6000054678B10AAA12E9030023695F7B01ABBA
:109E700083E80300079B0093FF22069B3946284690
:109E800001F014F8C4F8EC5005B96575636BA36371
:109E9000217DD4F82031B4F81C21E387B4F82431B3
:109EA000A287A4F8403031B142F0100243F04003E1
:109EB000A287A4F84030637D2BB1B4F8403043F062
:109EC0008003A4F840302B4BC4E91134236904F11A
:109ED0003801186803F0D0F8237DEBB123691B68C3
:109EE000D3F85422D36823F02003D360A6B9D4F862
:109EF000B0301A68136823F01F031360D4F8B03031
:109F000019680A68D207FCD4597A5A683D238B40F5
:109F100013602046FFF75CFED4F8843013B10123B0
:109F200084F8E930236F13B1012384F8E830124B31
:109F3000DB68E3642046FFF7F1FD236894F8011124
:109F4000DB6B2046984794F832302BB994F8E9300F
:109F500013B10A4B0A4A1A6005A8F9F785FA04A852
:109F6000F9F782FA7AE600BF95A40108CD9B0108B3
:109F7000A59F01080199010870A00020102300206E
:109F80002195010810B53023044683F31188D0F8D9
:109F9000B40002F0A7FC0023C4F8B43083F31188A6
:109FA00010BD0000FFF7EEBF2DE9F74FD0F8EC3001
:109FB00004460D4673B3DFF828B25DB394F801117F
:109FC0002046F9F7F9FA50B1636A43B123F00F0262
:109FD00003F00F03126922FA03F3DB071AD404F12A
:109FE000980840F25532414601A8F9F721FA04F1E8
:109FF0008007402D2A46616E28BF40223846FDF773
:10A00000A3FF1FFA80F98246B9F1000F05D101A81C
:10A01000F9F72AFA03B0BDE8F08F3846FDF79EFE47
:10A02000854228BF054601A8F9F71EFAD4F8EC00CE
:10A0300001F09AF8022003F08BF9D4F8EC00C27C0E
:10A04000002A00F0BC80626BB2F5E13F0FD8B4F893
:10A0500068600336B6B2B6F57A7FA4F8686006D9B0
:10A060000021617503B0BDE8F04F00F071BFFA2028
:10A07000584B42431FFA8AF1B2FBF3F2013291428C
:10A0800001D91FFA82F9302282F31188D4F8B42062
:10A0900011680A6822F01F020A60D4F8B42011681F
:10A0A0000E6816F00106FBD1507A51683D228240BD
:10A0B0000A60606E494604F081F9D4F8B420616EFC
:10A0C0001268454BD160D4F8B4201268C2F80490ED
:10A0D000D4F8B42011682269106940F2564242EA6D
:10A0E00040620A60D4F8B42011680A6842F00102A4
:10A0F0000A6009F10201626B5943B1FBF2F1374A80
:10A1000001F5FA71594588BF114686F3118802207E
:10A1100003F06AF9064670BB302282F31188D4F846
:10A12000B42011680A6822F01F020A60D4F8B42033
:10A130001068016811F00101FBD192F809C0506864
:10A140003D2202FA0CF20260D4F8B420126853687F
:10A1500099453DD9A9EB03031FFA83F9B9F1000F23
:10A1600003D0FDF77DFDC4F80401022003F0E6F8FA
:10A17000002282F31188D4F8EC00C6F3400100F00D
:10A18000E7FEB9F1000F3FF445AF40F2B13241466E
:10A1900001A8F9F74DF949463846FDF713FED4F802
:10A1A0000C214A44C4F80C21D4F810214A44C4F8C4
:10A1B000102101A8A5EB0905F9F756F9FDE6B4F859
:10A1C0006820002A3FF45FAF013AA4F868205AE7FC
:10A1D0008946CAE740420F0080969800A086010099
:10A1E0009F86010013B5D0F840310446CBB900F585
:10A1F000967003F0B7F81823C4F840312369186843
:10A20000019002F047FFB4F84030019823F00803B2
:10A2100004F13801A4F8403002B0BDE8104002F06B
:10A220002BBF02B010BD00002DE9F047044686B0F8
:10A230000D4640F2CA3200F1980101A8F9F7F8F88A
:10A2400094F8283123B1012D02D92046FFF7CAFF27
:10A2500004F180092A4602A94846FDF74BFE4FF05B
:10A260000008824602AD4746C2451FDD2269537988
:10A27000D3B910680268D669D5E90012B047061E46
:10A2800014DB05D0FDF7ECFC3744C4F80401BFB281
:10A29000083531464846FDF795FD55F8043C9E4289
:10A2A00004D108F10108DFE70026F1E7D4F80C310A
:10A2B0003B44C4F80C31D4F810313B44C4F810319D
:10A2C00001A8F9F7D1F806B0BDE8F08770B50446EB
:10A2D0008030FDF743FD0146B8B1637D2046ABB148
:10A2E000FFF762FE94F80131022B0ED1D4F8085129
:10A2F0001DB9FDF7B5FCC4E94205637D4BB1D4F847
:10A300000431A3B1012384F8013170BDFFF78CFF44
:10A31000E8E723691B689A6BD4F80C31C2F58071A9
:10A32000994204D2A3F580731344082BEAD8FDF7B1
:10A3300097FCD4F80831C01A0B4B9842E5D90B4B67
:10A3400022691B680A4998690A4BD21A0A4B921073
:10A350005A430368D2B21B68984723682046DB6BD8
:10A36000BDE870400021184720A107000825002003
:10A37000105D0208385D0208A38B2EBA10B5036A7F
:10A380000446E3B190F80111F9F716F9B8B104F1F8
:10A390006C00FDF7FDFC94F80221D4F8943080B2F3
:10A3A00072B198420BD2226A002384F8023122F063
:10A3B0000F01012302F00F0293409BB20B8310BDEB
:10A3C00010339842FBD9226A012322F00F0102F0D8
:10A3D0000F0284F8023193409BB24B83EFE70000F9
:10A3E00070B5124BC26CDB689A42044619D190F8E2
:10A3F000E83003F0FF0593B100F16C063046FDF73D
:10A40000ADFCD4F818311844C4F818013046FDF7F3
:10A4100093FC94F8023133B92046FFF7AFFF28468A
:10A4200070BD0025FBE71D46F9E700BF70A00020C6
:10A4300038B50D4B0546DB68C06C984210D195F8D5
:10A44000E8306BB105F16C00FDF79AFD044628B1C8
:10A4500095F8023113B92846FFF790FF204601E036
:10A460004FF0FF3038BD00BF70A0002038B590F825
:10A4700000510446FDF7FAFB85F0010504EBC50524
:10A48000C5E93C0194F8003183F0010384F8003100
:10A4900038BD000070B5037D0446002B4FD0D0F8C6
:10A4A000B0301B685D6890F858601A6822F01F028F
:10A4B0001A60D0F8B030C5F140051968ADB2F6B2F7
:10A4C0000A68D207FCD4597A5A683D238B4013603E
:10A4D0002046FFF77DFBADB104EB86062A46F16D01
:10A4E00004F16C00FDF7CAFCD4F81431D4F818213B
:10A4F0002B4415442D1AC4F81431C4F818512046C1
:10A50000FFF7B4FF236D93B104F16C00FDF726FC57
:10A51000B4F8543098420AD3302383F311884FF4AF
:10A520008061206D02F02AFF002383F3118894F8E4
:10A53000023123B12046BDE87040FFF71FBF70BD58
:10A540002DE9FF4700F16C0804464046FDF720FC6A
:10A55000694602464046FDF74FFC6E46814600279D
:10A5600004F5A47AB9450ADD2269537953B9106814
:10A570000268156AD6E90012A847051E03DA04B07E
:10A58000BDE8F087002594F85C313BB1504602F0FD
:10A59000E9FE10F0200F18BF4FF0FF35D4F840311E
:10A5A0005BB929464046FDF74FFCD4F814312B44E3
:10A5B000C4F814312046FFF759FF7368AB4206F127
:10A5C0000806DCD80137CDE730B590F8E93085B022
:10A5D0000446002B53D0D0F8403100F1B8051BB32E
:10A5E00040F2D742294603A8F8F722FF04F59670F7
:10A5F00002F0B8FED4F8403123EA0000C4F840016C
:10A6000078B923691868019002F044FDB4F840302D
:10A61000019843F00803A4F8403004F1380102F037
:10A620002BFD03A8F8F720FF94F82831DBB140F2A6
:10A63000F54204F1D00103A8F8F7FAFE2046FFF72F
:10A640007FFF236D63B104F16C00FDF787FBB4F865
:10A650005430984204D3206D4FF4806102F0A4FE80
:10A6600003A8F8F701FF40F2FD42294603A8F8F7D6
:10A67000DFFE2046FFF72AFE03A8F8F7F5FE05B037
:10A6800030BD0000F8B51E4D0446A36A3BB92B68E7
:10A69000986A03684FF47A719B689847F5E700263B
:10A6A0004FF47A7141F20C0002F09EFE0546FDF770
:10A6B000D7FA831BB3F57A7F2ABF06460027012706
:10A6C00029070AD594F84431C3B1E36C986B013083
:10A6D000B52828BFB52003F09DF994F8E930002B88
:10A6E000DED06A0706D42FB9D4F84031002BD7D07A
:10A6F000EB04D5D52046FFF767FFD1E73C20EAE71A
:10A700000825002008B5FFF7BDFF000037B590F819
:10A71000E830044603B390F82831EBB900F1D001DA
:10A720004FF48B6201A8F8F783FE237DB3B920466E
:10A73000FFF706FF236D63B104F16C00FDF70EFB1C
:10A74000B4F85430984204D3206D4FF4806102F085
:10A750002BFE01A8F8F788FE03B030BDD4F8B03066
:10A76000002BE7D0302383F31188D4F8B0301B6876
:10A770001A68D10738D45D68C5F1400515F0FF05AA
:10A780001DD094F8583004EB83032A46D96D04F1A8
:10A790006C00FDF773FBD4F81431D4F818212B4466
:10A7A00015442D1AC4F81431C4F818512046FFF787
:10A7B0005DFE94F8023113B12046FFF7DFFDD4F8B7
:10A7C000B0301A68136823F01F031360D4F8B03058
:10A7D00019680A68D207FCD4597A5A683D238B401D
:10A7E00013602046FFF7F4F9002383F31188237DDB
:10A7F000002B9FD19BE70000104B70B5104C1D68DB
:10A80000A86A226803689B681AB94FF47A7198475E
:10A81000F6E7A86A0B4E03684FF47A719B68984775
:10A820000B2456F8040B20B190F8E8300BB1FFF779
:10A830006DFF013C14F0FF04F3D1EAE70825002086
:10A84000949A0020689A002038B50446C8060D4640
:10A8500004D5E06910B1022103F09EFD690604D51C
:10A86000A06910B1022103F097FDAA0604D5E069A2
:10A8700010B1012103F090FD2B0606D5A06920B18F
:10A88000BDE83840012103F087BD38BD2DE9F04710
:10A8900003695D7904460E462DB1B1FA81F56D0963
:10A8A0002846BDE8F087C181D3F800809869D8F8C0
:10A8B0005422D2F810A05769D268294602F40059F0
:10A8C0001A7900F097FC2369E0611A79586901212F
:10A8D00000F090FC2369A0611A79D869042100F086
:10A8E00089FC236920621A79186A042100F082FC2D
:10A8F00023686062DB6B94F8011120469847236956
:10A9000016F0010F93F9241000F0868000290CDB6B
:10A910005A4A1268D0690268C9B2156993F82520AD
:10A92000A847E069002873D101252269B00792F990
:10A93000261040F185800029C0F296804F4B92F896
:10A9400027201B68D8690368C9B21B699847A069AA
:10A9500010B1022103F020FD16F0080F18BF0025EA
:10A960007107D4F8243140F1818043F00803C4F822
:10A97000243194F8283147F0080763B9236918682F
:10A980004FF48052182304F59671043002F0B2FCA3
:10A99000012384F82831237D93B1D4F8B0307BB102
:10A9A0001A68136823F01F031360D4F8B0301968D5
:10A9B0000A68D207FCD4597A5A683D238B40136049
:10A9C0000023A38231462046FFF73EFFD8F85432D9
:10A9D0001A69524503D15A69BA423FF461AFB9F1DD
:10A9E000000F03D0DA6822F40052DA60D8F854324B
:10A9F000C3F810A0D8F854325F61B9F1000F3FF4EA
:10AA00004FAFD8F85422D36843F40053D36047E7DC
:10AA1000022103F0C1FC87E7002985DB174A126891
:10AA2000D06993F825200368B2FA82F21B695209B3
:10AA3000C9B29847E06900283FF476AF0121E8E702
:10AA4000002989DB0D4B92F827201B68D869036821
:10AA5000B2FA82F21B695209C9B29847A06900286C
:10AA60003FF47AAF012175E7002575E723F008036D
:10AA700027F00807C4F82431A4E700BF0825002008
:10AA8000004870475C5E020800207047014B0020C0
:10AA900019707047989A0020704700000020704796
:10AAA0007047000003F068BB084609B103F060BBC3
:10AAB0007047000008B5134612780C2AA8BF0C2274
:10AAC00008461A70024904F063F8012008BD00BF6F
:10AAD000107AFF1F1046194603F0EEBB03F0FEBBD1
:10AAE0002DE9F34742F6F8216846F8F787FC53480A
:10AAF00001A9FBF737F9524B05461C6868B9A069F4
:10AB00004E4A03684F491B68984703246846F8F784
:10AB100081FC204602B0BDE8F087019B606B1F33CB
:10AB200023F01F030193036800211B689847019AD3
:10AB300001460746284604F01BF8A3691A68126804
:10AB400038B91846404990472846FBF74DF901248B
:10AB5000DCE73E49184690470026B146019B4B452D
:10AB600023D9606B03685FFA86F85B6841469847B3
:10AB7000824620B92846FBF737F90224C6E7A06AC7
:10AB800003684FF47A711B699847606B036841460C
:10AB9000DB689847013630B9A0692D4903681B6806
:10ABA00042469847E6E7D144D8E7A069234A0368BC
:10ABB00028491E68DFF8A8903B46B047606B0368E1
:10ABC00001215B6998474FF00108A06A03684FF4C0
:10ABD0007A711B699847606B03682A461E69019B5E
:10ABE0003946B0470646A0690368D6B94246D3F84D
:10ABF00000A049460A23D047A06A036864215B6825
:10AC000008F101089847B8F10B0FDED1606B0368BB
:10AC100031465B699847A0690F4903680A221B689F
:10AC2000BFE71B680D499847606B036800215B69AB
:10AC300098472846FBF7D8F8002467E7A01A0208CF
:10AC400008250020745E0208875E02089E5E0208E6
:10AC5000A75E0208B85E0208F45E0208EA5E020817
:10AC6000CB5E02082DE9F04F214B9DB01A7C0F926C
:10AC70005A7C10929A7C1192DA7C12925A7D1F7D36
:10AC800013929A7D1492DA7D159293F818B093F886
:10AC900019A093F81A9093F81B8016AB0C46054642
:10ACA00014491722184604F043FC139A0792149A89
:10ACB0000692159A05920F9A0492109A0392119A8D
:10ACC0000292129A0C4B0897CDE900020026CDE9BA
:10ACD0000989322221462846CDE90BAB8DF86F60F9
:10ACE000F8F7E4FC012084F831601DB0BDE8F08F76
:10ACF000007AFF1F25170208145F020803F0A2BBA9
:10AD00002DE9F0471B4A1C4CDFF87480DFF874A073
:10AD1000DFF8749086B010460F4603F055FB154AD5
:10AD20001649A41A03460094384600F08FFA02F040
:10AD300031FC0446D4B1256AE269A36B059245450E
:10AD4000284614BF661BAAEB0806049303F03CFBDD
:10AD5000DDE90432CDE9010649463846009500F0A8
:10AD600075FA204602F026FC0446E3E706B0BDE88B
:10AD7000F08700BF00010020000700204C5F0208A0
:10AD800000070020002300207F5F0208084600F033
:10AD9000F1B800002DE9F04188B00D4604A805A9DE
:10ADA00003F02EFA1549DFF858800646284600F0D1
:10ADB0004DFA00242746E0B286421CD9CDE9067739
:10ADC00010B1049B03EB441007AA06A902F068FA2D
:10ADD00005990C2262438818D0E901300290079847
:10ADE0000190069800908A589B0A4146284600F038
:10ADF0002DFA0134DFE708B0BDE8F081A45F020856
:10AE0000AF5F020808460AB903F084B9012A01D1EC
:10AE100003F0A6B9022AF7D0012003F0A5B900007B
:10AE200070B50C4615462AB9084603F0A1F92E461E
:10AE3000304670BD104619B9BDE8704003F066B9E0
:10AE400003F064F906460028F2D054F8042CAA4214
:10AE500028BF2A46214603F09BFE204603F088F9CE
:10AE6000E6E7000070B50C4615460026AE4204D257
:10AE7000F9F7EAF8A0530236F8E7EB0704D5F9F73B
:10AE8000E3F82C4404F8010C012070BDF8F7D8BB9E
:10AE900038B5054D00242846013402F0D7FA102CAD
:10AEA00005F12005F7D138BDA09A002082B010B579
:10AEB000914203934FF00003C0E90033C0E902332D
:10AEC00004460174427484BF02744174DDE90301D5
:10AED00084E80300DDE9050104F1080383E80300C9
:10AEE0002046BDE8104002B07047000000207047C7
:10AEF0000F2838B50AD8074B03EB40152846AC6835
:10AF000002F0E6FA14B1AB689C4201D1002038BDD2
:10AF10000120FCE7A09A00200F2938B50446154609
:10AF200010D8094800EB411002F0FEFA55B1074B6A
:10AF30001B683BB1227C02EB420203EB82039A685E
:10AF400001329A6038BD00BFA09A00209C9A002070
:10AF500013B5002304460A4683740191417CFFF730
:10AF6000DBFF019A217C204602B0BDE81040FFF7CC
:10AF7000D3BF00002DE9F04F314E2DED028B336829
:10AF80008BB007461BB9CC20F8F7C4F830602D49C8
:10AF90009FED2D8ADFF8B480384600F057F9002580
:10AFA0004FF00C09336809FB05F4EAB2195903EBB9
:10AFB000040C31B9DCF8041019B9DCF808100029C8
:10AFC00036D0191991ED007A53F804E0DCF804004A
:10AFD000DCF8081007910EEB0001013107EE901A22
:10AFE000B8EE477AF8EE677A27EE087ADCF804A024
:10AFF00053F804B0C7EE277A02F00703D2080132F3
:10B000000993089217EE900AF5F768FA079B0093E8
:10B01000CDE90401DDE90823CDE901AB414638461D
:10B0200000F014F9336800221A51336823445A603F
:10B030000135102DB6D10BB0BDEC028BBDE8F08F01
:10B040009C9A0020686002080000C8426F600208F5
:10B05000D0E900031847000038B50446007C0F28EB
:10B060000FD83F4D05EB4013D96951B1A14208D02B
:10B0700018461430FFF7ECFF237C05EB4315002343
:10B08000EB61607C0F280FD8354D05EB4013D96973
:10B0900051B1A14208D018461430FFF7D9FF637CA4
:10B0A00005EB43150023EB61227C0F2A04D82C4BBF
:10B0B00003EB4213DB693BB1627C0F2A26D8284B95
:10B0C00003EB4213DB690BBB21462046FFF7C0FFB1
:10B0D000237C0F2B0BD8224AD4E9020102EB431345
:10B0E000143383E80300237C02EB4312D461637CB6
:10B0F0000F2B0BD81A4AD4E9020102EB4313143385
:10B1000083E80300637C02EB4312D46115480268B4
:10B11000D2B1237C0F2B09D8E57C03EB43039900C4
:10B1200002EB83039DB1535801335350637C0F2BC3
:10B130000AD80268E07C03EB4303990002EB830327
:10B1400048B15358013353500123A37438BD5A6892
:10B1500001325A60EAE75A6801325A60F4E700BFE8
:10B16000A09A00209C9A002038B50446007CFFF786
:10B17000BFFE0546607CFFF7BBFE002D08BF0546FD
:10B18000E5742046BDE83840FFF766BF044B112246
:10B190000021013AC3E9051103F12003F9D17047F9
:10B1A000A09A002070470000704700007047000020
:10B1B00000207047704700000020704782B002A94D
:10B1C000002001E90C0002B0704700000020704729
:10B1D00000797047002070470020704700207047BA
:10B1E0007047000001207047014B0360704700BFAB
:10B1F000AC6002087047000070B5467B05460EBB88
:10B200004468836804EB8404A40804F50074E21A1B
:10B21000914288BFCC180C4B29681B68D86A036818
:10B22000621C1B6D984718B901232B73304670BD03
:10B23000AB68C5E90004E21A0021184403F0B6FC2B
:10B240000126F3E70026F1E7082500200EB470B5CB
:10B25000017B85B0044619BBD0E901239A421BD07B
:10B26000134B1E680AADD4E9012120680095521ADB
:10B27000099B03950144F06AF8F7F8F900280FDB01
:10B28000D4E90123D21A82420FD8411C2046FFF78D
:10B29000B3FF0028E7D103E0FFF7AEFF0028DFD1BE
:10B2A00005B0BDE8704003B070471844A060F7E7F0
:10B2B000082500202DE9F041456A15B94162BDE835
:10B2C000F0818B6823F06047C3F38A464FEAD37E50
:10B2D000C3F3807816EA230638BF3E46AC462B46B9
:10B2E0009A68BEEBD27F22F060440AD0002A18DAB6
:10B2F000A40CB44217D19D420FD10D60DEE7134676
:10B30000EEE7A74207D102F08044C2F380724245C3
:10B310000BD054B1EFE708D2EDE7CCF800100B608A
:10B32000CDE7B44201D0B442E5D81A689C46002A61
:10B33000E5D11960C3E700002DE9F047089D01F051
:10B3400007044FEAD508224405F0070500EBD100B9
:10B350004FF47F49944201D1BDE8F08704F007071C
:10B3600005F0070A57453E4638BF5646C6F108065F
:10B37000111B8E4228BF0E46E10808EBD50E415C3A
:10B3800013F80EC0B94029FA06F721FA0AF1FFB204
:10B390008CEA010147FA0AF739408CEA010C03F8FC
:10B3A0000EC034443544D5E780EA0120082341F239
:10B3B000210201B24000002980B203F1FF33B8BF7F
:10B3C000504013F0FF03F4D17047000038B50C462D
:10B3D0008D18A54200D138BD14F8011BFFF7E4FF1A
:10B3E000F7E7000042684AB11368436043898189E6
:10B3F00001339BB29942438138BF83811046704725
:10B4000070B588B0202204460D466846002103F03E
:10B41000CDFB20460495FFF7E5FF024658B16B4689
:10B42000054608AE1C4603CCB4422860696023463A
:10B4300005F10805F6D1104608B070BD082817D9E7
:10B4400009280CD00A280CD00B280CD00C280CD0C2
:10B450000D280CD00E2814BF4020302070470C203F
:10B460007047102070471420704718207047202024
:10B4700070470000082817D90C280CD910280CD9BF
:10B4800014280CD918280CD920280CD930288CBFA6
:10B490000F200E207047092070470A2070470B20AC
:10B4A00070470C2070470D20704700002DE9F843CD
:10B4B000078C072F04461ED9D0E9029800254FF6C5
:10B4C000FF73C5F12006A5F1200029FA05F108FA5D
:10B4D00006F628FA00F031430143C9B21846FFF7D7
:10B4E00063FF0835402D0346EBD1E1693A46BDE8DC
:10B4F000F843FFF76BBF4FF6FF70BDE8F88300001D
:10B5000010B54B6823B9CA8A63F30902CA8210BD19
:10B5100004691A681C600361C38A013BC3824A60E4
:10B52000EFE700002DE9F84F1D46CB8A0F46C3F325
:10B5300009010D29814692460B4630D00020AAB25F
:10B5400007F11A049EB20C2E1FFA80F80FD890450E
:10B5500003F1010306D3FB8A0A4462F30903FB8269
:10B5600001201AE01AF80060E6540130EAE790453D
:10B57000F1D2A1F10D0B24237C68BBFBF3F203FB9A
:10B5800012BB1FFA8BF6002C46D14846FFF72AFF64
:10B59000044638B978606FF00200BDE8F88F4FF0CC
:10B5A0000008E6E7002606607860ADB24FF0000BB9
:10B5B000454510D90AEB0803221D13F8011B9155CC
:10B5C000B1B208F1010823291FFA88F82CD04545AB
:10B5D00006F10106F1D8FB8AC3F30902154465F3AD
:10B5E0000903BCE7013292B21C462368002BF9D153
:10B5F000A5F10D030B442421B3FBF1F301339BB2FE
:10B600009A42D2D2BBF1000FCFD14846FFF7EAFEF3
:10B6100020B9C4F800B0BEE70122E6E7C0F800B0E8
:10B620005E4620600446C0E74545D4D94846FFF74A
:10B63000D9FE08B92060AEE7C0F800B0002620604F
:10B640000446B5E72DE9F04F2DED028B1C4683B083
:10B650005B69019207468846002B00F0B280238C7C
:10B660002BB1E269002A00F0AC80072B3AD807F131
:10B670000C00FFF7B7FE054638B96FF002063046FA
:10B6800003B0BDEC028BBDE8F08F2822002103F04F
:10B690008DFA228CE16905F1180003F079FA208C0B
:10B6A000013080B2FFF7E6FEFFF7C8FE013880B236
:10B6B0002084013085F820006369228C1B782A449D
:10B6C00003F01F0363F03F0348F000411376A960C5
:10B6D000D4E90A232946C5E904233846FFF7EAFDE1
:10B6E0000126CCE702339BB20722C18A0633B3FBA3
:10B6F000F2F3828A521A9BB292B29342BDD800F101
:10B700000C034FF0000908EE103A4FF0800ACB46C8
:10B710004E4618EE100AFFF765FE05460028ACD02D
:10B720002822002103F042FABBF1000F3CD1019B1B
:10B730002B83022205F1180E1FFA82FC0CF1010086
:10B74000BCF1060F218C80B201D88B452ED3FFF7B8
:10B7500091FEFFF773FE62691278013802F01F0252
:10B760008B4508BF4FF0400A42EA491215FA80F1B2
:10B770004AEA020A013048F0004281F818A0AA60A3
:10B7800085F82000D4E90A01C5E9040129463846B4
:10B79000FFF790FD228C01365A4536B289F0010937
:10B7A0004FF0000AB5D16AE70022C3E7E1690BF167
:10B7B000010311F80B100EF802101FFA83FB01327F
:10B7C000BAE76FF001065AE7F8B515460E46302283
:10B7D000002104461F4603F0E9F9B5F5201F069B3A
:10B7E000636038BF2822079BA76028BF4FF6FF720F
:10B7F000A36238BFB5FBF2F2E66197B204F1100024
:10B8000000239A4206D800230360A782E3822383A1
:10B81000E360F8BD0660013330462836F1E70000EA
:10B8200003781BB94BB2002BC8BF017070470000F2
:10B8300000787047F8B50C46C969074611B9238CE2
:10B84000002B37D1257E1F2D34D8387828BB228C89
:10B85000072A2CD8268A36F003032BD14FF6FF7027
:10B86000FFF7B4FD20F001003102400441EA056118
:10B87000400C41EA40254FF6FF72234629463846E0
:10B88000FFF7E0FE002807DD626913780133DBB2C1
:10B890001F2B88BF00231370F8BD218A2D0645EAAF
:10B8A000012505432046FFF701FE0246E5E76FF05C
:10B8B0000300F1E76FF00100EEE700002DE9F04131
:10B8C000D36905460C4616460BB9138C5BBB377E15
:10B8D0001F2F28D895F80080B8F1000F26D03046E9
:10B8E000FFF7E4FD3378210241EAC33141EA080160
:10B8F000338A41EA076141EA03410246334641F097
:10B9000080012846FFF79EFE00280ADD3378012BD0
:10B9100007D1726913780133DBB21F2B88BF002374
:10B920001370BDE8F0816FF00100FAE76FF00300DB
:10B93000F7E70000406A00B108307047436A1A68B0
:10B94000426202691A600361C38A013BC382704785
:10B950002DE9F041D0F820802A4E14461D4641467C
:10B96000002721B9416A0B4661BBBDE8F081D1E9EE
:10B970000232E31A65EB02029E4277EB02031ED20B
:10B98000036A8B420DD1FFF7BBFD036A1B6803629C
:10B9900003690B60C38A0161016A013BC382884667
:10B9A000DFE7FFF7ADFD0B68C8F8003003690B60F7
:10B9B000C38A0161013BC382D8F80010D1E78846F1
:10B9C0000968CEE7D1E90476A742AE410A680BD2F6
:10B9D000466A8E420BD1036942620B60C38A0161E1
:10B9E000416A013BC3820A460B461146BCE71A6016
:10B9F00002690A60C28A0161013AC2821A68194664
:10BA0000F2E700BF80841E002DE9F04F8BB00D4699
:10BA1000DDF8509014469B468046002800F01B81BC
:10BA2000B9F1000F00F01781531E3F2B00F2138174
:10BA3000012A03D1BBF1000F40F00D810023CDE9B5
:10BA40000833B8F81430B5EBC30F4FEAC30703D37C
:10BA500000200BB0BDE8F08F2B199F42D8F80C30B6
:10BA60003ABF7F1BFFB227461BB9D8F81030002B16
:10BA70007CD0672D4ED8C5F16806B7424FF0000361
:10BA80002CBFF6B23E4600932946D8F8080008AB12
:10BA90003246FFF751FCA7EB060A35445FFA8AFAF3
:10BAA000B8F8143003F100530D3BDB000493D8F8D1
:10BAB0000C3003936821039B13B1BAF1000F2CD112
:10BAC000D8F8100040B1BAF1000F05D0009608ABCD
:10BAD0005246691AFFF730FC38B2002FB8D066071B
:10BAE0000AD00AAB03EBD401624211F8083C02F021
:10BAF0000702134101F8083C082C3ED9102C40F2F3
:10BB0000B780202C40F2B980BBF1000F00F09E807E
:10BB1000082336E0BA460026C2E7049BB3F5907FBF
:10BB200028BF4FF4907306930B44AB42059314D98E
:10BB30005A1B03980096924534BF5246D2B2691AF6
:10BB400008AB04300792FFF7F7FB079A1644AAEBFD
:10BB5000020A1544F6B25FFA8AFA049B069A05991E
:10BB60009B1A0493039B1B680393A4E70093D8F8E4
:10BB7000080008AB3A462946ACE7BBF1000F13D0EA
:10BB80000123B4EBC30F6CD0082C12D89DF82030E1
:10BB9000621E23FA02F2D50706D54FF0FF3202FAF1
:10BBA00004F423438DF820309DF8203089F80030CC
:10BBB0004FE7102C12D8BDF82030621E23FA02F293
:10BBC000D10706D54FF0FF3202FA04F42343ADF853
:10BBD0002030BDF82030A9F800303AE7202C0FD8EB
:10BBE0000899631E21FA03F3DA0705D54FF0FF32F7
:10BBF00002FA04F40C430894089BC9F8003028E7C3
:10BC0000402C2BD0DDE90865611EC4F12102A4F1AE
:10BC1000210326FA01F105FA02F225FA03F3114392
:10BC20001943CB0712D50122A4F12003C4F120014E
:10BC300002FA03F322FA01F1A240524243EA01035D
:10BC400063EB430332432B43CDE90823DDE90823AB
:10BC5000C9E90023FDE66FF00100FAE66FF0080085
:10BC6000F7E6082CA0D9102CB3D9202CEED8C3E7C6
:10BC7000BBF1000FADD0022383E7BBF1000FBBD0B7
:10BC800004237EE730B5012A144638BF0124402C36
:10BC900085B028BF40240025012ACDE9025518D8D7
:10BCA0001B788DF8083063070AD004AB03EBD4058A
:10BCB000624215F8083C02F00702934005F8083C80
:10BCC000009103462246002102A8FFF735FB05B08C
:10BCD00030BD082AE4D9102A03D81B88ADF80830F3
:10BCE000E1E7202A8DBFD3E900231B680293CDE949
:10BCF0000223D8E710B5CB681BB98B600B618B8230
:10BD000010BD04691A681C600361C38A013BC382C9
:10BD1000CA60F0E703460A8B486918609A801846A3
:10BD20007047000082B08DED010A019820F00043B9
:10BD3000B3F1FF4F08D31BD047F6FF73000C00F49C
:10BD40000040184302B070470B4BDFED0C7A034004
:10BD500007EE103A67EE277A17EE903A03F5805314
:10BD6000B3F1786F28BF4FF07863C3F34F33E5E743
:10BD70004FF4F843E2E700BF00F0FF7F00008007C8
:10BD800003064CBFC0F3C0300220704708B502461E
:10BD9000FFF7F6FF022806D15306C2F30F2001D1A8
:10BDA00000F0030008BDC2F30740FBE72DE9F04FA8
:10BDB00093B0CDE903230A6804461046FFF7E0FF7D
:10BDC000022814BFC2F306260026002A0D4682462A
:10BDD00080F2FD8112F0C04940F0F981097E00290E
:10BDE00000F0F581022803D02378B34240F0F281BD
:10BDF000C2F304630693104602F07F030593FFF736
:10BE0000C5FF059B29444FEA834848EA0A4848EAA7
:10BE10004668CE7B00230022CDE90823F309834640
:10BE200048EA0008029367D0059B009302466768C2
:10BE3000534608A92046B847002800F0CE81276A5B
:10BE40004FB9414604F10C00FFF7DAFA074690B902
:10BE50006FF0020054E03B6998450DD03F68002F19
:10BE6000F9D1414604F10C00FFF7CAFA0746002851
:10BE7000EED0236A3B60276297F817C006F01F08D0
:10BE8000CCF3840CACEB08001FFA80FE0028B8BF8E
:10BE90000EF12000A8EB0C031FFA83FED7E9022164
:10BEA000B8BF00B2002B0793BEBF0EF120031BB238
:10BEB000079352EA010338D0039BDFF828E39A1A6C
:10BEC000049B4FF0000C63EB010196457CEB0103F2
:10BED0002BD36B7E97F81AE0734519D1029B002B88
:10BEE00079D0012821DC7868F8B9DFF8F4C29445EC
:10BEF00070EB010316D337E0276A27B96FF00C0007
:10BF000013B0BDE8F08F3B699845B5D03F68F4E7C2
:10BF1000B34890427CEB010301D30020F0E7029B81
:10BF2000002BFAD0079B0F2B17DCFA7DB30002F031
:10BF3000030203F07C031343FB7539462046FFF7E9
:10BF4000DFFA6B7EBB76029B3BB9FB7DC3F38402B9
:10BF5000013262F38603FB75D0E76A7EBB7E9A42AC
:10BF6000DBD1029B002B36D0B309022B33D0039BCD
:10BF7000BB60049BFB60142200210DA802F016FE9A
:10BF8000039B0A93049B0B9305F110030C932B7EE8
:10BF9000ADF83EB0013BDBB2ADF83C30069B8DF80E
:10BFA0004230059B8DF8433094F82C308DF840A03A
:10BFB00083F001038DF844308DF84180A3680AA90D
:10BFC00020469847FB7DC3F38403013303F01F032E
:10BFD0009B02FB82A1E7FB7DC6F34012B2EBD31FAD
:10BFE00040F00281C3F38403434540F00081029A8C
:10BFF0002B7EB609002A53D016F0010663D1032B1D
:10C0000040F2F880039BBB60049BFB60FB8A66F3F5
:10C010000903FB822B7E05F11206033BDBB232469D
:10C02000394604F10C00FFF77DFA00280CDA394696
:10C030002046FFF765FAFB7DC3F38403013303F069
:10C040001F039B02FB8203E7DDE908842B8A3B8305
:10C050004FF6FF73C9F12000A9F1200228FA09F177
:10C0600004FA00F0014324FA02F211431846C9B25F
:10C07000FFF79AF909F10809B9F1400F0346E9D130
:10C08000B8822A7E033AD2B23146FFF79FF9FB7D90
:10C09000B882DA43C2F3C01262F3C713FB753CE700
:10C0A0008EB905F11006013BDBB23246394604F188
:10C0B0000C00FFF737FA0028B9DB2A7EB88A013A6C
:10C0C000D2B23146E1E7F98AC1F30901013B0C29FB
:10C0D000DAB25DD805F11000002307F11B069A4281
:10C0E00008D910F801CB06F801C0013101330D2940
:10C0F000DBB2F4D103990A9104990B91934207F1B1
:10C100001B010C9138BF103379680D9134BF55FA7B
:10C1100083F300230E93FB8AADF83EB0C3F309030B
:10C120001A44069B8DF84230059B8DF8433094F8F5
:10C130002C30ADF83C2083F001038DF8443000230F
:10C140008DF840A08DF841807B602A7EB88A013A44
:10C1500005F11001FFF73AF93B8BB882834203D116
:10C16000A3680AA92046984720460AA9FFF7C2FDFE
:10C17000FB7DBA8AC3F38403013303F01F039B02E0
:10C18000FB823B8B9A420CBF00206FF01000B7E699
:10C190007B68002BAED00D2001E0243033461E68B2
:10C1A000002EFAD1091A081D05F11006184401EBFA
:10C1B000090CBCF1230F5FFA89F39BD89A4299D9F5
:10C1C00016F8013B00F8013B09F10109EFE76FF0B8
:10C1D000090095E66FF00A0092E66FF00B008FE61B
:10C1E00040420F0080841E006FF00D0088E66FF063
:10C1F0000E0085E66FF00F0082E600BFEFF30983C3
:10C2000005494A6B22F001024A63683383F30988C7
:10C21000002383F31188704700EF00E0302080F3A3
:10C22000118862B60C4B0D4AD96821F4E06109040B
:10C23000090C0A43DA60D3F8FC20094942F0807205
:10C24000C3F8FC200A6842F001020A602022DA7773
:10C2500083F82200704700BF00ED00E00003FA05FC
:10C26000001000E010B5302383F311880E4B5B689B
:10C2700013F4006314D0F1EE103AEFF30984683C34
:10C280004FF08073E361094BDB6B236684F309880D
:10C2900001F050FA10B1064BA36110BD054BFBE74E
:10C2A00083F31188F9E700BF00ED00E000EF00E044
:10C2B000CF100108D210010810B50D4C204600F037
:10C2C000F1FC0C4A0023C4E906230B4B23620B4B01
:10C2D0005A6A42F480725A625A6A22F480725A622E
:10C2E000BDE810405B6A0621122000F0ADBC00BF23
:10C2F000C09C002000200140162C020000380240A3
:10C3000010B50378012B044623D1124B984213D168
:10C310000346114A0621082000F08EFA03680F4AEE
:10C32000E0619A600E4B5A6C42F480725A645A6E05
:10C3300042F480725A665B6E0A4A536803F4400303
:10C3400043F480335360A36900225A609A6001224B
:10C350009A6010BDC09C002029C401084C200140F7
:10C3600000380240002301400269016A137830B5A9
:10C37000C5682BB1012D94BF41F4807141F48471E3
:10C38000C36984681B68DC60548865435D6019601C
:10C39000196841F001011960836900211960516930
:10C3A000D96091691961918B5962D18B9962116A37
:10C3B000013C41EA0454516ADC621963916A596391
:10C3C000D168126941F0806141F480715960510077
:10C3D00043BF22F0804121F0020140F2033042F4D9
:10C3E000407245BF0143024342F0010299609A60E6
:10C3F00030BD0000C16910B50C68236823F01F032D
:10C400002360226812F00102FBD14C68497A3D2377
:10C410008B40236083695A609A6822F080429A6058
:10C4200001229A6010BD000011F00C0F10B50446F7
:10C430001CD0FFF7DFFF03699B6833B10522027050
:10C44000012198472378052B03D102232370002371
:10C450002361302383F311884FF0FF3104F114007E
:10C4600001F0FCFA002383F311880FE003696BB13C
:10C470008A0620D51A7852B15B683BB1042202705B
:10C4800098472378042B01D10323237010BDFFF7B5
:10C49000B1FF03695B682BB10422027098472378CF
:10C4A000042B03D10223237000232361302383F361
:10C4B00011880021D2E7CA06E8D55B68002BE5D0D9
:10C4C000BDE810401847000038B51B4A1B4C1368E4
:10C4D00000211160226952B313F0200504D02278A4
:10C4E000032A14BF0D460225DB071ED545F00405BF
:10C4F0001248FFF77FFF23699B6833B10522227042
:10C50000294698472378052B03D102232370002363
:10C510002361302383F3118809484FF0FF3101F084
:10C520009DFA002383F3118801E0002DE0D1BDE8DE
:10C530003840FFF797BE00BF00200140C09C00209C
:10C54000D49C002008B5074B074A196801F03D014B
:10C55000996053680BB190689847BDE80840FFF7B1
:10C5600081BE00BF00600240E49C002008B5084B7B
:10C570001968890901F03D018A019A60054AD3686A
:10C580000BB110699847BDE80840FFF76BBE00BFCC
:10C5900000600240E49C002008B5084B1968090CB3
:10C5A00001F03D010A049A60054A53690BB1906994
:10C5B0009847BDE80840FFF755BE00BF0060024045
:10C5C000E49C002008B5084B1968890D01F03D0175
:10C5D0008A059A60054AD3690BB1106A9847BDE88D
:10C5E0000840FFF73FBE00BF00600240E49C00200F
:10C5F00008B5074B074A596801F03D01D960536AF5
:10C600000BB1906A9847BDE80840FFF72BBE00BF0A
:10C6100000600240E49C002008B5084B5968890975
:10C6200001F03D018A01DA60054AD36A0BB1106B53
:10C630009847BDE80840FFF715BE00BF0060024004
:10C64000E49C002008B5084B5968090C01F03D0135
:10C650000A04DA60054A536B0BB1906B9847BDE84A
:10C660000840FFF7FFBD00BF00600240E49C0020CF
:10C6700008B5084B5968890D01F03D018A05DA605B
:10C68000054AD36B0BB1106C9847BDE80840FFF723
:10C69000E9BD00BF00600240E49C002008B5074BE4
:10C6A000074A196801F03D019960536C0BB1906C19
:10C6B0009847BDE80840FFF7D5BD00BF00640240C1
:10C6C000E49C002008B5084B1968890901F03D0178
:10C6D0008A019A60054AD36C0BB1106D9847BDE88A
:10C6E0000840FFF7BFBD00BF00640240E49C00208B
:10C6F00008B5084B1968090C01F03D010A049A605D
:10C70000054A536D0BB1906D9847BDE80840FFF79F
:10C71000A9BD00BF00640240E49C002008B5084B9E
:10C720001968890D01F03D018A059A60054AD36DAB
:10C730000BB1106E9847BDE80840FFF793BD00BFEE
:10C7400000640240E49C002008B5074B074A596882
:10C7500001F03D01D960536E0BB1906E9847BDE872
:10C760000840FFF77FBD00BF00640240E49C00204A
:10C7700008B5084B5968890901F03D018A01DA6062
:10C78000054AD36E0BB1106F9847BDE80840FFF71C
:10C7900069BD00BF00640240E49C002008B5084B5E
:10C7A0005968090C01F03D010A04DA60054A536F2B
:10C7B0000BB1906F9847BDE80840FFF753BD00BF2D
:10C7C00000640240E49C002008B5084B5968890DBC
:10C7D00001F03D018A05DA60054AD36F13B1D2F842
:10C7E00080009847BDE80840FFF73CBD0064024068
:10C7F000E49C00200D4930B500230D4C0B600C2546
:10C800001A4605FB03F00059026001EBC300013337
:10C81000102B4260F5D1074A4FF0FF339360D3608D
:10C82000C2F80834C2F80C3430BD00BFE49C0020CC
:10C83000F0600208006002400F28F8B549D8DFF820
:10C84000A0C00125DCF8007085402F4241D1224C68
:10C850000CEBC00ECEE901230C262F43EBB206FBF6
:10C860000046CCF800704BB11C4B1F6B47F400170F
:10C870001F631F6D47F400171F651B6D15F47F4F75
:10C8800009D0164B1D6B45F480051D631D6D45F4E5
:10C8900080051D651B6D0C234343E3581D6825F07F
:10C8A0001F051D601D6815F00105FBD10C2707FB56
:10C8B00000403D2490F809C0476804FA0CF43C603D
:10C8C00021241D605C6112B1C07A00F0BDF93046D0
:10C8D000F8BD0026FBE700BFF06002080038024008
:10C8E000E49C002010B50446C07A00F0C3F9114959
:10C8F000A27A012303FA02F20B6823EA0203DAB2F6
:10C900000B604AB90C4A116B21F400111163116DCF
:10C9100021F400111165126D13F47F4F09D1064BFC
:10C920001A6B22F480021A631A6D22F480021A65CF
:10C930001B6D10BDE49C0020003802400023054A16
:10C9400019460133102BC2E9001102F10802F8D197
:10C95000704700BF689D00202DE9F74FC2F3C31355
:10C9600002F0030AC2F38009C2F3C108C2F3411EF8
:10C970000193574600224FF00F0BCB0737D5019C90
:10C9800002F007039B0004FA03FC0125446895406C
